:020000040000FA
:1000000047EF4AF0FFFFFFFF08D0FFFFFFFFFFFFB2
:10001000FFFFFFFFFFFFFFFF00D0E0CF02F1010174
:10002000D8CF01F1E8CF00F181509EB03AEC3BF01F
:10003000F2B421EC3BF0A1B236EC3BF09EBAE1EC1D
:100040003AF0F2B20FEC3BF0F0B015EC3BF000C12F
:10005000E8FF01C1D8FF02C1E0FF1000FFFFFFFF72
:10006000FFFFFFFFFFFFFFFFFFFFFFFFFFFFFFFFA0
:10007000FFFFFFFFFFFFFFFFFFFFFFFFFFFFFFFF90
:10008000FFFFFFFFFFFFFFFFFFFFFFFFFFFFFFFF80
:10009000FFFFFFFFFFFFFFFFFFFFFFFFFFFFFFFF70
:1000A000FFFFFFFFFFFFFFFFFFFFFFFFFFFFFFFF60
:1000B000FFFFFFFFFFFFFFFFFFFFFFFFFFFFFFFF50
:1000C000FFFFFFFFFFFFFFFFFFFFFFFFFFFFFFFF40
:1000D000FFFFFFFFFFFFFFFFFFFFFFFFFFFFFFFF30
:1000E000FFFFFFFFFFFFFFFFFFFFFFFFFFFFFFFF20
:1000F000FFFFFFFFFFFFFFFFFFFFFFFFFFFFFFFF10
:10010000001210180606080A0A0C0606080A060A53
:1001100006060808060E06060A0A08140C0A060A4D
:1001200008060606101010101010101010101010F5
:1001300010101010101010101010101010101010BF
:10014000101010101014161416120C140E1414148F
:100150000E180A0608080A060C0A08080808060607
:10016000040A0C120A0A0A060A0E140808061212D9
:10017000040E140806100E0C0606080606060606EF
:10018000080804040A16161614080A080806060ABF
:100190000808040A0C140A0C0A141010101010108D
:1001A000101010101010101010101010101010104F
:1001B00010101010101010101010140E0E0E080851
:1001C00006141414141414141414141414141414FD
:1001D00014141414141414141414141414141414DF
:1001E0001414141414141414141414140A0A0A08F9
:1001F0000808080E0614100A100C06060606060863
:10020000020E0E080808060606060A0A0408040E6E
:100210001412140E0A0E0C100E0A0A0A0E0C10000C
:10022000FFFFFFFFFFFFFFFFFFFFFFFFFFFFFFFFDE
:10023000FFFFFFFFFFFFFFFFFFFFFFFFFFFFFFFFCE
:10024000FFFFFFFFFFFFFFFFFFFFFFFFFFFFFFFFBE
:10025000FFFFFFFFFFFFFFFFFFFFFFFFFFFFFFFFAE
:10026000FFFFFFFFFFFFFFFFFFFFFFFFFFFFFFFF9E
:10027000FFFFFFFFFFFFFFFFFFFFFFFFFFFFFFFF8E
:10028000FFFFFFFFFFFFFFFFFFFFFFFFFFFFFFFF7E
:10029000FFFFFFFFFFFFFFFFFFFFFFFFFFFFFFFF6E
:1002A000FFFFFFFFFFFFFFFFFFFFFFFFFFFFFFFF5E
:1002B000FFFFFFFFFFFFFFFFFFFFFFFFFFFFFFFF4E
:1002C000FFFFFFFFFFFFFFFFFFFFFFFFFFFFFFFF3E
:1002D000FFFFFFFFFFFFFFFFFFFFFFFFFFFFFFFF2E
:1002E000FFFFFFFFFFFFFFFFFFFFFFFFFFFFFFFF1E
:1002F000FFFFFFFFFFFFFFFFFFFFFFFFFFFFFFFF0E
:100300000000010F0019010F0002010F4102010F4F
:100310004102010F1423010F1441010F1423010F97
:10032000145F010F147D010F14B9010F7302010F47
:100330000018010F0000010F3202010F0A1E010F09
:100340000A37010F0A50010F0A69010F0A82010FD3
:100350001423010F2041010F205F010F209B010F8B
:100360000600010F3702010F0E02010F2802010FD4
:100370003202010F1423010F6400010F6419010FF1
:10038000644B010F6464010F0000010F2823010F6B
:100390002823010F2823010F2823010F2823010FF1
:1003A0002823010F2823010F2823010F2823010FE1
:1003B0002823010F2823010F2823010F2823010FD1
:1003C0002823010F2823010F2823010F2823010FC1
:1003D0002823010F2823010F2823010F2823010FB1
:1003E0002823010F2823010F2823010F2823010FA1
:1003F0002823010F2823010F2823010F2823010F91
:100400002823010F2823010F2823010F0023010FA8
:100410000041010F005F010F007D010F009B010FE4
:1004200000B9010F00D7010F0023010F0041010F98
:10043000005F010F007D010F009B010F00B9010F4C
:1004400000D7010F6696010F0000010F6CD8010F55
:100450006CD8010F6400010F0000010F0000010FB4
:100460000000010F0000010F0000010F0000010F4C
:100470000000010F0000010F0000010F0000010F3C
:100480000000010F2802010F1423010F147D010F3A
:10049000557D010F557D010F557D020F557D010FD3
:1004A0000000010F0A02010F0000010F0000010F00
:1004B0001423010F1441010F1402010F0000010F5A
:1004C000145F010F0A02010F0009010F557D020F91
:1004D0000012010F001B010F0024010F002D010F5E
:1004E0000036010F6432010F6419010F6432010FED
:1004F000644B010F6464010F6400010F6419010F64
:100500001441010F4141010F4141010F6432010FBC
:100510000A00010F0A19010F0A32010F0A4B010FDD
:100520006432010F557D010F6978010F693C010F9D
:100530004102010F149B010F2A48010F3C02010FD9
:100540003460010F3478010F644B010FA07D010F5F
:100550000008010F0227010F0230010F557D010F26
:100560001441010F2823010F2823010F2823010F15
:100570002823010F2823010F2823010F2823010F0F
:100580002823010F2823010F2823010F2823010FFF
:100590002823010F2823010F2823010F2823010FEF
:1005A0002823010F2823010F2823010F2823010FDF
:1005B0002823010F2823010F2823010F2823010FCF
:1005C0002823010F2823010F2823010F2823010FBF
:1005D0002823010F2823010F2823010F2823010FAF
:1005E0002823010F0D02010F145F010F0002010FFC
:1005F0000230010F0000010F0000010F0000010F89
:100600000023010F0041010F005F010F007D010F6A
:10061000009B010F00B9010F00D7010F0023010F4C
:100620000041010F005F010F007D010F009B010FD2
:1006300000B9010F00D7010F0023010F0041010F86
:10064000005F010F007D010F009B010F00B9010F3A
:1006500000D7010F0023010F0041010F005F010FC0
:10066000007D010F009B010F00B9010F00D7010FA2
:100670000023010F0041010F005F010F007D010FFA
:10068000009B010F00B9010F00D7010F0023010FDC
:100690000041010F005F010F007D010F009B010F62
:1006A00000B9010F00D7010F0A02010F557D010F9C
:1006B000020C010F6419010F6400010F6400010FA7
:1006C0006419010F6400010F020C010F6464010F33
:1006D0001441010F021E010F147D010F1E02010FB4
:1006E0001423010F6419010F6432010F644B010FD1
:1006F0006464010F6400010F6432010F0000000FF9
:100700001423010F2802010F6923010F6923010F30
:100710006923010F0101010F41A8010F0730010BEF
:100720007887010F0227010F00D8010F0A08010F77
:100730000A10010F0000010F1802010F0023010F22
:100740000041010F005F010F007D010F145F010FD9
:100750001441010F145F010F147D010F149B010F51
:100760006432010F6400010F5A36010F145F010F4C
:10077000147D010F149B010FFFFFFFFFFFFFFFFF21
:10078000FFFFFFFFFFFFFFFFFFFFFFFFFFFFFFFF79
:10079000FFFFFFFFFFFFFFFFFFFFFFFFFFFFFFFF69
:1007A000FFFFFFFFFFFFFFFFFFFFFFFFFFFFFFFF59
:1007B0004275696C64696E67204D443220486173EC
:1007C000687D506C6561736520576169742E2E2EAB
:1007D0007D7D4865696E72696368735765696B6191
:1007E0006D70204F535443327D7D4D656E753F7D56
:1007F0004D656E753A7D4C6F67626F6F6B7D4761BB
:10080000732053657475707D5365742054696D65EC
:100810007D7D5265736574204D656E757D7D536574
:100820007475707D457869747D7D576169742E2E6D
:100830007D7D4D443220486173683A7D4465736123
:10084000747D496E746572666163657D537461720F
:10085000747D446174617D7D4865616465727D7DF0
:1008600050726F66696C657D446F6E652E7D436165
:100870006E63656C2052657365747D7D54696D652A
:100880003A7D446174653A7D53657420486F757292
:10089000737D52657365742E2E2E7D7D4C6F67625D
:1008A0006F6F6B7D437573746F6D2046756E6374E7
:1008B000696F6E7320497D7D5265736574204D6547
:1008C0006E757D7D5365742054696D653A7D4D6FFD
:1008D00072657D7D4465636F706C616E7D7D47617F
:1008E000736C6973747D4D6F72657D7D4578697435
:1008F0007D7D4E6F466C797D5374617274204469BE
:100900007665205B636D5D7D456E64204469766528
:100910002020205B636D5D7D456E642044656C61C5
:10092000792020205B735D7D506F776572204F6664
:10093000662020205B735D7D5072652D6D656E7540
:10094000202020205B735D7D76656C6F6369747910
:100950005B6D2F6D696E5D7D57616B652D757020C8
:10096000205B6D4261725D7D6D61782E537572669C
:100970002E5B6D4261725D7D474620646973706CC9
:10098000617920205B255D7D6D696E2E204F3220C0
:100990004469732E5B255D7D44697665206D656EC7
:1009A000757320205B735D7D53617475726174652E
:1009B000207820205B255D7D4465736174757261CC
:1009C000746520785B255D7D4E6F466C79205261A1
:1009D00074696F205B255D7D474620616C61726D97
:1009E000203120205B255D7D6E6F742075736564FA
:1009F000202020202020207D4465636F204F6666E4
:100A00007365745B646D5D7D70704F32206C6F77C1
:100A1000205B634261725D7D70704F322068696750
:100A2000685B634261725D7D70704F322073686FE6
:100A3000775B634261725D7D73616D706C696E6737
:100A4000207261746520207D44697669736F72201D
:100A500054656D702020207D44697669736F722023
:100A60004465636F6461747D44697669736F722055
:100A70004E6F74557365317D44697669736F72206A
:100A800070704F322020207D44697669736F722028
:100A9000446562756720207D44697669736F7220B2
:100AA0004E6F74557365327D434E532073686F7774
:100AB000202020205B255D7D4C6F67626F6F6B206F
:100AC0006F6666736574207D4C6173742044656342
:100AD0006F2061745B6D5D7D456E642041706E6F4B
:100AE00065205B6D696E5D7D53686F77205662612E
:100AF0007474205B3D315D7D546869732070726F42
:100B00006772616D2069737D64697374726962755F
:100B100074656420696E207468657D7D686F70659A
:100B200020746861742069742077696C6C20626538
:100B30007D7D75736566756C2C20627574205749D0
:100B400054484F55547D414E592057415252414EC1
:100B500054593B20776974686F75747D6576656E4E
:100B60002074686520696D706C6965647D7D77614E
:100B70007272616E7479206F667D4D4552434841B3
:100B80004E544142494C495459206F727D7D46492B
:100B9000544E45535320464F5220417D50415254AC
:100BA0004943554C415220505552504F53452E7D8C
:100BB0005365652074686520474E552047656E650E
:100BC00072616C7D5075626C6963204C6963656EFF
:100BD000736520666F727D7D6D6F726520646574CC
:100BE00061696C733A7D7777772E6865696E726993
:100BF0006368737765696B616D702E64657D4465AC
:100C0000636F73746F707D7D6D2F6D696E7D4E6F38
:100C10002053746F707D4465636F73756D7D446997
:100C2000766574696D657D7D44657074687D46691F
:100C3000727374204761733F7D7D44656661756C96
:100C4000743A7D7D4D696E757465737D4D6F6E74FC
:100C50006820207D446179202020207D59656172C3
:100C60002020207D536574207D7D47617323207D86
:100C70005965737D43757272656E743A7D7D5365F7
:100C8000747570204D656E753A7D437573746F6D24
:100C90002046756E6374696F6E73497D4465636F3A
:100CA000747970653A7D5A482D4C3136204F437D1A
:100CB0004761756765202020207D47617567657DE8
:100CC0005A482D4C31362043437D41637469766523
:100CD000204761733F207D7D4761732053657475A4
:100CE00070202D204761736C6973747D4465707446
:100CF00068202B7D4465707468202D7D4261636B94
:100D00007D7D43435220536574506F696E74204D4E
:100D1000656E757D43435220536574506F696E74E0
:100D2000204D656E757D5350237D426174746572EC
:100D30007920496E666F7D7D426174746572792099
:100D4000496E666F726D6174696F6E7D4379636C15
:100D500065733A7D41706E6F657D4C61737420439D
:100D60006F6D706C6574653A7D7D4C6F77657374DB
:100D70002056626174743A7D4C6F7765737420619C
:100D8000743A7D7D546D696E3A7D546D61783A7D1B
:100D9000536574204761737D4F32202B7D7D4F3228
:100DA000202D7D7D4865202B7D7D4865202D7D7D16
:100DB000457869747D7D44656C6574657D7D4465A9
:100DC0006275673A7D7D4F4E207D4F46467D446576
:100DD0006C2E20616C6C7D7D556E657870656374DA
:100DE00065642072657365742066726F6D7D4469F9
:100DF00076656D6F64652120506C65617365206850
:100E0000656C707D616E64207265706F72742074A1
:100E10006865204465627567207D496E666F726DF6
:100E20006174696F6E2062656C6F77217D7D4261B0
:100E3000696C6F75747D41706E6F65202020207D18
:100E400044657363656E747D537572666163657D19
:100E5000517569743F7D4D6F72657D7D436F6E6620
:100E600069726D3A7D7D4D656E7520323A7D4361C4
:100E70006E63656C7D7D4F4B217D53746F70776120
:100E8000742E7D7D3A2E2E2E2E2E2E2E2E2E3A7D37
:100E90004E4F542055534544212121212121212108
:100EA0002121217D4E6F742075736564217D4E6F05
:100EB0007420757365642121217D4C31362D4746A0
:100EC000204F437D437573746F6D2046756E637458
:100ED000696F6E7349497D7D4746204C6F772020AE
:100EE000202020205B255D7D4746204869676820DB
:100EF000202020205B255D7D436F6C6F7223204294
:100F0000617474657279207D436F6C6F7223205316
:100F100074616E646172647D436F6C6F72232044F0
:100F20006976656D61736B7D436F6C6F72232057BB
:100F300061726E696E67737D53686F772073656346
:100F4000732E205B3D315D7D6E6F7420757365641B
:100F5000202020202020207D6E6F74207573656412
:100F6000202020202020207D4176722E2044657094
:100F70007468205B3D315D7D426C696E6B2047611A
:100F80007320205B3D315D7D4465707468576172EC
:100F90006E5B6D4261725D7D434E53207761726E70
:100FA000696E67205B255D7D4746207761726E69BB
:100FB0006E6720205B255D7D70704F3220776172F7
:100FC0006E5B634261725D7D56656C2E7761726EF9
:100FD0005B6D2F6D696E5D7D6E6F742075736564DA
:100FE000202020202020207D6E6F74207573656482
:100FF000202020202020207D6E6F74207573656472
:10100000202020202020207D6E6F74207573656461
:10101000202020202020207D6E6F74207573656451
:10102000202020202020207D6E6F74207573656441
:10103000202020202020207D6E6F74207573656431
:10104000202020202020207D6E6F74207573656421
:10105000202020202020207D6E6F74207573656411
:10106000202020202020207D6E6F74207573656401
:10107000202020202020207D6E6F742075736564F1
:10108000202020202020207D6E6F742075736564E1
:10109000202020202020207D6E6F742075736564D1
:1010A000202020202020207D6E6F742075736564C1
:1010B000202020202020207D6E6F742075736564B1
:1010C000202020202020207D6E6F742075736564A1
:1010D000202020202020207D437573746F6D2046D2
:1010E000756E6374696F6E732049497D53686F77BD
:1010F000204C6963656E73657D7D53696D2E20524A
:101100006573756C74733A7D4E4F54205553454446
:1011100021212121217D70704F32202B7D7D707027
:101120004F32202D7D7D44696C2E7D7D4465636F3B
:10113000747970653A205A482D4C3136204F437DE2
:10114000466F72204F70656E2043697263756974D3
:101150002020207D4469766572732E20537570704F
:101160006F7274732035207D5472696D69782047E1
:10117000617365732E2020202020207D436F6E66D2
:10118000696775726520796F757220676173207D5C
:10119000696E204761737365747570206D656E7537
:1011A0002E20207D436865636B2043463131202625
:1011B000204346313220217D4465636F7479706528
:1011C0003A204761756765202020207D4469766557
:1011D00074696D652077696C6C20626520696E7D2D
:1011E0004D696E757465733A5365636F6E64732EE3
:1011F0002020207D4F535443322077696C6C206E41
:101200006F7420202020207D636F6D7075746520C1
:101210004465636F2C204E6F466C797D74696D65F3
:1012200020616E642044657361742E2D2020207D22
:1012300074696D6520617420616C6C212020202010
:101240002020207D4465636F747970653A5A482D7B
:101250004C3136204343207D466F72202853656D04
:10126000692D29436C6F73656420207D4369726327
:101270007569742072656272656174686572737DE8
:10128000436F6E66696775726520746865203320E8
:101290002020207D536574506F696E747320696ED1
:1012A00020434352202D207D5365747570206D6559
:1012B0006E752E2035206261696C2D7D6F7574739B
:1012C0002061726520617661696C61626C652E7D5A
:1012D0004465636F747970653A2041706E6F652064
:1012E0002020207D4F535443322077696C6C20645A
:1012F0006973706C6179207D6561636820646573D2
:1013000063656E742073657061722D7D6174656CA8
:101310007920696E204D696E3A5365632E20207DD9
:1013200057696C6C2074656D706F72616C6C79209C
:101330007365747D73616D706C6572617465207422
:101340006F2031207365637D4E6F204465636F208D
:1013500063616C63756C6174696F6E7D4465636F06
:10136000747970653A204C31362D4746204F437DC5
:101370004465636F6D7072657373696F6E2063612E
:101380006C2D207D63756C6174696F6E7320776955
:10139000746820746865207D47462D4D6574686FBC
:1013A00064202847465F6C6F2F47467D5F68692938
:1013B0002E20436865636B20434633322026207D10
:1013C0004346333321204F70656E20436972637545
:1013D0006974207D77697468204465657020537452
:1013E0006F70732E2020207D4465636F7479706563
:1013F0003A204C31362D47462043437D4465636F88
:101400006D7072657373696F6E2063616C2D207DE2
:1014100063756C6174696F6E73207769746820748A
:101420006865207D47462D4D6574686F64202847A8
:10143000465F6C6F2F47467D5F6869292E204368A1
:1014400065636B20434633322026207D4346333389
:1014500021436C6F73656420436972637569747DA1
:101460007769746820446565702053746F70732EBB
:101470002020207D4465636F6D6F64652063686123
:101480006E6765642120207D4C31362D4746204310
:10149000437D4E6F7420666F756E647D5365745026
:1014A0006F696E747D7D4E6F204465636F7D4772FA
:1014B000617068737D7D446973706C61797D4E6F76
:1014C000206465636F7D536561726368206D6F642E
:1014D000756C657D457869747D7D52657365742092
:1014E00043462C4761732026204465636F7D446921
:1014F0007361626C65206D6F64756C657D7D536989
:101500006D756C61746F727D4F5354432053696DD8
:10151000756C61746F727D7D53746172742044695F
:1015200076657D7D2B20316D7D7D2D20316D7D7D1E
:101530002B31306D7D7D2D31306D7D7D4578697429
:101540007D7D6E6F74207573657D787D44617465F3
:1015500020666F726D61743A7D7D5365747570207D
:101560004D656E7520323A7D4D4D444459597D7D0F
:1015700044444D4D59597D7D59594D4D44447D7DCF
:101580004F535443207D4261696C7D7D41697220D7
:101590007D7D41697220207D43616C696272617456
:1015A000657D4D61782044657074687D6E6F747DD3
:1015B000666F756E64217D7D6D563A7D4E65772030
:1015C0004346206164646564217D4E6577204375E0
:1015D00073746F6D46756E6374696F6E737D776536
:1015E00072652061646465642120436865636B7D76
:1015F0004346204920616E64204346204949204DDE
:10160000656E757D666F722044657461696C7321C7
:101610007D7D53616C696E6974793A7D426F747433
:101620006F6D2054696D653A7D7D4D61782E204443
:10163000657074683A7D43616C63756C6174652094
:101640004465636F7D7D53686F77204465636F7079
:101650006C616E7D4C656164205469737D7D4C6561
:101660006164205469737D7D53746F707761746316
:10167000687D5265736574204C6F67626F6F6B7D18
:101680005265626F6F74204F5354437D526573658A
:1016900074204465636F646174617D7D2C8B01D817
:1016A0001200278D05D8279D12002C8B01D812001F
:1016B0000B6F800EA66EF86A020EF76EFC0EF66EC9
:1016C0000BC14CF1000E2CBB010E4D6F040E4E6F82
:1016D0004F6BEBEC0BF04851F6264951F72209000D
:1016E000F55027BD02D0E8CF7DF00900F55027BDA9
:1016F00002D0E8CF7CF00900F5500108E8CF7EF079
:101700000900F5CF1BF10D6B0E6BF66AF86A010E3E
:10171000F76E01D02C9B0900F5500D27000E0E230B
:101720000B2FF9D72CBBF6D7F86AB00E0D25F66E45
:10173000070E0E21F76E27AD20EE60F009007D0E3A
:10174000F56201D00AD0F550DE6E09007D0EF5621B
:1017500001D003D0F550DE6EF1D727AD1DEC0EF0B1
:10176000120032C14CF133C14DF13C0E4E6F4F6B44
:101770004FD848C133F14CC132F11200D8904633F2
:101780004533472FFBD71200D8904B334A334933A8
:101790004833472FF9D712004951FF08496F485184
:1017A000D890FF08486F12001F975451525D506F38
:1017B00055515359516FD8A812001F8750C154F189
:1017C00051C155F1526953695451525D506F555191
:1017D0005359516F12004A6B4B6B4C514E03F350EF
:1017E000486FF450496F4C514F03F3504927F45060
:1017F0004A234D514E03F3504927F4504A23D8B0A1
:101800004B2B4D514F03F3504A27F4504B231200FA
:10181000486B496B4E514F11D8B4FF0C010E476F06
:101820004FBF05D0472BD8904E374F37F9D7D890B8
:10183000483749374E514C5F4F51D8A04F294D5F23
:10184000D8B005D04E514C274F514D2301D048817F
:101850004707D8B41200D8904F334E33E8D7200E44
:10186000476F4B514D6F4A514C6F4951536F48511F
:10187000526F4B6B4A6B496B486B556B546BD890EE
:10188000523753374C374D37543755374F51555DD5
:10189000D8A44DEF0CF04E51545DD8A057EF0CF08A
:1018A0004E51545FD8A055074F51555FD8804837E7
:1018B00049374A374B37472F3FEF0CF01200D8908B
:1018C00075337433762FFBD71200D8907A3379337F
:1018D00078337733762FF9D712007851FF08786F75
:1018E0007751D890FF08776F12002A978351815D56
:1018F0007F6F84518259806FD8A812002A877FC1D8
:1019000083F180C184F1816982698351815D7F6F38
:1019100084518259806F1200796B7A6B7B517D0301
:10192000F350776FF450786F7B517E03F350782734
:10193000F45079237C517D03F3507827F4507923B8
:10194000D8B07A2B7C517E03F3507927F4507A2358
:1019500012000A6FB5EF0CF000000000000000005C
:101960000000000000000000000000000000000077
:101970000000000000000000000000000000000067
:101980000000000000000000000000000000000057
:101990000000000000000000000000000000000047
:1019A00000000A2FACEF0CF01200096FE1EF0CF011
:1019B0000000000000000000000000000000000027
:1019C0000000000000000000000000000000000017
:1019D0000000000000000000000000000000000007
:1019E00000000000000000000000000000000000F7
:1019F000000000000000000000000000630EA9ECE1
:101A00000CF0092FD8EF0CF01200630E3261326F28
:101A100032C134F1356B1F950A0E3A6F366B67D8B9
:101A2000010E3A6F366B1F8562D8120032C134F155
:101A3000356B1F85F1D732C134F1356B1F95640EBC
:101A40003A6F366B54D8E8D7259F376F1F8B372BEB
:101A5000372F1F9B238B372B372F239B32C134F11A
:101A600033C135F11F95100E3A6F270E366F1FAD3B
:101A70003ED8E80E3A6F030E366F23BB07D025BF62
:101A800003D01F85372D1F9523B91F851FAD2FD874
:101A90001F9D640E3A6F366B27B924D023BB09D043
:101AA00025BF03D01F85372D1F9523B91F8523BB65
:101AB0001F851DD80A0E3A6F366B23BB09D025BF90
:101AC00003D01F85372D1F9523B91F8523BB1F8585
:101AD00029B708D00CD8010E3A6F366B1F8524A5A4
:101AE00006D824952799386B382B23991200396B27
:101AF0003651355DD8A00ED004E13A51345DD8A0FE
:101B000009D03651355F3A51345FD8A03507392BAB
:101B10001F85EED7382F1200382B300E39251FB510
:101B200004D01FBF04D0200E01D0258FDE6E372FCA
:101B300012002E0EDE6E23891200A96E2DD0A96E22
:101B400027D02B91010EAA6E690E03D02691AA6AA6
:101B5000640EAD6E238F040EA96E9D9A9E9A8186A7
:101B600046D8AECFA8FF818826BF0FD015D8819860
:101B7000A8CFADFF36D8A93EF3D781969E9A9D8A0D
:101B8000AA6A269F239FB4EF4AF0FF0EAD6EF5D7E9
:101B9000A69EA69CA6801200A69EA69CA684F29E47
:101BA000550EA76EAA0EA76EA682F28EA6B2FED71B
:101BB000A6941200948C948E240EAC6E900EAB6E94
:101BC000080EB86EB06A220EAF6EAE6A9E6A9D8A2B
:101BD0001200AC6AAB6A9D9A949C949E829C829EF1
:101BE0001200ABAE12000000ACA2FBD712009E9A0E
:101BF000269F436B446B9EBA120000000000000059
:101C000000009EBA120000000000000000009EBA12
:101C1000120000000000000000009EBA1200000048
:101C20000000000000009EBA1200442FE4D7432FAA
:101C3000E1D7AB98AB88268F1200DE6A7BC0FAF141
:101C40007AC0F9F134EC5AF00101FAC17BF0F9C124
:101C50007AF01200106F10C17DF0210E2DD9D890AE
:101C60001035000ED8B0010E2CD9D890103529D9D6
:101C700012000F6F0FC17CF0200E1ED9000E21D96B
:101C80000F511FD91200220E17D984807AC083FF0A
:101C9000809480847BC083FF80948084210E0CD943
:101CA000D8901035000ED8B0010E0BD9D89010374F
:101CB000102907D9200E00D9000E03D90F5101D9E0
:101CC000220EFAD884807AC083FF809480847BC0FF
:101CD00083FF809480841200220EEED884807AC024
:101CE00083FF809480847BC083FF80948084120073
:101CF000836A80968194809A84948094849212005E
:101D0000F4511DEC10F0F5C11CF11C51B2DFF7517C
:101D10002AEC0EF0E1DF1C2B1C51F663F6D71C51A8
:101D2000A8DFF7512AEC0EF0D7DFF5C11CF11C51EA
:101D3000A0DFF8512AEC0EF0CFDF1C2B1C51F6630C
:101D4000F6D71C5196DFF8512AEC0EF0C5DFF7C12B
:101D50001CF11C517FDFF5518CDF95DF1C2B1C51D2
:101D6000F863F7D7F7C11CF11C5174DFF65181DF1E
:101D70008ADF1C2B1C51F863F7D723EC1AF01200F2
:101D8000F4511DEC10F0350E97D8F7C11CF1D89026
:101D90001C35000ED8B0010E94D8D8901C3591D8BF
:101DA000360E8AD8F8C11CF1D8901C35000ED8B078
:101DB000010E87D8D8901C3584D8370E7DD8F5C150
:101DC0001CF11C517ED8F6C11CF11C517AD8200E92
:101DD00073D8000E76D8F5C11CF11C5172D8210EB3
:101DE0006BD8F7C11CF1D8901C35000ED8B0010E8D
:101DF00068D8D8901C3565D8220E5ED8F5C11CF184
:101E0000F6C11DF11C511D5F1D2BF7C11CF1F8C15E
:101E10001EF11C511E5F1E2B84801EC11CF17AC056
:101E200083FF809480847BC083FF809480847AC009
:101E300083FF809480847BC083FF809480841C2FE8
:101E4000EED71D2FEAD7000E37D823EC1AF0120078
:101E5000350E32D8000E35D8000E33D8360E2CD8B9
:101E6000010E2FD83F0E2DD8370E26D8000E29D8B8
:101E7000EF0E27D8200E20D8000E23D8000E21D830
:101E8000210E1AD8000E1DD8000E1BD8220E14D811
:101E90008480836A0A0E1E6F1E0E1D6F1C6B809459
:101EA0008084809480841C2FFAD71D2FF7D71E2F93
:101EB000F3D7000E01D812008490836E8094808442
:101EC00012008480836E8094808412008096200E9D
:101ED000D5EC0CF081840000809A00008482FA0E18
:101EE000D5EC0CF0848400008492020EA9EC0CF076
:101EF00084820A0ED5EC0CF0240EDEDF020EDCDF4D
:101F0000000EDFDF000EDDDF030ED6DF000ED9DFAF
:101F1000300ED7DF180ED0DF000ED3DF280ED1DF52
:101F2000F80ECADF000ECDDF0F0ECBDFF90EC4DFD7
:101F3000000EC7DF0F0EC5DF100EBEDF000EC1DFC3
:101F4000000EBFDF0CD884DF8086200ED5EC0CF0AD
:101F5000050EB2DF000EB5DF010EB3DF1200700E0A
:101F6000ABDF1F0EAEDF000EACDF710EA5DF230E60
:101F7000A8DF800EA6DF720E9FDF2A0EA2DF800E82
:101F8000A0DF730E99DF150E9CDF110E9ADF740E21
:101F900093DF1C0E96DF110E94DF750E8DDF1B0E86
:101FA00090DF150E8EDF760E87DF1A0E8ADF150E94
:101FB00088DF770E81DF1C0E84DF180E82DF780E3B
:101FC0007BDF210E7EDF150E7CDF1200700E74DFCA
:101FD000140E77DF000E75DF710E6EDF170E71DFE6
:101FE000000E6FDF720E68DF150E6BDF800E69DF8B
:101FF000730E62DF150E65DF110E63DF740E5CDF9A
:10200000140E5FDF0B0E5DDF750E56DF1B0E59DF02
:10201000150E57DF760E50DF130E53DF0E0E51DF15
:10202000770E4ADF1C0E4DDF180E4BDF780E44DFB3
:10203000150E47DF0E0E45DF12002E6F2EC12FF159
:10204000030E2F17000E2F4F500E2F4FA00E2F4FA5
:10205000F80E306F2EC12FF11C0E2F172F432F4378
:10206000000E2F4F040E2F4F080E2F4F0C0E2F4F28
:10207000100E2F4F140E2F4F200E2F4F3F0E316F8B
:102080003133303331333033313330332EC12FF1EC
:102090002E6B31332E3331332E3331332E33E00E6A
:1020A0002F172F432F432F432F432F43000E2F4F24
:1020B000040E2F4F080E2F4F0C0E2F4F100E2F4FC8
:1020C000140E2F4F200E2F4F3F0E316F31332E3312
:1020D00031332E3331332E3331332E3331332E33EC
:1020E0002EC17AF030C17BF01200E46F1F0EE46560
:1020F00005D0010EAA6E200EE45F01D0AA6AE45159
:10210000040DF350820FA96EC8EC0DF0A850AA6A16
:102110001200E46F1F0EE46505D0010EAA6E200EBA
:10212000E45F01D0AA6AE451040DF350820FA96E56
:10213000C8EC0DF0A8CF32F1A92AC8EC0DF0A8CF59
:1021400033F1AA6A12009A0EE36F2A8D03D0240E8F
:10215000E36F2A9D1F8F28EC0FF0010EBA6F2199B3
:1021600021972099AA6BA56B229D229F83EC2BF0CF
:10217000010EE8CF7FF02AAD04D0BA0E58EC0BF078
:1021800003D01B0E58EC0BF0000EE8CF7FF023ECD1
:102190001AF0010E2AAD000EAA6EB86B21912193A0
:1021A000140EE8CF7DF0230EE8CF7CF020EE60F037
:1021B000AAC132F1000E2ABD200E322732C1DCF155
:1021C000386B382B376B16EC0DF03A0EDE6E200EA6
:1021D000DE6E1DEC0EF0E351AA2558EC0BF01F0E3D
:1021E000DC5DD8B415D0260EDC5DD8B411D0270E36
:1021F000DC5DD8B40DD0280EDC5DD8B409D0290E32
:10220000DC5DD8B405D02A0EDC5DD8B401D003D093
:10221000010EDC6F01D0DC6B140EE8CF7DF0410EB7
:10222000E8CF7CF020EE60F02B0EDE6E2F0EDE6E1F
:102230002D0EDE6E3A0EDE6E200EDE6E2B0E22BDF1
:102240002D0EDE6E1DEC0EF0140EE8CF7DF05F0E4D
:10225000E8CF7CF020EE60F0310EDE6E2F0EDE6EE9
:10226000310EDE6E300EDE6E3A0EDE6E200EDE6E4B
:10227000310EDE6E300E22BFDE6E200EDE6E1DECE5
:102280000EF0140EE8CF7DF07D0EE8CF7CF020EE4E
:1022900060F0590E51EC0BF0A551800FA96EC8ECFF
:1022A0000DF0A8CF32F1A551810FA96EC8EC0DF049
:1022B000A8CF33F1339F386B382B376B375124EC71
:1022C0000DF02C0EDE6E310EA8AE380EDC67310E2E
:1022D000DE6E350EA8BEDE6E420EDE6E200EDE6EA7
:1022E000200EDE6E200EDE6E1DEC0EF0140EE8CF1A
:1022F0007DF09B0EE8CF7CF020EE60F0610E51EC9B
:102300000BF0A551820FA96EC8EC0DF0A8CF32F1E9
:10231000A551830FA96EC8EC0DF0A8CF33F1386B2F
:10232000382B376B375124EC0DF0200EDE6E200E6B
:10233000DE6E200EDE6E1DEC0EF00B0E58EC0BF078
:10234000F3EC12F09AEC1DF0FAEC31F021B30FD05F
:1023500021B11AD020B3B4EF4AF020B1F5EC3DF032
:1023600020B1E3EC43F0209120B91CD0EDD7BA2B7B
:10237000070EBA6302D0010EBA6FB86B9AEC1DF06B
:10238000F3EC12F02193E0D7AA6A010E2ABDAA6EDF
:10239000BA4F0FD0BA4F17D0BA4F19D0BA4F1BD07F
:1023A000BA4F39D0020E2AAD010EBA6FAA6A8EEF6B
:1023B00013F0AA2BAABBAA6BAA51040DF3CFA5F167
:1023C000010EBA6FE4D6227D020EBA6FE0D6227FEC
:1023D000030EBA6FDCD6A551800FA96EC8EC0DF0C4
:1023E000A8CF32F1A551810FA96EC8EC0DF0A8CF8E
:1023F00033F1339FA551820FA96E32C1A8FFCCECF7
:102400000DF0A551830FA96E33C1A8FFCCEC0DF0E0
:10241000040EBA6FBCD6A551820FA96EC8EC0DF0A0
:10242000A8CF32F1A551830FA96EC8EC0DF0A8CF4B
:1024300033F1A551810FA96EC8EC0DF0A8CFA6F11C
:10244000010EDC6305D032673269322B336B16D054
:1024500022AD0BD0010E22BF0A0E325F000EA6BFC6
:10246000335B7F0E33BF336F09D0010E22BF0A0EDC
:102470003227000EA6BF332333BF336BA551820F23
:10248000A96E32C1A8FFCCEC0DF0A551830FA96E47
:1024900033C1A8FFCCEC0DF0050EBA6F78D6E46F0F
:1024A0001F0EE46505D0010EAA6E200EE45F01D078
:1024B000AA6AE451040DF350800FA96EC8EC0DF028
:1024C000A8CF32F1A92AC8EC0DF0A8CF33F1AA6A3F
:1024D0001200CF4F14D0CF4F19D01200CF4F0FD0D2
:1024E000CF4F14D0CF4F19D0CF4F1ED0CF4F23D0C6
:1024F000CF4F28D0CF4F2FD0CF4F34D012000B0E5C
:102500003DD8B9EC12F0020ECF6F12000C0E49D874
:10251000B9EC12F0030ECF6F1200110E2FD8B9ECE8
:1025200012F0040ECF6F1200120E3BD8B9EC12F06D
:10253000050ECF6F1200130E34D8B9EC12F0060E50
:10254000CF6F1200060ECF6F1D0E3ED8B9EC12F001
:10255000070ECF6F1200200E24D8B9EC12F0080E2F
:10256000CF6F1200210E1DD8B9EC12F0010ECF6F03
:102570001200326F32671200EDEF28F0396F89ECEC
:1025800010F032C152F133C153F139514FEC12F016
:1025900032C154F133C155F1D4EC0BF01FA7FF0C3D
:1025A000000C396F89EC10F032C154F133C155F190
:1025B00039514FEC12F032C152F133C153F1D4EC26
:1025C0000BF01FA7FF0C000C396F89EC10F032C123
:1025D00054F133C155F1CFC152F1536BD4EC0BF030
:1025E0001FA7FF0C000C2497249912002B97010EB3
:1025F000BA6F1F9F28EC0FF0B86B2099219121939F
:10260000208F21872AEC1EF09AEC1DF02497249944
:1026100023EC13F021B124D020AFB4EF4AF020B165
:10262000F5EC3DF020B1E3EC43F020B12BEC3DF0B4
:1026300020B176EC48F0209120B9B4EF4AF020B3F5
:10264000B4EF4AF0E5D724A908D02183BA2B060EAF
:10265000BA6518D0010EBA6F15D024B721811200C7
:10266000BA4FB4EF2EF0BA4F91EF35F0BA4FF5EF05
:1026700014F0BA4F8BEF13F0BA4F48EF13F0BA4F84
:10268000B4EF4AF0B86B21B79AEC1DF02499120010
:10269000010EBA6F1F9F28EC0FF0B86B20992191A3
:1026A0002193208F21877EEC1EF09AEC1DF0249759
:1026B000249923EC13F0050EBA6304D0060EBA6F0A
:1026C0009AEC1DF021B115D020AF90D720B1F5ECD8
:1026D0003DF020B1E3EC43F020B12BEC3DF020B114
:1026E00076EC48F0209120B981D720B3B4EF4AF0BE
:1026F000E0D7BA4F9BEF16F0BA4F51EF33F0BA4F15
:1027000073EF34F0BA4FA6EF4BF0BA4FA6EF4BF091
:10271000050EBA6F6ED72B97010EBA6F1F9F28EC6C
:102720000FF048EC1EF0B86B209921912193208F77
:102730002187D8EC13F084EC14F09AEC1DF0249768
:10274000249923EC13F021B117D020AFB4EF4AF055
:1027500020B1F5EC3DF020B1E3EC43F020B12BECDF
:102760003DF020B176EC48F0209120B9B4EF4AF06A
:1027700020B3B4EF4AF0E5D7BA4FA7EF10F0BA4F45
:10278000A3EF10F0BA4FACD0BA4F03D0BA4F5CD021
:1027900036D02B87220E9FEC0DF0A82A060EA862D9
:1027A00001D0A86ACCEC0DF0040EBA6F2499BBD707
:1027B000220E9FEC0DF0A86604D0650E58EC0BF0CD
:1027C0001200A82E04D0660E58EC0BF01200A82EB2
:1027D00004D0680E58EC0BF01200A82E04D08A0E1C
:1027E00058EC0BF01200A82E04D0980E58EC0BF009
:1027F0001200A82E1200EC0E58EC0BF012002BA7C2
:10280000B4EF4AF028EC0FF083EC2BF0010EE8CF88
:102810007FF0EB0E58EC0BF0000EE8CF7FF0220EAD
:102820009FEC0DF0070EA802F350C10FBA6F070E10
:10283000396FBA5158EC0BF0BA2B392FFAD71E0E5C
:102840004FEC4BF0B4EF4AF0010EBA6F1F9F28EC2B
:102850000FF066EC1EF0B86B209921912193208F28
:102860002187E6EC14F0C0EC14F09AEC1DF02497EC
:10287000249923EC13F0040EBA6304D0060EBA6F49
:102880009AEC1DF021B117D020AFB4EF4AF020B17F
:10289000F5EC3DF020B1E3EC43F020B12BEC3DF042
:1028A00020B176EC48F0209120B98BEF13F020B3E3
:1028B000B4EF4AF0DED7BA4F54D0BA4F74D0BA4F03
:1028C00007D0BA4F28D7BA4F26D7050EBA6F26D7EA
:1028D0002FEC4BF04AEC4BF0030EBA6F2499B6D7AD
:1028E0001A0E9FEC0DF0A82A630EA8640AD0690E98
:1028F000A86007D01A0E9DEC0DF0030EBA6F249954
:1029000012D7640EA86EF6D71A0E9FEC0DF0630E68
:10291000A86421D8690EA8601ED85F0EE8CF7CF0AD
:10292000530EE8CF7DF0000EE8CF7EF020EE60F091
:10293000A8CF32F1336B1F8F030E24EC0DF01F9FD5
:102940006B0EDE6E670EDE6E2F0EDE6E6C0EDE6EB2
:102950001DEC0EF01200640EA86E1A0E9DEC0DF028
:1029600012005B0E9FEC0DF0A82A020EA86401D0A5
:10297000A86A5B0E9DEC0DF0010EBA6F24996BD71F
:102980005B0E9FEC0DF0A86604D0030E55EC0BF027
:102990001200A82E04D0040E55EC0BF01200050E08
:1029A00055EC0BF01200270E9FEC0DF0A82A010E3B
:1029B000A86401D0A86A270E9DEC0DF02A85010EAF
:1029C000A8622A95020EBA6F249945D7270E9FEC6C
:1029D0000DF0A86603D0830E58EC0BF0A806A8668D
:1029E000F6D6820E58EC0BF01200010EBA6F28ECEE
:1029F0000FF099EC1EF0B86B209921912193208F54
:102A0000218799EC1EF09AEC1DF02497249923EC71
:102A100013F021B116D020AFE9D520B1F5EC3DF08F
:102A200020B1E3EC43F020B12BEC3DF020B176EC8B
:102A300048F0209120B9F6EF12F020B3B4EF4AF03D
:102A4000E6D7BA4F08D0BA4F3AD0BA4F16D0BA4FDD
:102A500005D0BA4F20D0030EBA6FCBD508EC22F0C8
:102A6000BA6FBA6701D0F7D778EC0EF0000E9B6E04
:102A70007E0ED36EFF0000EF00F008EC22F0BA6F7C
:102A8000BA6701D0E8D728EC0FF0190E58EC0BF01C
:102A900074EC16F0E0D708EC22F0BA6FBA6701D0F8
:102AA000DAD728EC0FF0190E58EC0BF08DC100F5B9
:102AB0008EC101F520EC80F00101B4EF4AF008EC82
:102AC00022F0BA6FBA6701D0C6D728EC0FF0190E02
:102AD00058EC0BF08DC100F58EC101F520EC80F0B3
:102AE0000101AA6A030EA96E336B150EE5D8150E07
:102AF000E3D8150EE1D8150EDFD8150EDDD8150E6A
:102B0000DBD8010EA86E210E9DEC0DF0A86A220EF6
:102B10009DEC0DF0A86A230E9DEC0DF0000EA86A46
:102B2000270E9DEC0DF0A86A5A0E9DEC0DF0A86AD8
:102B30005B0E9DEC0DF0640E1A0E9DEC0DF01F0E59
:102B4000A86E1B0E9DEC0DF0A86A1C0E9DEC0DF0FE
:102B5000A86A1D0E9DEC0DF0A86A1E0E9DEC0DF0EE
:102B6000A86A1F0E9DEC0DF0A86A200E9DEC0DF0DA
:102B7000640EA86E240E9DEC0DF0250E9DEC0DF05C
:102B8000260E9DEC0DF0010ECC6FCD6B7F0EA96E65
:102B9000336B640E91D81E0E8FD8F00E8DD8780E40
:102BA0008BD8050E89D8070E87D8040E336F338F64
:102BB000880E82D8040E336F338F4C0E7DD8140EDE
:102BC0007BD8140E79D81E0E77D86E0E75D85A0E93
:102BD00073D83C0E71D8640E6FD8640E6DD80A0E8F
:102BE0006BD8130E69D8A00E67D8960E65D80A0E5A
:102BF00063D8060E61D8060E5FD8000E5DD8000EB1
:102C00005BD80C0E59D8000E57D8140E55D8336B1C
:102C1000338F000E51D8030E4FD80A0E4DD8000E38
:102C20004BD8010EAA6E7F0EA96E336B1E0E44D8D0
:102C30005A0E42D8C70E40D8FF0E3ED83E0E3CD8A2
:102C4000E00E3AD8000E38D8000E36D8000E34D830
:102C5000000E32D8000E30D8320E336F338FC80ECC
:102C60002BD8650E29D8650E27D8A10E25D80F0EB2
:102C700023D8000E21D8000E1FD8000E1DD8000E3C
:102C80001BD8000E19D8000E17D8000E15D8000E4C
:102C900013D8000E11D8000E0FD8000E0DD8000E5C
:102CA0000BD8000E09D8000E07D8000E05D8000E6C
:102CB00003D8AA6AB4EF4AF0326FA92A32C1A8FF3A
:102CC000CCEC0DF0A92A33C1A8FFCCEC0DF0A92A59
:102CD00032C1A8FFCCEC0DF0A92A339F33C1A8FF65
:102CE000CCEC0DF0336B1200BD6BBE6B020E366F79
:102CF000376B400E3A6F23933B693B51B4EC2DF098
:102D00003A2FFAD7C58469EC2EF0070ED5EC0CF0FB
:102D1000372FEFD7362FECD72393BD6BBE6BFD0E4D
:102D2000A8EC2DF0FD0EA8EC2DF0FE0EA8EC2DF079
:102D3000BD6BBE6B120028EC0FF0219521992197F5
:102D4000B86B219121932099229122932295BB6BFC
:102D500083EC2BF0010EE8CF7FF01D0E58EC0BF04A
:102D6000000EE8CF7FF0160E58EC0BF0170E58EC63
:102D70000BF0D5EC16F0180E58EC0BF024972499B4
:102D800024B79AEC17F024B966EC17F021B942D0B9
:102D900020B1F5EC3DF020B1E3EC43F0209120B9F7
:102DA00091D020B3B4EF4AF0EBD7460EE8CF7DF0D8
:102DB000410EE8CF7CF020EE60F005C132F1386BB7
:102DC000382B376B16EC0DF03A0EDE6E04C132F183
:102DD000386B382B376B16EC0DF0200EDE6E200EA4
:102DE000DE6E1DEC0EF0460EE8CF7DF05F0EE8CFF4
:102DF0007CF020EE60F007C1F1F106C1F2F108C1EC
:102E0000F3F171EC24F0200EDE6E200EDE6E1DEC70
:102E10000EF0120007C132F1324F1F0E324F1C0E5E
:102E2000324F1F0E324F1E0E324F1F0E324F1E0EEC
:102E3000324F1F0E324F1F0E324F1E0E324F1F0EDB
:102E4000324F1E0E324F1F0E066502D0010E066F66
:102E5000200EE8CF7DF09B0EE8CF7CF0080E396F96
:102E600014EC1DF0050E0A6F036B209120A1FED714
:102E70002091F3EC16F0460EE8CF7DF0410EE8CF3E
:102E80007CF020EE60F005C132F1386B382B376BE7
:102E900016EC0DF03A0EDE6E04C132F1386B382BB1
:102EA000376B16EC0DF03A0EDE6E03C132F1386B63
:102EB000382B376B16EC0DF0200EDE6E1DEC0EF08D
:102EC0000A2FD4D7010EBA6F4AEF13F022B121892D
:102ED000BB2BBBC1BCF1BC4F2185BC4F2285BC4F75
:102EE0002283BC4F2281200EE8CF7DF09B0EE8CFDD
:102EF0007CF020EE60F05E0E51EC0BF0BBC1BCF13B
:102F0000BC2F04D05A0E51EC0BF00FD0BC2F04D0C4
:102F10005B0E51EC0BF009D0BC2F04D05C0E51ECD1
:102F20000BF003D05D0E51EC0BF01DEC0EF0F3EC4A
:102F300012F012002499036B22B120D022B310D0DA
:102F400022B515D021B506D0052B170E05651CD06E
:102F5000056B1AD0042B3B0E046516D0046B14D0FD
:102F6000062B1F0E066510D0010E066F0DD0072B25
:102F70000C0E076509D0010E076F06D0082B140E42
:102F8000086502D0080E086FD5EC16F0F3EC12F0CD
:102F900012007C6B080E7B6F6CC17DF16DC17EF100
:102FA0008CEC0CF0100E7727270E782372C181F17C
:102FB00073C182F177C183F178C184F175EC0CF0B3
:102FC0007FC185F180C186F12AB71ED0239585C1C6
:102FD0007BF186C17CF185C17DF186C17EF18CECEF
:102FE0000CF0110E766F65EC0CF085C181F186C195
:102FF00082F177C183F178C184F175EC0CF07FC167
:1030000087F180C188F117D0238585C17BF186C106
:103010007CF185C17DF186C17EF18CEC0CF00F0E48
:10302000766F65EC0CF0855177278651782377C150
:1030300087F178C188F16AC181F16BC182F1FA0E22
:10304000836F846B75EC0CF07FC17BF180C17CF1E8
:1030500085C17DF186C17EF18CEC0CF077C174F1F5
:1030600078C175F10C0E766F5FEC0CF074C177F1DE
:1030700075C178F12AA70DD064517727655178235F
:10308000100E7727270E782377C189F178C18AF14E
:103090000FD064C181F165C182F177C183F178C13C
:1030A00084F175EC0CF07FC177F180C178F1E8D73D
:1030B00066C168F167C169F1C80E6827000E69230F
:1030C00068C17BF169C17CF185C17DF186C17EF16A
:1030D0008CEC0CF077C174F178C175F10D0E766F40
:1030E0005FEC0CF074C18BF175C18CF162C174F1AD
:1030F00063C175F1010E766F5FEC0CF074518B2794
:1031000075518C23B80E8B270B0E8C2370C181F167
:1031100071C182F189C183F18AC184F175EC0CF02F
:103120007FC17BF180C17CF18BC17DF18CC17EF1CF
:103130008CEC0CF00C0E766F65EC0CF02AB76DEC95
:103140000CF0E80E7727030E782377C18DF178C154
:103150008EF125AD04D0C6C18DF1C7C18EF16EC10F
:1031600068F16FC169F1640E6827000E692368C1B8
:103170007BF169C17CF187C17DF188C17EF18CEC66
:103180000CF00B0E766F65EC0CF0249D23B509D086
:10319000C80E7727000E782377C197F178C198F190
:1031A0001200C80E816F826B77C183F178C184F100
:1031B00075EC0CF02AB7248D7FC197F180C198F18E
:1031C0001200C7D8A00E3D6F0C0E586FFBD812002E
:1031D000D6D857C171F156C170F11200BAD8900E0D
:1031E000F2D7CDD857C173F156C172F11200B1D8E0
:1031F0000D0E586F540E3D6FE5D8C1D857C15BF125
:1032000056C15AF10D0E586F580E3D6FDBD8B7D826
:1032100057C15DF156C15CF10D0E586F640E3D6FE4
:10322000D1D8ADD857C15FF156C15EF10D0E586FC0
:10323000680E3D6FC7D8A3D857C161F156C160F180
:103240005BC163F1D8906333D8906333D890633314
:103250005AC162F1D8805BA1D8906233D8805BA359
:10326000D8906233D8805BA5D89062335CC164F19A
:10327000D8805DA1D8906433D8805DA3D8906433A2
:10328000D8805DA5D8906433D8805DA7D89064338A
:10329000D8805DA9D8906433D8805DABD890643372
:1032A0005DC165F1D8805AA1D8906533D8805AA302
:1032B000D8906533D8805AA5D8906533D8906533B7
:1032C000D8906533D89065335FC166F1D8805EAF22
:1032D000D8906637D8805EADD8906637676B5FBF91
:1032E00067835FBD678161C16AF1D88060AFD890A4
:1032F0006A376B6B61BF6B815EC16CF16C9D5CB1B9
:103300006C8D6C9F5CB36C8F6D6B5CB56D815CB7C5
:103310006D835CB96D855CBB6D876F6B60C16EF151
:103320006E9F239F120080820000808E00000000AC
:103330000000000000000000809E1200809200004B
:10334000808E000000000000000000000000809E51
:103350001200E9DFF3DFE7DFF1DFE5DFEFDFE3DFD7
:10336000EDDFE1DFEBDFDFDFE9DFDDDFE7DFDBDF45
:10337000E5DFE4DFE3DFE2DFE1DFE0DF1200080E9C
:10338000586F10D83DC157F1080E586F0BD83DC18A
:1033900056F1808E000000000000000000000000D8
:1033A000809E1200808E00000000000000000000DF
:1033B0000000809E80A8D89080B8D8803D37582FD4
:1033C000F1D71200809E8082030E585F808E00002D
:1033D00000000000000000000000809E00000000CF
:1033E0000000000000000000808E000000000000CF
:1033F000000000000000809E0000000000000000AF
:1034000000000000808E00000000000000000000AE
:103410000000809E3DAF80923DBF8082D8903D37B6
:10342000808E000000000000000000000000809E70
:10343000582FF0D71200240E75EC10F007D0250E8F
:1034400075EC10F003D0230E75EC10F02E6F000E0B
:103450002E6301D018D0040E2E6301D014D0080EB4
:103460002E6301D010D0C00E2E6301D00CD0C40E3C
:103470002E6301D008D0C80E2E6301D004D02E5187
:103480001DEC10F01200FF0E1DEC10F01200DB6FAF
:10349000DB4F08D0DB4F2DD0DB4F39D0DB4F45D091
:1034A000DB4F59D033C135F132C134F190C133F122
:1034B0008FC132F170EC2DF032C152F133C153F1B2
:1034C0002B0E89EC10F032C154F133C155F1D4EC1C
:1034D0000BF01FA707D023EC1AF035C133F134C12C
:1034E00032F112001FEC1AF035C133F134C132F160
:1034F000120065C532F12C0E75EC10F0325DD8B0BB
:1035000003D023EC1AF012001FEC1AF0120032C59F
:1035100032F12D0E75EC10F0325DD8B003D023ECF3
:103520001AF012001FEC1AF0120048C152F149C102
:1035300053F12E0E75EC10F0640DF3CF54F1F4CF6F
:1035400055F1D4EC0BF01FA703D023EC1AF01200B6
:103550001FEC1AF0120045C132F12F0E75EC10F07D
:10356000325DD8B003D023EC1AF012001FEC1AF031
:103570001200DB6FD9C1DAF1D8C1D9F1D7C1D8F1C6
:10358000D6C1D7F1D5C1D6F1DBC1D5F12AA512003C
:10359000C80EE8CF7CF0640EE8CF7DF0000EE8CFD7
:1035A0007EF0000EE8CF7FF023EC1AF020EE60F002
:1035B000D551DE6ED651DE6ED751DE6ED851DE6E3D
:1035C000D951DE6EDA51DE6E200EDE6E1DEC0EF08D
:1035D00012008188819666EC0FF028EC0FF023EC46
:1035E0001AF0850E58EC0BF0860E58EC0BF0870E97
:1035F00058EC0BF0880E58EC0BF0640EE8CF7CF022
:103600000A0EE8CF7DF0000EE8CF7EF0000EE8CF86
:103610007FF023EC1AF020EE60F0D551DE6ED6512B
:10362000DE6ED751DE6ED851DE6ED951DE6EDA51C4
:10363000DE6E2E0EDE6E200EDE6E1FC132F1386B96
:10364000382B376B1BEC0DF0200EDE6E20C132F1F3
:10365000386B382B376B1BEC0DF01DEC0EF07D0E2C
:10366000E8CF7CF00A0EE8CF7DF0000EE8CF7EF0C8
:10367000000EE8CF7FF023EC1AF020EE60F021C1BD
:1036800032F1386B382B376B1BEC0DF0200EDE6EF1
:1036900022C132F1386B382B376B1BEC0DF0200E4A
:1036A000DE6E23C132F1386B382B376B1BEC0DF01B
:1036B000200EDE6E24C132F1386B382B376B1BECD9
:1036C0000DF0200EDE6E25C132F1386B382B376BD2
:1036D0001BEC0DF01DEC0EF0960EE8CF7CF00A0E00
:1036E000E8CF7DF0000EE8CF7EF0000EE8CF7FF04F
:1036F00023EC1AF020EE60F026C132F1386B382B43
:10370000376B1BEC0DF0200EDE6E27C132F1386BEB
:10371000382B376B1BEC0DF0200EDE6E28C132F11A
:10372000386B382B376B1BEC0DF0200EDE6E29C189
:1037300032F1386B382B376B1BEC0DF0200EDE6E40
:103740002AC132F1386B382B376B1BEC0DF01DECB6
:103750000EF024A7FED7819812001BEC1AF00B0E76
:1037600055EC0BF0560E58EC0BF0570E58EC0BF0D6
:1037700023EC1AF01200000EE8CFF4F13C0EE8CF73
:10378000F5F1EF0EE8CFF6F15A0EE8CFF7F19F0E04
:10379000E8CFF8F1C0EC0EF003EC1FF070EC1FF076
:1037A0001200E9DF1BEC1AF0540E58EC0BF023EC7E
:1037B0001AF0080E396F910EE8CF7CF0000EE8CFBA
:1037C0007DF014EC1DF012002BB512007A0EB9EC4E
:1037D0001AF0B90EE8CF7CF0770EE8CF7DF0010E3D
:1037E000E8CF7EF0000EE8CF7FF023EC1AF020EE59
:1037F00060F022C532F1386B382B376B1BEC0DF0C3
:10380000270EDE6E1DEC0EF0000EE8CF7EF01200EB
:10381000B2DF1BEC1AF0550E58EC0BF023EC1AF04B
:1038200012002BB5120020BF31D0790EB9EC1AF07E
:103830001BEC1AF0520E58EC0BF023EC1AF0760E3B
:10384000E8CF7CF05E0EE8CF7DF0010EE8CF7EF091
:10385000000EE8CF7FF023EC1AF020EE60F02BC5CD
:1038600032F1386B382B376B05EC0DF06D0EDE6ED8
:1038700024C532F1386B382B376B05EC0DF0270E71
:10388000DE6E1DEC0EF0000EE8CF7EF02BB51200C0
:10389000780EB9EC1AF0B90EE8CF7CF0770EE8CFCD
:1038A0007DF0010EE8CF7EF0000EE8CF7FF023EC34
:1038B0001AF020EE60F031C532F1C70E3261326F7E
:1038C0001F9F386B382B376B1BEC0DF0270EDE6E0D
:1038D0001DEC0EF032C532F1080E75EC10F03261BD
:1038E00001D067D7770EB9EC1AF0910EE8CF7CF0D3
:1038F000000EE8CF7DF0000EE8CF7EF0030E47EC1F
:103900001AF020EE60F0470EDE6E460EDE6E3A0EC6
:10391000DE6E32C532F1386B382B376B1BEC0DF095
:10392000250EDE6E200EDE6E1DEC0EF023EC1AF07E
:103930001200410EE8CF7CF0690EE8CF7DF0000E5A
:10394000E8CF7EF023EC1AF020EE60F0EBC132F10C
:103950001F8F386B382B376B1BEC0DF01F9F6D0ED4
:10396000DE6E690EDE6E6E0EDE6E200EDE6E1DECFD
:103970000EF05F0EE8CF7CF0640EE8CF7DF0000E15
:10398000E8CF7EF023EC1AF020EE60F0ECC132F1CB
:103990001F8F386B382B376B1BEC0DF01F9F6D0E94
:1039A000DE6E200EDE6E1DEC0EF012002BB5120046
:1039B000760EB9EC1AF05A0EE8CF7CF0000EE8CF84
:1039C0007DF0000EE8CF7EF0050E47EC1AF020EEF9
:1039D00060F02D0E1FB72B0EDE6E45C132F1386B35
:1039E000382B376B05EC0DF0530E51EC0BF01DEC42
:1039F0000EF023EC1AF02B891200080E396F5A0EC4
:103A0000E8CF7CF0000EE8CF7DF02B990DD0060EAC
:103A1000396F020EE8CF7CF0730EE8CF7DF004D052
:103A2000010EE8CF7EF003D0000EE8CF7EF020EE4E
:103A300060F0200EDE6E392FFCD71DEC0EF0000E6C
:103A4000E8CF7EF01200630EB9EC1AF0320EE8CF28
:103A50007CF0000EE8CF7DF0000EE8CF7EF0000E87
:103A6000E8CF7FF023EC1AF020EE60F019C132F1BC
:103A7000326705D01AC132F1326701D039D02DAF8B
:103A800034D0B72F01D034D02D8F060EB76125D892
:103A900019C132F11AC133F1B1EC0BF0335132C11B
:103AA00033F1326F490EDE6E6E0EDE6E740EDE6E18
:103AB0003A0EDE6E386B382B376B16EC0DF03A0E83
:103AC000DE6E33C132F1386B382B376B16EC0DF0EC
:103AD000200EDE6E1DEC0EF012002D9F050EB76F4E
:103AE00012002D8F050EB76F1200B72F01D0CCD763
:103AF0002D9F060EB761F5DF05C132F1386B382B0B
:103B0000376B16EC0DF03A0EDE6E04C132F1386BF5
:103B1000382B376B16EC0DF03A0EDE6E03C132F126
:103B2000386B382B376B16EC0DF0200EDE6E1DEC6B
:103B30000EF01200230EE8CF7CF0000EE8CF7DF0EF
:103B4000000EE8CF7EF0000EE8CF7FF023EC1AF0F5
:103B500020EE60F0B80EDE6E1DEC0EF0410EE8CFE8
:103B60007CF0000EE8CF7DF0000EE8CF7EF0000E76
:103B7000E8CF7FF020EE60F0B80EDE6E1DEC0EF0A8
:103B80005F0EE8CF7CF0000EE8CF7DF0000EE8CFAE
:103B90007EF0000EE8CF7FF020EE60F0B80EDE6E13
:103BA0001DEC0EF07D0EE8CF7CF0000EE8CF7DF02E
:103BB000000EE8CF7EF0000EE8CF7FF020EE60F040
:103BC000B80EDE6E1DEC0EF09B0EE8CF7CF0000E02
:103BD000E8CF7DF0000EE8CF7EF0000EE8CF7FF05A
:103BE00023EC1AF020EE60F0B80EDE6E1DEC0EF045
:103BF000B90EE8CF7CF0000EE8CF7DF0000EE8CFE4
:103C00007EF0000EE8CF7FF020EE60F0B80EDE6EA2
:103C10001DEC0EF0BAC139F1394F230E394F410E68
:103C2000394F5F0E394F7D0E394F9B0E394FB90E0C
:103C3000E8CF7CF0000EE8CF7DF0000EE8CF7EF0FC
:103C4000000EE8CF7FF020EE60F0B70EDE6E1DECC8
:103C50000EF0120083EC2BF0010EE8CF7FF0050E82
:103C600058EC0BF0000EE8CF7FF0060E58EC0BF08E
:103C7000070E58EC0BF0090E58EC0BF00A0E58EC3E
:103C80000BF08E0E58EC0BF00B0E58EC0BF01200F4
:103C900083EC2BF0010EE8CF7FF0620E58EC0BF0B6
:103CA000000EE8CF7FF0630E58EC0BF0990E58EC45
:103CB0000BF0140E55EC0BF0640E58EC0BF08E0E5E
:103CC00058EC0BF00B0E58EC0BF0120083EC2BF0C1
:103CD000010EE8CF7FF0020E55EC0BF0000EE8CF9E
:103CE0007FF0010E55EC0BF0810E58EC0BF0BB0E83
:103CF00058EC0BF00B0E58EC0BF0120083EC2BF091
:103D0000010EE8CF7FF0900E58EC0BF0000EE8CFDC
:103D10007FF0080E58EC0BF06E0E58EC0BF0710EA5
:103D200058EC0BF0F70E58EC0BF00B0E58EC0BF0B8
:103D3000120083EC2BF0010EE8CF7FF01C0E58EC44
:103D40000BF0000EE8CF7FF0150E58EC0BF0F50EDF
:103D500058EC0BF01C0E55EC0BF01D0E55EC0BF057
:103D60001E0E55EC0BF00B0E58EC0BF0120083EC12
:103D70002BF0010EE8CF7FF0F80E58EC0BF0000EA0
:103D8000E8CF7FF0F90E58EC0BF0150E55EC0BF068
:103D9000160E55EC0BF0170E55EC0BF0180E55ECFB
:103DA0000BF00B0E58EC0BF01200650EB9EC1AF08C
:103DB00097C199F198C19AF1640EE8CF7CF0000E9A
:103DC000E8CF7DF0000EE8CF7EF0000EE8CF7FF068
:103DD00023EC1AF020EE60F02D0E24BDDE6E97C1AC
:103DE00032F198C133F1030E386F1F8F020E24ECAD
:103DF0000DF01F9FB00EDE6E430EDE6E200EDE6EE7
:103E00001DEC0EF012002BB51200750EB9EC1AF075
:103E100097C199F198C19AF1D80EE8CF7CF0410E84
:103E2000E8CF7DF0000EE8CF7EF0000EE8CF7FF007
:103E300023EC1AF020EE60F02D0E24BDDE6E97C14B
:103E400032F198C133F1030E386F1F8F020E24EC4C
:103E50000DF01F9FB00EDE6E200EDE6E1DEC0EF01C
:103E60001200740EB9EC1AF0780EE8CF7CF0000E58
:103E7000E8CF7DF0000EE8CF7EF0040E47EC1AF09C
:103E800020EE60F0700EDE6E700EDE6E4F0EDE6E97
:103E9000320EDE6E3A0EDE6E48C132F149C133F1A8
:103EA0002987010E24EC0DF02997200EDE6E1DEC03
:103EB0000EF023EC1AF012000A0E396F780EE8CFDC
:103EC0007CF0000EE8CF7DF014EC1DF01200C00E67
:103ED000E8CF7CF0410EE8CF7DF0050E396FA4D518
:103EE0002ABB12002BB51200000EE8CF7FF08EEC3B
:103EF0001FF02CAD12002A0E75EC10F0326F010E7F
:103F0000326312002D772DA71200010EE8CF7FF04B
:103F10008EEC1FF0000EE8CF7FF01200730EB9ECAC
:103F20001AF0C00EE8CF7CF0410EE8CF7DF0000E15
:103F3000E8CF7EF023EC1AF0640E10C532F1D88081
:103F4000325511C532F1D8803257090E75EC10F098
:103F500011C533F1326501D005D0336703D0050EAA
:103F6000396F62D5150E32630ED033670CD020EE58
:103F700060F0080E4EEC0BF0200E2CBD2A0EDE6E0B
:103F80001DEC0EF0120020EE60F01F8F386B382B06
:103F9000376B1BEC0DF02F0EDE6E11C532F1386B56
:103FA000382B376B1BEC0DF0200E2CBD2A0EDE6E6D
:103FB0001F9F1DEC0EF01200550EE8CF7DF0000E95
:103FC000E8CF7EF0000EE8CF7FF0AA6A220E9FECC9
:103FD0000DF0A86620D07D0EE8CF7CF023EC1AF01F
:103FE00020EE60F04F0EDE6E1DEC0EF0550EE8CFA9
:103FF0007DF0000EE8CF7EF0000EE8CF7FF0960E49
:10400000E8CF7CF023EC1AF020EE60F0430EDE6E79
:104010001DEC0EF01200A806A86601D01200A8063A
:10402000A86629D07D0EE8CF7CF023EC1AF020EEB4
:1040300060F0430EDE6E550EE8CF7DF0000EE8CF47
:104040007EF0000EE8CF7FF01DEC0EF0960EE8CF6C
:104050007CF023EC1AF020EE60F0430EDE6E550E7D
:10406000E8CF7DF0000EE8CF7EF0000EE8CF7FF0C5
:104070001DEC0EF01200A806A86601D01200A806DA
:10408000A86629D07D0EE8CF7CF020EE60F0470EC8
:10409000DE6E550EE8CF7DF0000EE8CF7EF0000E0C
:1040A000E8CF7FF023EC1AF01DEC0EF0960EE8CF6F
:1040B0007CF020EE60F0460EDE6E550EE8CF7DF00F
:1040C000000EE8CF7EF0000EE8CF7FF023EC1AF070
:1040D0001DEC0EF012007D0EE8CF7CF020EE60F0BB
:1040E000470EDE6E550EE8CF7DF0000EE8CF7EF075
:1040F000000EE8CF7FF023EC1AF01DEC0EF0960EC8
:10410000E8CF7CF020EE60F0460EDE6E550EE8CF74
:104110007DF0000EE8CF7EF0000EE8CF7FF023ECBC
:104120001AF01DEC0EF01200000EE8CFF4F1190E9B
:10413000E8CFF5F1780EE8CFF6F1520EE8CFF7F1BF
:104140009F0EE8CFF8F1C0EC0EF029B15ED06D0EF5
:10415000B9EC1AF05A0EE8CF7DF0000EE8CF7EF0F1
:104160001F8F020E0A6F000E096F336B332B040E84
:104170000A2720EE60F0470EDE6E33C132F1386B55
:10418000382B376B1BEC0DF03A0EDE6E200EDE6E18
:104190000AC1A9FFC8EC0DF0A8CF32F1386B382B5B
:1041A000376B1BEC0DF02F0EDE6EA92AC8EC0DF05C
:1041B000A8CF32F1386B382B376B1BEC0DF01B0E90
:1041C0009FEC0DF033C132F1A832322FFDD7D8B0B9
:1041D00004D04A0E1DEC10F002D023EC1AF0210E90
:1041E0009FEC0DF0A850336301D009D0190E0927B8
:1041F0005A0EE8CF7DF009C17CF01DEC0EF023ECE7
:104200001AF0050E3363B2D712005A0EE8CF7DF0D4
:10421000000EE8CF7EF01F8F230E0A6F000E096F8D
:10422000E66B0A2BE62B190E09275A0EE8CF7DF014
:1042300009C17CF020EE60F0530EDE6E500EDE6E93
:10424000E6C132F1386B382B376B1BEC0DF03A0EB0
:10425000DE6E200EDE6E0AC1A9FFC8EC0DF0A8CFFD
:1042600032F1336B030E24EC0DF01DEC0EF0030E57
:10427000E663D7D7210E9FEC0DF0A8CFD1F1D10581
:10428000040DF350070FA96EC8EC0DF0A8CF33F161
:10429000D105040DF350060FA96EC8EC0DF0A8CFA0
:1042A00032F15A0EE8CF7DF0640EE8CF7CF020EEBC
:1042B00060F0440EDE6E690EDE6E6C0EDE6E3A0E3F
:1042C000DE6E386B382B376B1BEC0DF02F0EDE6E6D
:1042D00033C132F1386B382B376B1BEC0DF01DEC12
:1042E0000EF01F9F1200710EB9EC1AF02ABB1200DB
:1042F00028BF120029A123D0870EE8CF7CF05A0EE8
:10430000E8CF7DF0000EE8CF7EF0000EE8CF7FF022
:1043100023EC1AF020EE60F0240E9FEC0DF0A8CFF5
:1043200032F1336B030E24EC0DF0420EDE6E610EA3
:10433000DE6E720EDE6E1F9F1DEC0EF057D0820EE9
:10434000E8CF7CF0640EE8CF7DF0010EE8CF7EF080
:10435000000EE8CF7FF023EC1AF0210E9FEC0DF059
:10436000A8CFD1F1D105040DF350070FA96EC8EC09
:104370000DF0A8CF11F5D105040DF350060FA96E6D
:10438000C8EC0DF0A8CFD0F111C50AF1D880640EA9
:104390000A55D880A856A8CF10F5640E10C532F182
:1043A000D880325511C532F1D880325711C533F15A
:1043B000150E326306D0336704D0090E55EC0BF0AE
:1043C00015D020EE60F01F8F386B382B376B1BEC4D
:1043D0000DF02F0EDE6E11C532F1386B382B376BB6
:1043E0001BEC0DF01F9F1DEC0EF000D0000EE8CF6F
:1043F000F4F17A0EE8CFF5F1AF0EE8CFF6F1520EF8
:10440000E8CFF7F19F0EE8CFF8F180EC0EF0120044
:10441000000EE8CFF4F1440EE8CFF5F1920EE8CFAC
:10442000F6F1220EE8CFF7F1650EE8CFF8F1C0EC17
:104430000EF0230E75EC10F0E8CFF4F1460EE8CF45
:10444000F5F1900EE8CFF6F1230EE8CFF7F1640E08
:10445000E8CFF8F180EC0EF08F0E58EC0BF0910ED7
:1044600058EC0BF0920E58EC0BF0010EBA6F000EE8
:10447000E8CFF4F1600EE8CFF5F18F0EE8CFF6F15A
:10448000270EE8CFF7F1330EE8CFF8F1C0EC0EF0CD
:10449000BAC139F1600E394F600E394F780EE8CF4E
:1044A0007CF0270EE8CF7DF0000EE8CF7EF0000E06
:1044B000E8CF7FF023EC1AF020EE60F0B70EDE6E4E
:1044C0001DEC0EF020992191219324992497B86B2B
:1044D000640ED5EC0CF0FAEC31F021B315D021B11B
:1044E0000ED020B1F5EC3DF020B1E3EC43F020918B
:1044F00020B903D020B301D0EED7000C010CBA4F85
:10450000FCD7BA4FFBD7F9D7BA2B030EBA6302D048
:10451000010EBA6FACD7720EB9EC1AF090C133F13C
:104520008FC132F170EC2DF0270E336171D02BBBAF
:104530002FEC23F02B9B20EE60F0030E536FE80E60
:10454000526F33C155F132C154F1542B000E552333
:10455000D4EC0BF01FA780D8180EE8CF7CF0000E2B
:10456000E8CF7DF0020EE8CF7EF0000EE8CF7FF0BE
:10457000010E47EC1AF0000E536F630E526F33C1F9
:1045800055F132C154F1D4EC0BF01FA70AD01F8FA4
:104590002987386B382B376B375124EC0DF01F9F70
:1045A00002D0300EDE6E1DEC0EF02997010EE8CF22
:1045B0007EF0320EE8CF7CF0280EE8CF7DF0010EC1
:1045C00047EC1AF090C133F18FC132F170EC2DF04D
:1045D00020EE60F02E0EDE6E000E536F090E526F4D
:1045E00033C155F132C154F1D4EC0BF01FA707D001
:1045F000040E386F2485000E24EC0DF002D0300E2E
:10460000DE6E1DEC0EF02495000EE8CF7EF0120059
:104610002BAB2FEC23F020EE60F0180EE8CF7CF0EF
:10462000000EE8CF7DF0020EE8CF7EF0000EE8CF5E
:104630007FF0010E47EC1AF029871F8F386B382B5B
:10464000376B375124EC0DF01F9F1DEC0EF02997AE
:10465000000EE8CF7EF01200200EDE6E1200000E7B
:10466000E8CFF4F1180EE8CFF5F15A0EE8CFF6F1E5
:10467000000EE8CFF7F15A0EE8CFF8F1C0EC0EF0DB
:104680002B8B1200680EB9EC1AF0960EE8CF7CF076
:10469000000EE8CF7DF0000EE8CF7EF0000EE8CFF0
:1046A0007FF023EC1AF020EE60F00E0E51EC0BF0D0
:1046B000200EDE6E20C532F121C533F1B1EC0BF0D6
:1046C0001F8F325133C132F1336F386B382B376B58
:1046D0001BEC0DF03A0EDE6E33C132F1386B382B25
:1046E000376B16EC0DF01F9F1DEC0EF01200670EDD
:1046F000B9EC1AF07D0EE8CF7CF0000EE8CF7DF02B
:10470000000EE8CF7EF0000EE8CF7FF023EC1AF029
:1047100020EE60F0230E51EC0BF0200EDE6ECCC1CB
:1047200032F1CDC133F1B1EC0BF01F8F325133C1F7
:1047300032F1336F386B382B376B1BEC0DF03A0EC0
:10474000DE6E33C132F1320732BF326B386B382B39
:10475000376B16EC0DF01F9F1DEC0EF0120020BD04
:104760001200620EB9EC1AF0190EE8CF7CF0000EC0
:10477000E8CF7DF0000EE8CF7EF0000EE8CF7FF0AE
:1047800023EC1AF020EE60F08DC132F18EC133F1CE
:104790001F8F386B382B376B375124EC0DF01F9F70
:1047A0006D0EDE6E620EDE6E610EDE6E720EDE6EFF
:1047B000200EDE6E1DEC0EF01200660EB9EC1AF043
:1047C0001F0E75EC10F0326F010E326323D0AF0E66
:1047D000E8CF7CF0000EE8CF7DF0000EE8CF7EF051
:1047E000000EE8CF7FF023EC1AF020EE60F0C2C19B
:1047F00032F1C3C133F1010E386F24851F8F020ED1
:1048000024EC0DF01F9F560EDE6E200EDE6E1DECAA
:104810000EF01200230E75EC10F0E8CFF4F1AE0E9E
:10482000E8CFF5F1C20EE8CFF6F1000EE8CFF7F1D0
:104830001F0EE8CFF8F180EC0EF0040E526F100E50
:10484000536FC2C154F1C3C155F1D4EC0BF01FB783
:1048500045D0AC0E546F0D0E556FC2C152F1C3C19D
:1048600053F1D4EC0BF01FB736D050C14CF151C10D
:104870004DF1140E4E6F4F6B08EC0CF048C10AF16D
:10488000020E0A650A6F230E75EC10F0E8CFF4F102
:10489000B50EE8CFF5F1BB0EE8CFF6F11F0EE8CF6D
:1048A000F7F1210EE8CFF8F1C0EC0EF0220E75EC16
:1048B00010F0E8CFF4F1B00EE8CFF5F1C00EE8CF7C
:1048C000F6F1010EE8CFF7F10AC1F8F1C0EC0EF0F5
:1048D00023EC1AF01200010E0A6FD5D71E0E0A6FD4
:1048E000D2D75B0E9FEC0DF0A8660ED0F1C132F16D
:1048F0001F8F386B382B376B16EC0DF01F9F2F0E68
:10490000DE6EF2C132F112D05B0E9FEC0DF0A82EDC
:104910001FD0F2C132F11F8F386B382B376B16EC7A
:104920000DF01F9F2F0EDE6EF1C132F11F8F386B1D
:10493000382B376B16EC0DF01F9F2F0EDE6EF3C178
:1049400032F11F8F386B382B376B16EC0DF01200DD
:10495000F3C132F11F8F386B382B376B16EC0DF02B
:104960001F9F2F0EDE6EF1C132F11F8F386B382B77
:10497000376B16EC0DF01F9F2F0EDE6EF2C132F179
:104980001F8F386B382B376B16EC0DF012005B0E57
:104990009FEC0DF0A86615D0F1C132F11F8F386B76
:1049A000382B376B16EC0DF01F9F2F0EDE6EF2C109
:1049B00032F11F8F386B382B376B16EC0DF01F9FC1
:1049C00012005B0E9FEC0DF0A82EE6D7F2C132F17B
:1049D0001F8F386B382B376B16EC0DF01F9F2F0E87
:1049E000DE6EF1C132F11F8F386B382B376B16EC4E
:1049F0000DF01F9F1200640EB9EC1AF04B0EE8CFB9
:104A00007CF0000EE8CF7DF0000EE8CF7EF0000EC7
:104A1000E8CF7FF023EC1AF020EE60F007C1F1F14F
:104A200006C1F2F108C1F3F171EC24F01DEC0EF0B7
:104A30001200000EE8CFF4F1000EE8CFF5F11A0EE7
:104A4000E8CFF6F1410EE8CFF7F1640EE8CFF8F1C8
:104A5000C0EC0EF012002BB51200700EB9EC1AF07B
:104A6000B80EE8CF7CF0000EE8CF7DF0010EE8CF65
:104A70007EF0000EE8CF7FF023EC1AF020EE60F01D
:104A800091C132F192C133F170EC2DF01F8F24856A
:104A9000030E24EC0DF01F9F1F9D1DEC0EF0000E69
:104AA000E8CF7EF0120020BF1200410EB9EC1AF0E0
:104AB00028BF92D02ABB90D0260E75EC10F0326F32
:104AC000010E326301D088D0A5C132F1A6C133F105
:104AD0001F9F20EE60F0386B382B376B1F8D3751DE
:104AE00024EC0DF0140EE8CF7CF0780EE8CF7DF0CA
:104AF000010EE8CF7EF023EC1AF01DEC0EF0000E54
:104B0000E8CF7EF0120020BF12001BEC1AF08C0ED2
:104B100058EC0BF023EC1AF0550EE8CF7CF05A0E4F
:104B2000E8CF7DF0010EE8CF7EF023EC1AF0E1C172
:104B300032F11F9F20EE60F0386B382B376B1BEC87
:104B40000DF03A0EDE6EE2C132F1386B382B376B66
:104B500016EC0DF01DEC0EF0000EE8CF7EF012000A
:104B6000000EE8CFF4F13C0EE8CFF5F1770EE8CF78
:104B7000F6F15A0EE8CFF7F19F0EE8CFF8F1C0EC4E
:104B80000EF012001BEC1AF08B0E58EC0BF023EC1D
:104B90001AF0910EE8CF7CF05A0EE8CF7DF0010EAE
:104BA000E8CF7EF023EC1AF0DCC132F120EE60F0A9
:104BB000386B382B376B1BEC0DF03A0EDE6EDDC117
:104BC00032F1386B382B376B16EC0DF01DEC0EF014
:104BD000000EE8CF7EF01200A5C132F1A6C133F17C
:104BE0001F9F1F8D20EE60F0386B382B376B1F8DA9
:104BF000375124EC0DF03A0EDE6EA7C132F1386B5E
:104C0000382B376B16EC0DF0140EE8CF7CF05A0EF3
:104C1000E8CF7DF0010EE8CF7EF023EC1AF01DEC1A
:104C20000EF01F9D000EE8CF7EF01200000EE8CFC0
:104C3000F4F1360EE8CFF5F1660EE8CFF6F13E0E50
:104C4000E8CFF7F19F0EE8CFF8F1C0EC0EF01200BC
:104C500020BF1200560EB9EC1AF01BEC1AF01B0E16
:104C600055EC0BF023EC1AF0500EE8CF7CF06E0EF2
:104C7000E8CF7DF0000EE8CF7EF023EC1AF020EEB6
:104C800060F017C132F118C133F1020E325F000E2D
:104C9000335BB1EC0BF032C10AF133C132F1336B4B
:104CA000000E1F9F1F8D386B382B376B1F8D3751B0
:104CB00024EC0DF03A0EDE6E0AC132F1386B382B5F
:104CC000376B16EC0DF01F9F1DEC0EF0550EB9EC76
:104CD0001AF0500EE8CF7CF03E0EE8CF7DF0000ECB
:104CE000E8CF7EF023EC1AF020EE60F093C132F1B1
:104CF00094C133F170EC2DF01F8F2485030E24EC4A
:104D00000DF01F9F6D0EDE6E200EDE6E1DEC0EF0A0
:104D10001200610EB9EC1AF0000EE8CF7CF0000E24
:104D2000E8CF7DF0000EE8CF7EF0000EE8CF7FF0F8
:104D300023EC1AF020EE60F0060E4EEC0BF0AA6A9F
:104D4000A96AC8EC0DF0A8CF32F1A92AC8EC0DF081
:104D5000A8CF33F11F8F386B382B376B375124ECCA
:104D60000DF0200EDE6E560EDE6E010E326F1F8FBE
:104D7000386B382B376B1BEC0DF02E0EDE6E3E0EB3
:104D8000326F1F8F386B382B376B16EC0DF01F9F6F
:104D90001DEC0EF012006F0EB9EC1AF019EC25F0B4
:104DA0001F0E58EC0BF029B107D0200E58EC0BF079
:104DB0007A0E58EC0BF006D0EE0E58EC0BF0890E84
:104DC00058EC0BF0210E58EC0BF0220E58EC0BF0C7
:104DD00012006F0EB9EC1AF0F00E58EC0BF0F10E59
:104DE00058EC0BF0190E55EC0BF0930E58EC0BF041
:104DF000F40E58EC0BF01200640EE8CF7DF0000EBC
:104E0000E8CF7CF0000EE8CF7EF023EC1AF020EE25
:104E100060F0530EDE6E650EDE6E6C0EDE6E180EEA
:104E20009FEC0DF0A8CF32F11F9F386B382B376BFA
:104E300005EC0DF02F0EDE6E190E9FEC0DF0A8CFD5
:104E400032F1386B382B376B05EC0DF01DEC0EF0A2
:104E50007B0E58EC0BF07C0E58EC0BF07D0E58ECF2
:104E60000BF07E0E58EC0BF01200FE0E58EC0BF01F
:104E7000FA0E58EC0BF0FB0E58EC0BF0FC0E58EC55
:104E80000BF0FD0E58EC0BF01200230E75EC10F039
:104E9000E8CFF4F17C2B7CC0F5F17CC0F6F1120E6A
:104EA000F6277A0EE8CFF7F1322732078A0E326101
:104EB000326F32C1F8F1C0EC0EF0000EE8CFF4F121
:104EC0007CC0F5F17CC0F6F1120EF62732C1F7F185
:104ED000F72B8B0EE8CFF8F1C0EC0EF01200000EAD
:104EE000E8CFF4F133C1F5F17D0EE8CFF6F1640EB1
:104EF000E8CFF7F19F0EE8CFF8F1C0EC0EF012000A
:104F00006E0EB9EC1AF02BC532F1326706D053ECB5
:104F100028F0EF0E58EC0BF01200E669E70EE76F91
:104F2000190EE727E62B99EC27F0050EE663F8D774
:104F300012001F8F640EE8CF7DF0E7C17CF0E7C15F
:104F400033F115EE2BF0E651E3CF32F13251D8B404
:104F50006FEF27F020EE60F0386B382B376B1BECCF
:104F60000DF06D0EDE6E1DEC0EF08C0EE8CF7DF0B8
:104F7000E7C17CF015EE24F0E651E3CF32F120EEEC
:104F800060F0386B382B376B16EC0DF0270EDE6EA9
:104F90001DEC0EF045EC27F012006D0EB9EC1AF086
:104FA000640EE8CF7DF0000EE8CF7EF01F8F020E7A
:104FB0000A6FE70E096F336B332B040E0A27190EA5
:104FC0000927640EE8CF7DF009C17CF020EE60F087
:104FD000470EDE6E33C132F1386B382B376B1BEC6A
:104FE0000DF03A0EDE6E0AC1A9FFC8EC0DF0A8CF95
:104FF00032F1386B382B376B1BEC0DF02F0EDE6E59
:10500000A92AC8EC0DF0A8CF32F1386B382B376BDA
:105010001BEC0DF01B0E9FEC0DF033C132F1A832EA
:10502000322FFDD74A0ED8A01DEC10F01DEC0EF06B
:1050300023EC1AF0050E3363BFD71200640EE8CFDD
:105040007DF0000EE8CF7EF01F8F230E0A6FE70E73
:10505000096FE66B0A2BE62B190E092709C17CF0B4
:10506000640EE8CF7DF020EE60F0530EDE6E500E41
:10507000DE6EE6C132F1386B382B376B1BEC0DF06E
:105080003A0EDE6E0AC1A9FFC8EC0DF0A8CF32F1CE
:10509000336B030E24EC0DF01DEC0EF0030EE663F3
:1050A000D9D71F9F1200000EE8CFF4F1000EE8CF11
:1050B000F5F1B90EE8CFF6F1520EE8CFF7F19F0EF9
:1050C000E8CFF8F1C0EC0EF012006C0EB9EC1AF05B
:1050D000000EE8CF7CF0550EE8CF7DF0000EE8CF53
:1050E0007EF0000EE8CF7FF023EC1AF020EE60F0A7
:1050F000B80EDE6E1DEC0EF0190EE8CF7CF0550EEA
:10510000E8CF7DF0000EE8CF7EF0000EE8CF7FF014
:1051100023EC1AF020EE60F0B80EDE6E1DEC0EF0FF
:10512000320EE8CF7CF0550EE8CF7DF0000EE8CFD0
:105130007EF0000EE8CF7FF023EC1AF020EE60F056
:10514000B80EDE6E1DEC0EF04B0EE8CF7CF0550E67
:10515000E8CF7DF0000EE8CF7EF0000EE8CF7FF0C4
:1051600023EC1AF020EE60F0B80EDE6E1DEC0EF0AF
:10517000640EE8CF7CF0550EE8CF7DF0000EE8CF4E
:105180007EF0000EE8CF7FF023EC1AF020EE60F006
:10519000B80EDE6E1DEC0EF0BAC139F1000E394FBB
:1051A000000E394F190E394F320E394F4B0E394F11
:1051B000640EE8CF7CF0550EE8CF7DF0000EE8CF0E
:1051C0007EF0000EE8CF7FF023EC1AF020EE60F0C6
:1051D000B70EDE6E1DEC0EF01200000EE8CFF4F1FB
:1051E000380EE8CFF5F1580EE8CFF6F1450EE8CFCE
:1051F000F7F1730EE8CFF8F1C0EC0EF0230E75EC6A
:1052000010F0E8CFF4F13A0EE8CFF5F1560EE8CF02
:10521000F6F1460EE8CFF7F1720EE8CFF8F180EC28
:105220000EF03C0EE8CF7CF0470EE8CF7DF0000E8C
:10523000E8CF7EF0010EE8CF7FF01FEC1AF020EEF1
:1052400060F0430EDE6E460EDE6E39C132F1386B11
:10525000382B376B1BEC0DF0210EDE6E1DEC0EF0C3
:10526000000EE8CF7FF023EC1AF01200680EB9ECC4
:105270001AF0690EB9EC1AF0000EE8CFF4F1190E2D
:10528000E8CFF5F1780EE8CFF6F1520EE8CFF7F15E
:105290009F0EE8CFF8F1C0EC0EF0230E75EC10F085
:1052A000E8CFF4F1190EE8CFF5F1780EE8CFF6F17A
:1052B000520EE8CFF7F19F0EE8CFF8F180EC0EF038
:1052C00025EE33F0100E0A6F096B230E75EC10F00B
:1052D000E8CFF4F11C0E0925E8CFF5F11C0E0925E5
:1052E000E8CFF6F1092B092B640EE8CFF7F1DECFFA
:1052F000F8F1D890F833D890F833640EF8279D0E63
:10530000F861F86FC0EC0EF00A2FDFD725EE43F0FE
:10531000100E0A6F096B230E75EC10F0E8CFF4F154
:10532000560E0925E8CFF5F1560E0925E8CFF6F11E
:10533000092B092B640EE8CFF7F1DECFF8F1D890F6
:10534000F833D890F833640EF8279D0EF861F86FA3
:10535000C0EC0EF00A2FDFD7540EE8CF7DF0200E00
:10536000E8CF7CF023EC1AF020EE60F04E0EDE6EFB
:10537000320EDE6E1DEC0EF0540EE8CF7DF05A0EAC
:10538000E8CF7CF023EC1AF020EE60F0480EDE6EE1
:10539000650EDE6E1DEC0EF063C50AF120EE60F0C6
:1053A00015EE33F00A2BE6CF32F10A2FFCD7386B1B
:1053B000382B376B1BEC0DF0250EDE6E200EDE6EEB
:1053C000540EE8CF7DF03E0EE8CF7CF0000EE8CF23
:1053D0007EF023EC1AF01DEC0EF01F9F230E75ECEF
:1053E00010F0E8CFF4F1490EE8CFF5F14A0EE8CF1E
:1053F000F6F1790EE8CFF7F19D0EE8CFF8F180ECE9
:105400000EF0230E75EC10F0E8CFF4F13D0EE8CF6E
:10541000F5F1540EE8CFF6F1790EE8CFF7F17A0EF8
:10542000E8CFF8F1C0EC0EF0230E75EC10F0E8CFE9
:10543000F4F1410EE8CFF5F1500EE8CFF6F1820E0F
:10544000E8CFF7F1830EE8CFF8F1C0EC0EF0230EB1
:1054500075EC10F0E8CFF4F1410EE8CFF5F1500E05
:10546000E8CFF6F18B0EE8CFF7F18C0EE8CFF8F12C
:10547000C0EC0EF0230E75EC10F0E8CFF4F1410E05
:10548000E8CFF5F1500EE8CFF6F1940EE8CFF7F142
:10549000950EE8CFF8F1C0EC0EF0230E75EC10F08D
:1054A000E8CFF4F13D0EE8CFF5F1540EE8CFF6F178
:1054B0009D0EE8CFF7F19E0EE8CFF8F1C0EC0EF0AC
:1054C000120083EC2BF0010EE8CF7FF0030E58ECB6
:1054D0000BF0000EE8CF7FF0440E58EC0BF0450EB9
:1054E00058EC0BF0460E58EC0BF0470E58EC0BF056
:1054F000480E58EC0BF0490E58EC0BF04A0E58ECE5
:105500000BF0120083EC2BF0010EE8CF7FF0030EBE
:1055100058EC0BF0000EE8CF7FF04B0E58EC0BF080
:105520004C0E58EC0BF04D0E58EC0BF04E0E58ECA8
:105530000BF04F0E58EC0BF0500E58EC0BF0510ED8
:1055400058EC0BF0120083EC2BF0010EE8CF7FF04B
:105550000F0E55EC0BF0000EE8CF7FF0100E55EC5F
:105560000BF0110E55EC0BF0120E55EC0BF0130E68
:1055700055EC0BF012002BB512006A0EB9EC1AF0C4
:10558000A80EE8CF7CF0410EE8CF7DF0000EE8CF0A
:105590007EF0000EE8CF7FF020EE60F018C532F10B
:1055A000326708D023EC1AF0070E4EEC0BF01DEC1E
:1055B0000EF012008DC14CF18EC14DF10A0E4E6FEE
:1055C0004F6B08EC0CF04967486959C1E8FF486126
:1055D00003D048C118F52FD08DC14CF18EC14DF1CB
:1055E0000A0E4E6F4F6B08EC0CF048C14CF149C1EC
:1055F0004DF1D0C14EF14F6BEBEC0BF048C154F1C3
:1056000049C155F159C1E8FF640DF3CF52F1F4CF10
:1056100053F1D4EC0BF01FA70CD048C14CF149C199
:105620004DF1640E4E6F4F6B08EC0CF048C118F54D
:1056300002D059C118F5040E47EC1AF018C532F122
:10564000336B1F8F030E24EC0DF01F9F1DEC0EF02B
:1056500023EC1AF0120030EC80F001011A0E55EC28
:105660000BF020EE60F0230EDE6E63C532F163C5F1
:105670000AF11F8F386B382B376B1BEC0DF0200EA7
:10568000DE6E280EDE6E100E0A6105D04E0EDE6E46
:10569000320EDE6E04D0480EDE6E650EDE6E290E12
:1056A000DE6E200EDE6E640EE8CF7DF0190EE8CFC0
:1056B0007CF0000EE8CF7EF023EC1AF01DEC0EF02B
:1056C00020EE60F015EE33F00A2BE6CF32F10A2F10
:1056D000FCD7386B382B376B1BEC0DF0250EDE6ECC
:1056E000200EDE6E640EE8CF7DF0320EE8CF7CF047
:1056F000000EE8CF7EF023EC1AF01DEC0EF01F9F99
:105700001200000E03D0230E75EC10F0E8CFF4F178
:10571000000EE8CFF5F11A0EE8CFF6F1000EE8CF53
:10572000F7F19F0EE8CFF8F1C0EC0EF012002BB5A8
:10573000120028BF12002ABB12002BB912006B0EF8
:10574000B9EC1AF05A0EE8CF7CF0000EE8CF7DF0ED
:10575000000EE8CF7EF0020E47EC1AF020EE60F06B
:10576000430EDE6E4E0EDE6E530EDE6E3A0EDE6EB3
:1057700065C532F11F8F386B382B376B1BEC0DF082
:105780001F9F250EDE6E1DEC0EF01200400E9FECEA
:105790000DF0010EA86229D0C80EE8CF7CF0000EF3
:1057A000E8CF7DF0000EE8CF7EF0000EE8CF7FF06E
:1057B0001BEC1AF020EE60F0400E326F180E336FC3
:1057C000322BF0EC2BF07D0EA86201D004D0A8CFD4
:1057D000DEFF332FF5D71DEC0EF023EC1AF012008C
:1057E00032C1A9FFC8EC0DF01200180E396FC80EB7
:1057F000E8CF7CF0000EE8CF7DF014EC1DF0120035
:10580000000EE8CF7DF0A00EE8CF7CF020EE60F037
:105810001DC532F1386B382B376B1BEC0DF01DECCE
:105820000EF0190EE8CF7DF0A00EE8CF7CF039EC39
:105830000EF020EE60F01CC532F1386B382B376B60
:105840001BEC0DF01DEC0EF0320EE8CF7DF0A00E3B
:10585000E8CF7CF020EE60F01BC532F1386B382BBE
:10586000376B1BEC0DF01DEC0EF04B0EE8CF7DF00E
:10587000A00EE8CF7CF020EE60F033C132F1386B3F
:10588000382B376B1BEC0DF01DEC0EF01200000EE8
:10589000E8CFF4F1000EE8CFF5F1EF0EE8CFF6F126
:1058A000520EE8CFF7F19F0EE8CFF8F1C0EC0EF002
:1058B00012004FC20AF14EC209F1095303E066EC2F
:1058C0002CF01200F20E58EC0BF01200090EE66FED
:1058D000E70EE76F12EE50F0190EE72773EC2CF08D
:1058E000E62FFAD712001F8F640EE8CF7DF0E7C1D4
:1058F0007CF0E7C133F1E6CF32F1325120EE60F0B7
:10590000386B382B376B1BEC0DF06D0EDE6E1DEC1B
:105910000EF08C0EE8CF7DF0E7C17CF0E6CF32F1DF
:1059200020EE60F0386B382B376B16EC0DF0270E3D
:10593000DE6E1DEC0EF0120029B164D06D0EB9ECD4
:105940001AF0000EE8CF7DF0000EE8CF7EF01F8F3A
:10595000020E0A6F0A0E096F336B332B040E0A27EF
:1059600020EE60F0470EDE6E33C132F1386B382B1B
:10597000376B1BEC0DF03A0EDE6E0AC1A9FFC8ECC6
:105980000DF0A8CF32F1386B382B376B1BEC0DF0D4
:105990002F0EDE6EA92AC8EC0DF0A8CF32F1386BBD
:1059A000382B376B1BEC0DF0200EDE6E33511B0FC6
:1059B0009FEC0DF0A8CF32F1386B382B376B05EC2C
:1059C0000DF06D0EDE6E1B0E9FEC0DF033C132F14B
:1059D000A832322FFDD7D8B004D04A0E1DEC10F0FB
:1059E00002D023EC1AF0190E0927000EE8CF7DF043
:1059F00009C17CF01DEC0EF023EC1AF0050E3363A8
:105A0000ACD71200000EE8CF7DF0000EE8CF7EF09C
:105A10001F8F230E0A6F0A0E096FE66B0A2BE62B07
:105A2000190E0927000EE8CF7DF009C17CF020EEA9
:105A300060F0530EDE6E500EDE6EE6C132F1386B52
:105A4000382B376B1BEC0DF03A0EDE6E200EDE6E3F
:105A50000AC1A9FFC8EC0DF0A8CF32F1336B030ED9
:105A600024EC0DF01DEC0EF0030EE663D7D7210EEB
:105A70009FEC0DF0A8CFD1F1D105040DF350070F25
:105A8000A96EC8EC0DF0A8CF33F1D105040DF35089
:105A9000060FA96EC8EC0DF0A8CF32F1000EE8CFCA
:105AA0007DF06E0EE8CF7CF020EE60F0440EDE6EEE
:105AB000690EDE6E6C0EDE6E3A0EDE6E386B382BC3
:105AC000376B1BEC0DF02F0EDE6E33C132F1386BED
:105AD000382B376B1BEC0DF01DEC0EF01F9F1200E6
:105AE00025BD12001A0E9FEC0DF0A8CF0AF1690E29
:105AF0000A611200630E0A65120032C14CF133C113
:105B00004DF1640E4E6F4F6BEBEC0BF00AC14EF192
:105B10004F6B2FEC0CF048C132F149C133F1120048
:105B20003B6F010EBD27000EBE23BEAF02D0BD6B82
:105B3000BE6B3B2FF6D712003B6F010EBD5F000E10
:105B4000BE5BBEAF02D07F0EBE6F3B2FF6D71200FA
:105B50009CD8010EBD27000EBE232391BEAF1200BC
:105B6000BD6BBE6B2381120023B31CD823A30BD8BB
:105B70002383000EBD2BBE232391BEAF1200BD6B4D
:105B8000BE6B238112003B6FC580A3D8A60EC96EE1
:105B9000A0D894D8BEC1C9FF9CD890D8BDC1C9FFB8
:105BA00098D88CD83BC1C9FF94D888D812003B6BD9
:105BB0003C6B229F229DC5848CD8C5808AD8A60EB6
:105BC000C96E87D8C5BCF7D73CC1C9FF82D876D883
:105BD0003BC1C9FF7ED872D8C5827BD8A70EC96EDB
:105BE00078D86CD8C58675D822BD05D0228DFD0E1B
:105BF000C962229D11D022BF05D0228FFD0EC9623D
:105C000009D00AD0FE0EC96205D03BC1BDF13CC12E
:105C1000BEF10DD0229F229D010E3B27000E3C239A
:105C20003CBF03D0C58855D8DDD7BD6BBE6BC584DE
:105C300050D8229F229D1200C5844BD8C58049D8D8
:105C4000A60EC96E46D8C5BCF7D7BEC1C9FF41D89C
:105C500035D8BDC1C9FF3DD831D8C5823AD8A70EC5
:105C6000C96E37D82BD8C58634D8C950C58431D829
:105C70001200E2DF010EBD27000EBE232391BEAF4E
:105C80001200BD6BBE6B238112003B6FC58021D813
:105C9000A60EC96E1ED812D8BEC1C9FF1AD80ED81A
:105CA000BDC1C9FF16D80AD83BC1C9FF12D806D852
:105CB000C5840FD8060ED5EC0CF01200C5BC01D877
:105CC00012004D0EB9EC1AF081880BD89E96C46B69
:105CD0001200C42F01D0F5D79EA6FBD7C46B9E96A9
:105CE0001200C66A4E0EB9EC1AF0C56AC76A9496DD
:105CF00094888296090EC46F8286000082B804D010
:105D000082968296C42FF8D79486C66A0A0ED5EC7E
:105D10000CF0000EC76E280EC66E000EC56E080E83
:105D2000C86E81984F0EB9EC1AF01200C56FC5808D
:105D3000D0DF900EC96ECDDFC1DFC5C1C9FFC9DF9D
:105D4000BDDFC584C6DF12009E96C580C2DF910EFE
:105D5000C96EBFDFB3DFC586BCDFC9CFC5F1C5885B
:105D6000B8DFC584B6DF12002595299528EC0FF021
:105D7000259325972599BC6BBB6BC16B010EE8CFB2
:105D80007FF00C0E58EC0BF0000EE8CF7FF0A56B07
:105D9000A66B71EC2EF0D7EC2DF0396B3A6B050E3B
:105DA000BA6F010EE8CF7FF00C0E58EC0BF0000E2E
:105DB000E8CF7FF0229D229F010EA527000EA6238B
:105DC000A6BF27D0010E9CEC2DF01CEC2EF022BDBE
:105DD00005D0228DFA0EC962229D10D022BF05D0B7
:105DE000228FFA0EC96207D809D0BDC1BFF1BEC16A
:105DF000C0F1C12B13D0229F229D1200010E392722
:105E0000000E3A233ABF01D0D7D725A9F6EF12F0FA
:105E10002CD0C151D8B4F9D7258327D0030E90ECEC
:105E20002DF025A704D0A751C163DED264D025B3DD
:105E30001CD0F5DA050EBA6316D0C1C1ACF1BFC1F2
:105E4000AAF1C0C1ABF1A5C191F1A6C192F139C1CE
:105E5000F0F13AC1A8F1030EAA27000EAB23030EFE
:105E6000915F000E925BBA2FBFD225A97DD783EC3C
:105E70002BF0010EE8CF7FF01A0E58EC0BF0000E5D
:105E8000E8CF7FF00B0E58EC0BF020992191219375
:105E9000219724992497B86B010E25B5AD51BA6F9F
:105EA000259525999AEC1DF0FAEC31F021B3A7D293
:105EB00021B10ED020B1F5EC3DF020B1E3EC43F080
:105EC000209120B9F6EF12F020B3B4EF4AF0ECD7EE
:105ED0002191060EBA6302D0F6EF12F0BAC1ADF10D
:105EE0002585BB51050DF350BA25A76F28EC0FF09F
:105EF0002587C16B43D7259707EC1DF0000EE8CF2F
:105F00007CF0000EE8CF7DF020EE60F0230EDE6E18
:105F10001C0E89EC10F0326703D0336701D016D025
:105F2000010E3227000E332332C152F133C153F137
:105F3000A7C154F1556BD4EC0BF050C132F151C1F3
:105F400033F11F8F0A0E24EC0DF007D0A7C132F1F8
:105F5000386B382B376B16EC0DF0200EDE6E39ECFB
:105F60002EF0C9CF32F139EC2EF0C9CF32F1BDC1DC
:105F7000AFF1BEC1AEF1200E90EC2DF01CEC2EF076
:105F8000C9CFA9F1AFC1BDF1AEC1BEF132C1F1F1CE
:105F900039EC2EF0C9CFF2F139EC2EF0C9CFF3F184
:105FA00071EC24F0200EDE6E39EC2EF0C9CF32F108
:105FB000386B382B376B16EC0DF03A0EDE6E39EC81
:105FC0002EF0C9CF32F1386B382B376B16EC0DF051
:105FD0001DEC0EF0190EE8CF7CF0050EE8CF7DF039
:105FE00020EE60F039EC2EF0C9CF32F139EC2EF012
:105FF000C9CF33F132C14CF133C14DF1A40E4E6F14
:106000004F6B08EC0CF048C1C6F149C1C7F1C62B73
:10601000000EC7231F8F030E24EC0DF06D0EDE6EF5
:10602000200EDE6E39EC2EF0C9CF32F139EC2EF0B5
:10603000C9CF33F132C14CF133C14DF13C0E4E6F3B
:106040004F6BEBEC0BF01F8F386B382B376B3751E6
:1060500024EC0DF0270EDE6E39EC2EF0C9CF32F1B4
:1060600032514827000E492348C14CF149C14DF136
:106070009F0E4E6F4F6B08EC0CF048C14CF149C1BC
:106080004DF1A9514E6F4F6B08EC0CF048C1C8F1AF
:1060900049C1C9F1C82B000EC9231F8F386B382B9B
:1060A000376B16EC0DF0220EDE6E200EDE6E39EC34
:1060B0002EF0C9CF32F139EC2EF0C9CF33F1030EF7
:1060C000386F1F8F020E24EC0DF0B00EDE6E430E03
:1060D000DE6E1DEC0EF0320EE8CF7CF0050EE8CF40
:1060E0007DF020EE60F039EC2EF0C9CF32F139ECC2
:1060F0002EF0C9CF33F11F8F386B382B376B3751E8
:1061000024EC0DF06D0EDE6E620EDE6E610EDE6E44
:10611000720EDE6E200EDE6E440EDE6E650EDE6EDC
:10612000730EDE6E610EDE6E740EDE6E200EDE6E9F
:1061300039EC2EF0C9CF32F139EC2EF0C9CF33F162
:10614000B1EC0BF01F8F325133C132F1336F386B2A
:10615000382B376B1BEC0DF03A0EDE6E33C132F18B
:10616000386B382B376B16EC0DF01F9F1DEC0EF0C3
:1061700039EC2EF039EC2EF039EC2EF039EC2EF013
:1061800039EC2EF039EC2EF039EC2EF039EC2EF003
:1061900039EC2EF039EC2EF039EC2EF039EC2EF0F3
:1061A00039EC2EF039EC2EF039EC2EF039EC2EF0E3
:1061B00039EC2EF039EC2EF039EC2EF0C9CFB1F1DC
:1061C000B199B19BB19DB19FB12BB1C1EBF139EC4C
:1061D0002EF0C9CFB2F1B299B29BB29DB29FB2C1BB
:1061E000ECF139EC2EF0C9CFB3F139EC2EF0C9CF78
:1061F000B4F139EC2EF0C9CFB5F139EC2EF0C9CF9E
:10620000B6F139EC2EF039EC2EF0010EE8CFF4F1B6
:106210004B0EE8CFF5F1EF0EE8CFF6F1000EE8CF28
:10622000F7F19F0EE8CFF8F1C0EC0EF039EC2EF04C
:10623000B86B39EC2EF09E0E386F229F050EB96FA9
:106240004B0EDC6FB9292AEC0EF0C8C1CAF1C9C1E6
:10625000CBF1CB2B61D822BF23D0C6C14EF1C7C131
:106260004FF132C14CF133C14DF108EC0CF04B0E43
:10627000482769EC31F048C1DCF1485139EC0EF0A7
:10628000B92BB9512AEC0EF023EC1AF043EC0EF0C6
:10629000CA4F02D041D8FCD7CB2FFAD7382FD5D749
:1062A00020992191219324992497B86BFAEC31F02D
:1062B00021B177D021B375D020B1F5EC3DF020B1FC
:1062C000E3EC43F0209120B96CD020B3B4EF4AF056
:1062D000EDD74851DC6301D012004851DC650ED087
:1062E000DCC149F14907495139EC0EF023EC1AF0B1
:1062F0006CEC0EF048514963F5D7120048C149F1E2
:106300004907495139EC0EF023EC1AF06CEC0EF011
:10631000DC514963F5D7120039EC2EF0C9CF32F1C8
:1063200039EC2EF0C9CF33F139EC2EF0C9CFB8F1EA
:10633000289BB8BF288BB89FFD0E326305D0FD0E99
:10634000336302D0228F1200B22F23D0ECC1B2F1FE
:1063500028AB11D039EC2EF0B807000EC9B8020FE7
:10636000C9BA010FEF6FEF6701D005D039EC2EF0FD
:10637000B807EF2FFBD7040EB86306D039EC2EF028
:10638000B80739EC2EF0B80739EC2EF0B82FFCD74F
:106390001200B86701D0120039EC2EF0B82FFCD7EC
:1063A00012002099B86BAAC1BDF1ABC1BEF191C179
:1063B000A5F192C1A6F1ACC1C1F1F0C139F1A8C1FA
:1063C0003AF1C1072593BB07BC6B050EBA6FBB2B17
:1063D00028EC0FF0E6D425B3B5EF2EF0BC6B050E1C
:1063E000BA6FBB2B28EC0FF0BFC1BDF1C0C1BEF12D
:1063F000D1EF2EF024B9218324B721811200BA2BCA
:10640000070EBA6301D0E7D7BC29BA6302D0060EE3
:10641000BA6FB86B9AEC1DF02499219345D5258964
:10642000BC2B29B50CD083EC2BF0010EE8CF7FF00C
:106430001A0E58EC0BF0000EE8CF7FF02985140EF1
:10644000E8CF7DF0BB51050DF350C15D1E0DF3503B
:10645000050FE8CF7CF020EE60F0C1C132F1386B5F
:10646000382B376B16EC0DF0200EDE6E39EC2EF06B
:10647000C9CF32F10D0E326504D039EC2EF0C9CF00
:1064800032F132C1F1F139EC2EF0C9CFF2F139EC31
:106490002EF0C9CFF3F1C7EC24F039EC2EF039EC33
:1064A0002EF0200EDE6E39EC2EF0C9CF32F139EC31
:1064B0002EF0C9CF33F11F8F2485030E24EC0DF08D
:1064C0006D0EDE6E200EDE6E39EC2EF0C9CF32F18D
:1064D00039EC2EF0C9CF33F11F8F386B382B376B67
:1064E000375124EC0DF0270EDE6E1DEC0EF012007D
:1064F0002D939D9A818616EC4CF06B0EAD6EF1ECEF
:106500000DF081969D8A74EF3CF028959D9A8186C6
:1065100020EC80F0010130EC80F0010118EC80F0FB
:106520000101010ECC6FCD6B680EAD6EF1EC0DF07C
:10653000208581969D8A74EF3CF028939D9A8186F0
:10654000AA6AA3D881969D8A74EF3CF02A9F9D9AEF
:106550008186010EAA6E99D8AA6A81969D8A74EFE7
:106560003CF0279F9D9A8186F1EC0DF0010EAD6EF7
:10657000F1EC0DF03E0EAD6E29EE4AF0100E396FC3
:10658000F1EC0DF0DECFADFF392FFAD781969D8A61
:1065900074EF3CF0259B9D9A818628EC0FF083ECEC
:1065A0002BF0010EE8CF7FF00F0E58EC0BF0000E31
:1065B000E8CF7FF0050E436FAA0EAD6EF1EC0DF043
:1065C000432FFAD7550EAD6E100E58EC0BF0D7ECEA
:1065D0002DF0010EBD27000EBE23110E58EC0BF05E
:1065E00054D8F1EC0DF0C2C1ADFFF1EC0DF0C3C118
:1065F000ADFFF1EC0DF0010EAD6EF1EC0DF03E0EC5
:10660000AD6E120E58EC0BF0436B446BC58069EC19
:106610002EF0A60EC96E69EC2EF0C5BCF7D7BEC130
:10662000C9FF69EC2EF05EEC2EF0BDC1C9FF69EC2C
:106630002EF05EEC2EF0C58269EC2EF0A70EC96E2E
:1066400069EC2EF05EEC2EF0130E58EC0BF0F1EC32
:106650000DF0C58669EC2EF0C9CFADFF010E4327C2
:10666000000E442344BF04D0C58869EC2EF0EFD758
:10667000C58469EC2EF0140E58EC0BF0FA0ED5EC34
:106680000CF081969D8A01EF3CF0436BA96AC8EC3F
:106690000DF0A8CFADFFA92AF1EC0DF0432FF7D7ED
:1066A0001200010EBA6F219921972099AA6B229DA1
:1066B000229F28EC0FF083EC2BF0010EE8CF7FF047
:1066C0006F0E58EC0BF0000EE8CF7FF0B86B219105
:1066D0002193140EE8CF7DF0230EE8CF7CF020EE5E
:1066E00060F0700E51EC0BF0AAC132F1322B1F8F0B
:1066F000386B382B376B05EC0DF0200EDE6E280E54
:10670000DE6EC00E51EC0BF0200EDE6E210E9FEC03
:106710000DF0A8CFD1F1D105040DF350060FA96EED
:10672000C8EC0DF0A8CF32F11F8F386B382B376BC8
:1067300005EC0DF02F0EDE6ED105040DF350070FA2
:10674000A96EC8EC0DF0A8CF32F11F8F386B382B33
:10675000376B05EC0DF0290EDE6E1DEC0EF0140EFD
:10676000E8CF7DF0410EE8CF7CF020EE60F0610EC6
:1067700051EC0BF0AA51240FA96EC8EC0DF0A8CF74
:1067800032F1336B1F8F030E24EC0DF01F9F420E6E
:10679000DE6E610EDE6E720EDE6E200EDE6E1DECA3
:1067A0000EF0140EE8CF7DF05F0EE8CF7CF020EE07
:1067B00060F0BE0E51EC0BF01DEC0EF0140EE8CFA5
:1067C0007DF07D0EE8CF7CF020EE60F0BF0E51EC46
:1067D0000BF01DEC0EF0140EE8CF7DF09B0EE8CF11
:1067E0007CF020EE60F0590E51EC0BF0310EDE6EB5
:1067F0002E0EDE6E300EDE6E300EDE6E1DEC0EF0F6
:106800000B0E58EC0BF0F3EC12F09AEC1DF0FAECD6
:1068100031F021B30FD021B11ED020B3B4EF4AF034
:1068200020B1F5EC3DF020B1E3EC43F0209120B92C
:106830001CD0EDD7BA2B020EBA6301D0BA2B070ECB
:10684000BA6302D0010EBA6FB86B9AEC1DF0F3EC8C
:1068500012F02193DCD7BA4F3ED0BA4F0AD0BA4FCC
:1068600008D0BA4F1AD0BA4F2CD0020EBA6F4AEFE6
:1068700013F0AA51240FA96EC8EC0DF0A8CF32F185
:10688000322BFB0E326302D0FA0E326F32C1A8FFF8
:10689000CCEC0DF0030EBA6F19D7AA51240FA96ED4
:1068A000C8EC0DF0A8CF32F13207FF0E326302D0F0
:1068B000000E326F32C1A8FFCCEC0DF0040EBA6F9F
:1068C00005D7AA51240FA96E640EA86ECCEC0DF06A
:1068D000050EBA6FFBD6AA2B030EAA6301D0AA6BD2
:1068E000010EBA6FF3D628EC0FF083EC2BF0010EFB
:1068F000E8CF7FF0720E58EC0BF0000EE8CF7FF07F
:10690000230EE8CF7CF0000EE8CF7DF0000EE8CF3C
:106910007EF020EE60F0730E51EC0BF0320E9FEC27
:106920000DF0A8CF32F1330E9FEC0DF0A8CF33F16C
:106930001F8F386B382B376B375124EC0DF0200E3E
:10694000DE6E280EDE6E340E9FEC0DF0A8CF32F115
:10695000350E9FEC0DF0A8CF33F11F8F386B382B1D
:10696000376B375124EC0DF0290EDE6E1DEC0EF066
:10697000410EE8CF7CF020EE60F0750E51EC0BF08C
:106980002F0E9FEC0DF0A8CFF1F1300E9FEC0DF023
:10699000A8CFF2F1310E9FEC0DF0A8CFF3F171EC1E
:1069A00024F01DEC0EF05F0EE8CF7CF020EE60F0DE
:1069B000760E51EC0BF0280E9FEC0DF0A8CF32F1C3
:1069C000290E9FEC0DF0A8CF33F1010E386F1F8F09
:1069D000020E24EC0DF01F9F560EDE6E1DEC0EF025
:1069E0007D0EE8CF7CF020EE60F0770E51EC0BF0DE
:1069F0002A0E9FEC0DF0A8CFF1F12B0E9FEC0DF0BD
:106A0000A8CFF2F12C0E9FEC0DF0A8CFF3F171ECB2
:106A100024F01DEC0EF09B0EE8CF7CF020EE60F031
:106A2000780E51EC0BF0360E9FEC0DF0A8CF32F142
:106A3000370E9FEC0DF0A8CF33F1030E386F1F8F88
:106A4000020E24EC0DF01F9FB00EDE6E200EDE6EE7
:106A5000280EDE6E380E9FEC0DF0A8CFF1F1390E46
:106A60009FEC0DF0A8CFF2F13A0E9FEC0DF0A8CFFD
:106A7000F3F171EC24F0290EDE6E200EDE6E1DECBB
:106A80000EF0B90EE8CF7CF020EE60F0790E51ECFC
:106A90000BF03B0E9FEC0DF0A8CF32F13C0E9FECBB
:106AA0000DF0A8CF33F1030E386F1F8F020E24ECC8
:106AB0000DF01F9FB00EDE6E200EDE6E280EDE6E15
:106AC0003D0E9FEC0DF0A8CFF1F13E0E9FEC0DF0C6
:106AD000A8CFF2F13F0E9FEC0DF0A8CFF3F171ECCF
:106AE00024F0290EDE6E200EDE6E1DEC0EF081A06D
:106AF000FED7249724992191FAEC31F021B10DD0E1
:106B000020B3B4EF4AF020B1F5EC3DF020B1E3EC56
:106B100043F0209120B901D0EFD7030EBA6F4AEFAE
:106B200013F0010EBA6F28EC0FF037EC3AF0B86BA7
:106B300020992191219383EC2BF0010EE8CF7FF077
:106B40006A0E58EC0BF0000EE8CF7FF0AA6BA56B35
:106B5000050E096F020E0A6F140EE8CF7DF0040EC9
:106B60000A271E0E09270951E8CF7CF020EE60F0BD
:106B7000470EDE6EAAC132F1322B1F8F386B382BD5
:106B8000376B05EC0DF03A0EDE6EDFEC39F01DECE4
:106B90000EF0280EE8CF7DF00951E8CF7CF020EE12
:106BA00060F0210EA96EC8EC0DF0A804AA6302D013
:106BB0002A0EDE6EDFEC39F01DEC0EF0300EE8CF61
:106BC0007DF00951E8CF7CF020EE60F00AC1A9FF0A
:106BD000A92AC8EC0DF0A8CF32F13253000E32656D
:106BE0001AD0D8EC39F00AC1A9FFC8EC0DF0A8CF33
:106BF00032F1386B382B376B1BEC0DF02F0EDE6E3D
:106C0000A92AC8EC0DF0A8CF32F1386B382B376BBE
:106C10001BEC0DF03FD00AC1A9FFC8EC0DF0A8CFC6
:106C200032F13253150E326517D0640E326108D03E
:106C3000D1EC39F0386B382B376B1BEC0DF02AD0C8
:106C40004F0EDE6E320EDE6E200EDE6E386B382B8F
:106C5000376B1BEC0DF01ED032633DEC36F0410E6D
:106C6000DE6E490EDE6E520EDE6E200EDE6E386B6C
:106C7000382B376B1BEC0DF00DD0450EDE6E520E2F
:106C8000DE6E520EDE6E200EDE6E386B382B376BEA
:106C90001BEC0DF0DFEC39F01DEC0EF0690EE8CFC7
:106CA0007DF00951E8CF7CF020EE60F0200EDE6E22
:106CB000690EDE6E6E0EDE6E200EDE6EAA511C0FA9
:106CC000A96EC8EC0DF0A8CF32F1386B382B376BBA
:106CD0001BEC0DF06D0EDE6EDFEC39F01DEC0EF0EE
:106CE00023EC1AF0AA2B050EAA63ACEF35F00B0EBD
:106CF00058EC0BF0F3EC12F09AEC1DF0FAEC31F0DA
:106D000021B30FD021B11ED020B3B4EF4AF020B18F
:106D1000F5EC3DF020B1E3EC43F0209120B90ED02A
:106D2000EDD7BA2B070EBA6302D0010EBA6FB86B5B
:106D30009AEC1DF0F3EC12F02193E0D7020EBA6F3B
:106D4000F9EF12F0BA4F09D0BA4F0CD0BA4F0FD0AA
:106D5000BA4F12D0BA4F15D0F1D7000EAA6F000E5D
:106D6000A56F14D0010EAA6F040EA56F0FD0020EEE
:106D7000AA6F080EA56F0AD0030EAA6F0C0EA56F9E
:106D800005D0040EAA6F100EA56F00D0010EBA6FC9
:106D90002993219921972099229D28EC0FF01E0E0E
:106DA00058EC0BF00B0E58EC0BF0B86B21912193C3
:106DB0004ADA410EE8CF7CF0140EE8CF7DF020EEE9
:106DC00060F04F0EDE6E320EDE6E3A0EDE6E200E7C
:106DD000DE6EA551060FA96EC8EC0DF0A8CF32F1FA
:106DE000386B382B376B1BEC0DF0250EDE6E200E4A
:106DF000DE6E280EDE6E4D0EDE6E4F0EDE6E440E23
:106E0000DE6E3A0EDE6E120E75EC10F00A0DF3CF48
:106E10004CF1F4CF4DF1A551060FA96EC8EC0DF061
:106E2000A8CF4EF14F6B08EC0CF00A0E485F48C13A
:106E300032F1000E495B49C133F1386B382B376BA7
:106E4000375124EC0DF06D0EDE6E290EDE6E200E35
:106E5000DE6E200EDE6E1DEC0EF05F0EE8CF7CF0D5
:106E600020EE60F0480EDE6E650EDE6E3A0EDE6ECF
:106E7000200EDE6EA551070FA96EC8EC0DF0A8CF4D
:106E800032F1386B382B376B1BEC0DF0250EDE6EB4
:106E9000200EDE6E200EDE6E1DEC0EF07D0EE8CFB5
:106EA0007CF020EE60F02B0EDE6E2F0EDE6E2D0ECF
:106EB000DE6E3A0EDE6E200EDE6E2B0E22BD2D0E25
:106EC000DE6E1DEC0EF09B0EE8CF7CF020EE60F045
:106ED000590E51EC0BF0A551040FA96EC8EC0DF042
:106EE000A8CF32F1386B382B376B1BEC0DF02F0E1F
:106EF000DE6EA551050FA96EC8EC0DF0A8CF32F1DA
:106F0000386B382B376B1BEC0DF0200EDE6E200E2D
:106F1000DE6E1DEC0EF0F3EC12F09AEC1DF0FAECC4
:106F200031F021B30FD021B11AD020B3B4EF4AF021
:106F300020B1F5EC3DF020B1E3EC43F0209120B915
:106F400018D0EDD7BA2B070EBA6302D0010EBA6F74
:106F5000B86B9AEC1DF0F3EC12F02193E0D7BA4F26
:106F600090D0BA4F11D0BA4F43D0BA4F06D0BA4FD3
:106F700069D0AAC1BAF1BA2BD6D5227D040EBA6F58
:106F800014D7010EBA6F09D7A551060FA96EC8EC28
:106F90000DF0A8CF32F122BD07D0322B650E32633F
:106FA00010D0040E326F0DD03207030E326309D0B9
:106FB000A551070FA96EC8EC0DF0640E326FA850F2
:106FC000325FA551070FA96EC8EC0DF0A85032250D
:106FD000336F650E336302D0040E326FA551060F76
:106FE000A96E32C1A8FFCCEC0DF0020EBA6FDDD64F
:106FF000A551070FA96EC8EC0DF0A8CF32F122BD44
:1070000006D0322B5C0E326307D0326B05D03207CC
:10701000FF0E326301D0326BA551060FA96EC8EC8A
:107020000DF0A8503225336F650E336301D032075F
:10703000A551070FA96E32C1A8FFCCEC0DF0030ECD
:10704000BA6FB3D6A551040FA96EC8EC0DF0A8CF46
:1070500032F1A551050FA96EC8EC0DF0A8CF33F1A0
:10706000A551060FA96E32C1A8FFCCEC0DF0A551B9
:10707000070FA96E33C1A8FFCCEC0DF0050EBA6F57
:1070800094D628EC0FF0010EBA6F6D0E58EC0BF091
:107090000B0E58EC0BF0B86B21912193D4D8A4D9E6
:1070A000410EE8CF7CF0140EE8CF7DF020EE60F0CA
:1070B000690E51EC0BF01B0E9FEC0DF0AAC132F1E2
:1070C000322BA832322FFDD7D8A004D0600E51EC5D
:1070D0000BF006D0200EDE6E200EDE6E200EDE6E71
:1070E0001DEC0EF05F0EE8CF7CF0140EE8CF7DF0C3
:1070F00020EE60F0580E51EC0BF0200EDE6E210EEB
:10710000A96EC8EC0DF0A804AA6304D0600E51EC7F
:107110000BF006D0200EDE6E200EDE6E200EDE6E30
:107120001DEC0EF07D0EE8CF7CF0140EE8CF7DF064
:1071300020EE60F06B0E51EC0BF01DEC0EF09B0E90
:10714000E8CF7CF0140EE8CF7DF020EE60F06C0EFE
:1071500051EC0BF01DEC0EF0F3EC12F09AEC1DF07C
:10716000FAEC31F021B30FD021B11AD020B3B4EF33
:107170004AF020B1F5EC3DF020B1E3EC43F0209172
:1071800020B9F7D6EDD7BA2B070EBA6302D0010E9D
:10719000BA6FB86B9AEC1DF0F3EC12F02193E0D7C4
:1071A000BA4FEFD6BA4F11D0BA4F05D0BA4F23D04D
:1071B000BA4F35D0DED6AAC1A8FFA82A210EA96EE3
:1071C000CCEC0DF0030EBA6F66D71B0E9FEC0DF0E2
:1071D000AAC132F1322B324FA870324FA872324F0F
:1071E000A874324FA876324FA8781B0E9DEC0DF094
:1071F000020EBA6F50D7AA511C0FA96EC8EC0DF041
:10720000A8CF32F1322B640E326302D0630E326F9C
:1072100032C1A8FFCCEC0DF0040EBA6F3CD7AA51D6
:107220001C0FA96EC8EC0DF0A8CF32F13207FF0E8B
:10723000326302D0000E326F32C1A8FFCCEC0DF0E9
:10724000050EBA6F28D783EC2BF0010EE8CF7FF044
:10725000020EE8CF7CF0000EE8CF7DF020EE60F06B
:107260005F0E51EC0BF0AAC132F1322B1F8F386B3D
:10727000382B376B05EC0DF03A0EDE6E200EDE6E0D
:107280001DEC0EF0020EE8CF7CF0320EE8CF7DF060
:1072900020EE60F0A551070FA96EC8EC0DF0A8CF45
:1072A00032F13253000E32651DD0D8EC39F0A551C1
:1072B000060FA96EC8EC0DF0A8CF32F1386B382B51
:1072C000376B1BEC0DF02F0EDE6EA551070FA96E6C
:1072D000C8EC0DF0A8CF32F1386B382B376B1BECB4
:1072E0000DF041D0A551060FA96EC8EC0DF0A8CF46
:1072F00032F13253150E3263326517D0640E3261AB
:1073000008D0D1EC39F0386B382B376B1BEC0DF013
:107310002AD04F0EDE6E320EDE6E200EDE6E386B21
:10732000382B376B1BEC0DF01ED032630ED0410EA4
:10733000DE6E490EDE6E520EDE6E200EDE6E386B95
:10734000382B376B1BEC0DF00ED0450EDE6E520E57
:10735000DE6E520EDE6E200EDE6E386B382B376B13
:107360001BEC0DF000D0200EDE6E690EDE6E6E0E90
:10737000DE6E200EDE6EAA511C0FA96EC8EC0DF059
:10738000A8CF32F1386B382B376B1BEC0DF06D0E3C
:10739000DE6E200EDE6E1DEC0EF0000EE8CF7FF0EC
:1073A00012004E0EDE6E580EDE6E200EDE6E1200E5
:1073B000540EDE6E580EDE6E200EDE6E12001B0EB8
:1073C0009FEC0DF0AAC132F1322BA832322FFDD73B
:1073D000D8A006D0230E75EC10F01DEC10F01200B2
:1073E0004A0E1DEC10F01200A551060FA96EC8EC54
:1073F0000DF0A8CF33F1AA511C0FA96EC8EC0DF007
:10740000A8CF32F10A0E322733513203F3CF4CF1B9
:10741000F4CF4DF10A0E4E6F4F6B08EC0CF048C1E3
:1074200032F149C133F1370EE8CF7DF0230EE8CFBA
:107430007CF020EE60F0280EDE6E700EDE6E700EB8
:10744000DE6E4F0EDE6E320EDE6E3A0EDE6E030E16
:1074500024EC0DF0420EDE6E610EDE6E720EDE6EFC
:10746000290EDE6E200EDE6E1DEC0EF01200030EF5
:10747000A96EAA6A20EE60F0A92AC8EC0DF0A8CF88
:10748000DEFF170EA962F8D71C0E9FEC0DF0A8CFF7
:10749000DEFF1D0E9FEC0DF0A8CFDEFF1E0E9FEC51
:1074A0000DF0A8CFDEFF1F0E9FEC0DF0A8CFDEFF82
:1074B000200E9FEC0DF0A8CFDEFF1B0E9FEC0DF011
:1074C000A8CFDEFF20EE74F0050EED6FEB6BDE5003
:1074D000EB27ED2FFCD7EB6701D012002191630E53
:1074E000EE6F2DD8050EEF6F3ED8EBC1A8FF200E32
:1074F0009DEC0DF024D8040EEF6F35D8EBC1A8FF3A
:107500001F0E9DEC0DF01BD8030EEF6F2CD8EBC1B6
:10751000A8FF1E0E9DEC0DF012D8020EEF6F23D8BF
:10752000EBC1A8FF1D0E9DEC0DF009D8010EEF6F09
:107530001AD8EBC1A8FF1C0E9DEC0DF01200EC6BED
:10754000EB6BED6B20EE74F0DE50EE6505D0EB6179
:1075500003D0EB6FECC1EDF1EC2B050EEC63F4D72F
:10756000EBC1EEF1120020EE60F0ED51040DF3508E
:10757000D926000EDA2221B10CD0210E9FEC0DF09D
:10758000ED29A86206D0EFC1A8FF210E9DEC0DF0F9
:107590002181EF51040DF3CFA9FFDECFA8FFCCEC82
:1075A0000DF0A92ADECFA8FFCCEC0DF0A92ADECF82
:1075B000A8FFCCEC0DF0A92ADECFA8FFCCEC0DF093
:1075C000120025BD1FD0AECF43F1600E435F434F85
:1075D000258B434F248B434F258D434F2681434FAB
:1075E000278F434F2881434F2883434F2885434F9C
:1075F0002B81434F2A8F434F2D83AE509E9AAB98D9
:10760000AB8812002CB7F9D78186AE6601D0AE2ABE
:10761000AE50640DF3CFC6F1F4CFC7F1EED7F292BE
:10762000D5BE09D02487D58E1200F090D5BE03D0E8
:107630002489D58E1200F294D56AD76AD66AD58E7F
:107640001200F294D59ED76AD66A1200F19C2A9154
:10765000000ED56ED58E1200F18C1200F19A2A938D
:10766000000ED56ED58E1200F18A1200A192B19E45
:10767000CA9412009E908198080ECF60412B080E8C
:10768000CF5E412B0F0E416502D0A7EC3BF020A945
:1076900001D0120023BF1200422B010E42630AD018
:1076A000239D3F6B406B9B6B9C6BF1EC18F0E1EC06
:1076B00018F01200020E42630FD0E8EC18F0EEEC66
:1076C00018F0C9EC17F08D513F278E514023975188
:1076D0009B2798519C231200030E426301D0E5D7EB
:1076E000040E426301D0E9D7050E426301D0DDD715
:1076F000060E426301D0E1D7070E426301D0D5D711
:10770000DCDF426B020E3E6FD89040333F33D8909F
:107710009C339B333E2FF8D740C18EF13FC18DF192
:107720009CC198F19BC197F1238D25AD04D0E80E43
:107730009F6F030EA06F1F979F518D5D8F6FA0519C
:107740008E59906FD8A812008F6B906B1200416B0E
:107750002081D89420A31CD0A82BA905A86502D00D
:10776000A86B2287172BD8B4182B22A911D0A72BCE
:107770003B0EA76505D0A76B2087A52BD8B4A62BF9
:107780002AAB06D0DD2B3B0EDD6502D0DD6BDC2B9A
:10779000032B3B0E03651200036B2085042B3B0E6D
:1077A00004651200046B052B170E05651200056BAE
:1077B000062B2A0E036F07C176F1764F1F0E764F08
:1077C0001C0E764F1F0E764F1E0E764F1F0E764FF5
:1077D0001E0E764F1F0E764F1F0E764F1E0E764FE3
:1077E0001F0E764F1E0E764F1F0E06651200010EFD
:1077F000066F072B0C0E07651200010E076F082B92
:107800001200FCEC4AF0326B32C118F5AFEC0FF00D
:1078100071EC2EF0DAEC0DF066EC0FF089EC26F04E
:1078200023EC1DF0FBEC24F0A3C100F5A4C101F58D
:10783000A3C102F5A4C103F528BF10D02ABB0ED006
:1078400042EC23F077EC23F02DA539EC29F02DB58F
:1078500094EC20F073EC21F0DCEC1FF028AF03D0A7
:10786000670E58EC0BF02AAB03D0740E58EC0BF0FB
:10787000B86BB96B209D209F239D956B966B996B80
:107880009A6B050EB76F81968198259D2C97000EF7
:10789000E8CF7CF0000EE8CF7DF0000EE8CF7EF060
:1078A000000EE8CF7FF023EC1AF02497249973ECB4
:1078B00021F0C6EC2BF0010ECF6F470EB9EC1AF099
:1078C0000C0E75EC10F00A6F0AC113F50B0E75EC77
:1078D00010F00A6F0AC112F530EC80F00101480E79
:1078E000B9EC1AF0F3EC12F020A119D029A101D0C3
:1078F00000D023EC1DF02BEC3DF0F5EC3DF076ECE8
:1079000048F0DDEC23F0B1EC3DF001EC3DF06EEC25
:1079100012F0DCEC1FF02CB13AEC48F02091CEECE8
:107920003DF023BDAFEC23F023BDD5EC1EF023BD0D
:10793000E3EC43F0239D20B5C6EC3CF020BFF6EF0E
:1079400012F020B301EF3EF020B97FEF47F025BBE6
:10795000CAEF32F024BBF2EF49F026B1A6EF0DF0EA
:107960002BB1A1EF0DF027BFB1EF32F028B146EFF8
:107970004AF028B39DEF32F028B585EF32F02ABFE8
:10798000A6EF32F02DB378EF32F0AED7FBEC24F057
:1079900004EC3DF09BEC49F0C6EC2BF0F1EC3CF034
:1079A00028BF0ED02ABB0CD077EC23F042EC23F09A
:1079B00020BD06D02DA539EC29F02DB594EC20F092
:1079C000E4EC3CF0209512002781010ECC5F000E04
:1079D000CD5BCC671200CD67120027918196CC2B2E
:1079E000120020C532F121C533F1326705D033676B
:1079F00003D0196B1A6B1200010E1927000E1A23FF
:107A0000120027B1817612008188490EB9EC1AF074
:107A10009FC102F5A0C103F50A6B0AC111F54F0E13
:107A20000A6F0AC110F58DC100F58EC101F50B0E6C
:107A300075EC10F00A6F0AC112F50C0E75EC10F01F
:107A40000A6F0AC113F540EC80F001014A0EB9EC4F
:107A50001AF08198120094928282249182A4248147
:107A6000829294820A0EA9EC0CF0249382A42483BF
:107A70009492829224B171D024B364D0948229A9C3
:107A800044D0299F2999320E9FEC0DF0A8CF39F1EF
:107A9000330E9FEC0DF0A8CF3AF1D890010E3927A4
:107AA000000E3A2339C1A8FF320E9DEC0DF03AC109
:107AB000A8FF330E9DEC0DF0340E9FEC0DF0A8CF17
:107AC00039F1350E9FEC0DF0A8CF3AF1D890010EA8
:107AD0003927000E3A2339C1A8FF340E9DEC0DF072
:107AE0003AC1A8FF350E9DEC0DF007C1A8FF2F0E7F
:107AF0009DEC0DF006C1A8FF300E9DEC0DF008C105
:107B0000A8FF310E9DEC0DF0120029AF1200299F45
:107B1000320E9FEC0DF0A8CF39F1330E9FEC0DF033
:107B2000A8CF3AF1D890010E3927000E3A2339C177
:107B3000A8FF320E9DEC0DF03AC1A8FF330E9DEC6C
:107B40000DF012008188640ED5EC0CF08198640E63
:107B5000D5EC0CF08188298912008188298F299918
:107B6000120020AD1200B92B040E75EC10F0B965AF
:107B70001200209D81EC2BF028BF08D02ABB06D034
:107B80002DA539EC29F02DB594EC20F0AFEC23F0C5
:107B900089EC26F0B96B24972499120024B718D0E9
:107BA00024B907D0D59EF294D76AD66AF292F090A3
:107BB0001200249983EC2BF0010EE8CF7FF0040E25
:107BC00058EC0BF0000EE8CF7FF0208DB86B120060
:107BD000249720AD02D0208F12002D752DA539ECF1
:107BE00029F02DB594EC20F01200B82B030E75ECA3
:107BF00010F0050FD8B0FF0EE806B8651200208916
:107C000012002EEC44F0520EB9EC1AF028EC0FF0F2
:107C1000ADEC1BF070EC1FF003EC1FF02ABB2087CB
:107C200028BF04D02ABB02D0D1EC1BF020A142D047
:107C300028BF09D02ABB17D029B118D000EC41F0D9
:107C4000D9EC3EF01BD020AD53EC25F071EC43F0A5
:107C50002CB328EC26F024BF04D0248F09EC44F088
:107C60000DD0249F0BD08AEC3EF008D0BBEC2AF05C
:107C7000D9EC3EF02CB502EC41F000D071EC43F0B1
:107C800023B7DDEC23F020BD80EC3EF020BF35ECC7
:107C900047F0BAEC3EF02CB13AEC48F02CB328ECAB
:107CA00026F02091260E75EC10F0326F010E326333
:107CB00001D0268326A30BD020BD08D053EC25F09D
:107CC00029B1BBEC2AF027B500EC41F0269320AF98
:107CD000E9EC44F020BF2DEC45F020A398D323BD60
:107CE00096EC43F0239D20B5B5EC43F022B7E4ECCD
:107CF0003FF020BF04D025BD02D00300000096D77E
:107D0000B92B040E75EC10F0B9651200209D19EC2A
:107D100025F01200C2EC25F022B90DD083EC25F03D
:107D2000E22B3C0EE26302D0E26BE12B269722B9F4
:107D300012002687120026A712000BD8B0EC25F0FF
:107D4000E06BE26BE16BDD6BDC6B916B926B26970A
:107D50001200DEC152F1DFC153F191C154F192C161
:107D600055F1D4EC0BF01FA7120091C1DEF192C1C6
:107D7000DFF11200819832C532F10E0E75EC10F071
:107D80003261D4EC3EF027BB81881FC532F1322D21
:107D9000120066C532F10E0E75EC10F03261D4ECB3
:107DA0003EF027BB818812008188020EB06F288BBD
:107DB000120024BFBDD0248F09EC44F0CBEC40F07E
:107DC0008DC14CF18EC14DF10A0E4E6F000E4F6BFE
:107DD00008EC0CF048C14CF149C14DF1D0C14EF155
:107DE0004F6BEBEC0BF048C14CF149C14DF1640E07
:107DF0004E6F000E4F6B08EC0CF048C107F529B12F
:107E000018C507F528EC80F0010165C532F11B0E9D
:107E100075EC10F0325DD8B097EC2BF05BEC41F0D4
:107E200025A179D0336B15EE0FF0332B5BD8040E00
:107E30003363FBD71B0E9FEC0DF0A8CF33F11D0E63
:107E40009FEC0DF0000E33B3A850E8CF6AF51E0E7C
:107E50009FEC0DF0000E33B5A850E8CF69F51F0E6A
:107E60009FEC0DF0000E33B7A850E8CF68F5200E58
:107E70009FEC0DF0000E33B9A850E8CF67F5DAECAF
:107E80000DF00FC5ADFFF1EC0DF00EC5ADFFF1EC3F
:107E90000DF00DC5ADFFF1EC0DF00CC5ADFFF1EC33
:107EA0000DF00BC5ADFFF1EC0DF00AC5ADFFF1EC27
:107EB0000DF009C5ADFFF1EC0DF008C5ADFFF1EC1B
:107EC0000DF06AC5ADFFF1EC0DF069C5ADFFF1EC49
:107ED0000DF068C5ADFFF1EC0DF067C5ADFFF1EC3D
:107EE0000DF012003351040DF350070FA96EC8ECCA
:107EF0000DF0A8CFE7FF3351040DF350060FA96E24
:107F0000C8EC0DF0E5CF0AF1D880640E0A55A856EA
:107F1000A8CFE5FF1200460EB9EC1AF0326B32C161
:107F20006AF532C169F532C168F532C167F51200F0
:107F3000249F28BF12002ABB1200420EB9EC1AF08F
:107F4000BAEC3FF000EC80F00101430EB9EC1AF0FE
:107F500023C5CEF1CE6712002BC50AF10A6729D0DE
:107F600025B1D1EC1BF02591AA6B22C5ABF1E4EC55
:107F70001BF012008DC100F58EC101F50B0E75ECE2
:107F800010F00A6F0AC112F50C0E75EC10F00A6FB2
:107F90000AC113F5100E75EC10F00A6F0AC117F53F
:107FA0001D0E75EC10F00A6F0AC11EF5FCEC4AF0CC
:107FB000120025A108EC1CF025812BC5AAF124C5CF
:107FC000ABF111EC1CF0120022972683819825BD9D
:107FD000120022BB08D0228BBDC1BFF1BEC1C0F1CF
:107FE0002F0E90EC2DF08F51A8EC2DF09051A8ECB5
:107FF0002DF0AE6BB12D02D0020EAE27B22D02D005
:10800000020EAE27B32D02D0020EAE27B42D02D041
:10801000030EAE27B52D02D0090EAE27B62D02D025
:10802000000EAE2728AB11D0010EAE27AF6BB051BA
:10803000AF27B06B28A703D0020EAE27AF8928A9BF
:1080400003D0010EAE27AF8BAE8FAE51A8EC2DF052
:1080500028AB16D0AF51A8EC2DF028A70CD0180EE5
:108060009FEC0DF0A850A8EC2DF0190E9FEC0DF030
:10807000A850A8EC2DF028A903D0D151A8EC2DF0E0
:10808000289B28972899B12F01D07AD8B22F01D0F8
:108090006CD8B32F01D05ED8B42F01D04DD8B52FF6
:1080A00001D018D8B62F01D010D8B1BFB16BB2BF74
:1080B000B26BB3BFB36BB4BFB46BB5BFB56BB6BF78
:1080C000B66B440EB9EC1AF012001A0E75EC10F0F3
:1080D000B66F120031C9B5F1B551A8EC2DF030C919
:1080E000B5F1B551A8EC2DF033C9B5F1B551A8ECF7
:1080F0002DF032C9B5F1B551A8EC2DF035C9B5F167
:10810000B551A8EC2DF034C9B5F1B551A8EC2DF05E
:1081100037C9B5F1B551A8EC2DF036C9B5F1B55157
:10812000A8EC2DF038C9B5F1B551A8EC2DF0190E19
:1081300075EC10F0B56F1200000EA8EC2DF0000EDB
:10814000A8EC2DF0000EA8EC2DF0180E75EC10F038
:10815000B46F1200000EA8EC2DF0000EA8EC2DF06C
:10816000170E75EC10F0B36F1200AA51A8EC2DF0A9
:10817000AB51A8EC2DF0160E75EC10F0B26F12009A
:108180009751A8EC2DF09851A8EC2DF0150E75EC38
:1081900010F0B16F120020A32DD08DC152F18EC10D
:1081A00053F195C154F196C155F18DC195F18EC130
:1081B00096F1D4EC0BF050C14CF151C14DF1270EAA
:1081C0004E6F4F6BEBEC0BF048C145F149C146F1E6
:1081D000070E476FBEEC0BF0630E456501D0456F8F
:1081E000050E75EC10F0455DD8A004D0218BD6ECBF
:1081F0001CF0120021AB1200219BFDEC1CF01200C0
:1082000029B112008DC14CF18EC14DF10A0E4E6F95
:108210004F6B08EC0CF048C14CF149C14DF1D0C195
:108220004EF14F6BEBEC0BF048C154F149C155F1E5
:10823000130E75EC10F0640DF3CF52F1F4CF53F13F
:10824000D4EC0BF027951FB72785279B48C154F125
:1082500049C155F1120E75EC10F0640DF3CF52F1D7
:10826000F4CF53F1D4EC0BF01FA704D0278B050EED
:10827000B06F288B48C154F149C155F1110E75EC0E
:1082800010F0640DF3CF52F1F4CF53F1D4EC0BF0B6
:108290001FB705D0278B2785040EB06F288B27B515
:1082A00006D027A307D05CEC1FF0279303D031EC56
:1082B0001FF0278312002C9D8FC14CF190C14DF10E
:1082C000640E4E6F4F6B08EC0CF01B0E9FEC0DF024
:1082D000A8A011D0010ED16301D00DD01C0E9FECCF
:1082E0000DF0030EA86407D04851A86404D0030E13
:1082F000A85C48612C8D1B0E9FEC0DF0A8A211D03C
:10830000020ED16301D00DD01D0E9FEC0DF0030EB7
:10831000A86407D04851A86404D0030EA85C486143
:108320002C8D1B0E9FEC0DF0A8A411D0030ED16371
:1083300001D00DD01E0E9FEC0DF0030EA86407D0E7
:108340004851A86404D0030EA85C48612C8D1B0E14
:108350009FEC0DF0A8A610D0040ED16301D00CD074
:108360001F0E9FEC0DF0A86407D04851A86404D0FC
:10837000030EA85C48612C8D1B0E9FEC0DF0A8A885
:1083800010D0050ED16301D00CD0200E9FEC0DF063
:10839000A86407D04851A86404D0030EA85C4861C3
:1083A0002C8D70EC1FF0120020C54CF121C54DF151
:1083B0004C6707D04D6705D0010ECC6FCD6B279170
:1083C00012004CC104F54DC105F50D0E75EC10F011
:1083D0004E6F4EC106F54B0EB9EC1AF01CEC80F056
:1083E00001014C0EB9EC1AF004C54CF105C54DF174
:1083F0004C6707D04D6705D0010ECC6FCD6B279130
:1084000012004CC1CCF14DC1CDF12781120020A743
:1084100066EF43F025BD66EF43F02ABB9ADCA3C1AB
:1084200000F5A4C101F50C0E75EC10F00A6F0AC13D
:1084300013F5470EB9EC1AF030EC80F00101B4DF0F
:10844000480EB9EC1AF0FD0EA8EC2DF0FD0EA8ECCC
:108450002DF0FE0EA8EC2DF0BFC1BDF1C0C1BEF1E4
:10846000FA0EA8EC2DF0FA0EA8EC2DF0200EA8ECD8
:108470002DF00751A8EC2DF00651A8EC2DF0085175
:10848000A8EC2DF00551A8EC2DF00451A8EC2DF02E
:108490002AAB11D0DEC132F1DFC133F170EC2DF027
:1084A00032C1DEF133C1DFF1DE51A8EC2DF0DF5136
:1084B000A8EC2DF010D091C132F192C133F170ECE3
:1084C0002DF032C191F133C192F19151A8EC2DF010
:1084D0009251A8EC2DF0A551A8EC2DF0A651A8ECD6
:1084E0002DF0A751A8EC2DF0AC51A8EC2DF0AD511A
:1084F000A8EC2DF0A351A8EC2DF0A451A8EC2DF080
:1085000020C532F121C533F13251A8EC2DF03351A1
:10851000A8EC2DF0060E9FEC0DF0A850A8EC2DF065
:10852000070E9FEC0DF0A850A8EC2DF00A0E9FEC62
:108530000DF0A850A8EC2DF00B0E9FEC0DF0A850FC
:10854000A8EC2DF00E0E9FEC0DF0A850A8EC2DF02D
:108550000F0E9FEC0DF0A850A8EC2DF0120E9FEC22
:108560000DF0A850A8EC2DF0130E9FEC0DF0A850C4
:10857000A8EC2DF0160E9FEC0DF0A850A8EC2DF0F5
:10858000170E9FEC0DF0A850A8EC2DF0180E9FECE4
:108590000DF0A850A8EC2DF0190E9FEC0DF0A8508E
:1085A000A8EC2DF0210E9FEC0DF0A850A8EC2DF0BA
:1085B000010EA8EC2DF03E0EA8EC2DF0C251A8EC57
:1085C0002DF0C351A8EC2DF0140E75EC10F02ABB61
:1085D000010EA8EC2DF0020E396F393B150E75EC2B
:1085E00010F03925A8EC2DF0020E396F393B160E2C
:1085F00075EC10F03925A8EC2DF0020E396F393BDF
:10860000170E75EC10F03925A8EC2DF0030E396F1C
:10861000393B180E75EC10F03925A8EC2DF0090E39
:10862000396F393B190E75EC10F03925A8EC2DF097
:10863000000E396F393B1A0E75EC10F03925A8EC95
:108640002DF01A0E9FEC0DF0A850A8EC2DF0000EA6
:10865000A8EC2DF0FB0EA8EC2DF0FB0EA8EC2DF0F5
:1086600025BD33D0020E9FEC0DF0A8CF39F1030EDB
:108670009FEC0DF0A8CF3AF1D890010E3927000EEB
:108680003A2339C1A8FF020E9DEC0DF03AC1A8FFB4
:10869000030E9DEC0DF01C0E89EC10F0326703D038
:1086A000336701D012D0010E3227000E3323700E33
:1086B000820FA96E32C1A8FFCCEC0DF0700E830FB3
:1086C000A96E33C1A8FFCCEC0DF08196259D2DB18C
:1086D00021EC4CF060EC80F00101196B1A6B01EF9A
:1086E0003CF020A712002ABB0ED025BD19D0209344
:1086F000B72B020E75EC10F0020FD8B0FF0EE80693
:10870000B76520831200B72B3C0EB7631200B76B1E
:108710002093E02B1E0E75EC10F0E0632083120016
:108720002093B72B050EB76520831200E3EC43F0CE
:1087300020B3BFEC43F020B3D2EC43F0219D97511E
:108740009963218D98519A63218D21BD03EC1FF00F
:10875000219F8D519563218F8E519663218F25BD69
:10876000218F21BF8BEC22F0120076EC48F0F9EC5F
:1087700043F02BEC25F09BEC49F02095120091C1C1
:1087800052F192C153F18FC154F190C155F1D4EC23
:108790000BF01FA712008FC191F190C192F12BEC49
:1087A00025F01200ACC152F1ADC153F197C154F1A3
:1087B00098C155F1D4EC0BF01FB7120097C1ACF182
:1087C00098C1ADF112002299000E75EC10F0526FB5
:1087D000536B8FC154F190C155F1D4EC0BF01FA72E
:1087E00005D020B7B76B20832289120020A72093E1
:1087F000120023B709D00C0EC36501D01200070E7A
:10880000B06F288B238712000D0EC365F8D723970E
:1088100012008FC115F190C116F115511127165193
:108820001223000E1323142315511127165112235E
:10883000000E1323142317C14EF118C14FF111C1BB
:1088400048F112C149F113C14AF114C14BF12FECA7
:108850000CF048C193F149C194F11200510EB9ECEA
:108860001AF0916B926B936B946BE6EC0FF05A0ECF
:108870009FEC0DF0000EA864AFEC0FF0116B126BC3
:10888000136B146B010E176F186B010EDE6FDF6B2D
:10889000E16BE26BDC6BDD6BA56BA66BA76BA86B6A
:1088A000E06BB76BB86BB06B289B2B9BD269E86B06
:1088B00025912C952C9DD7EC2DF0A4C103F5A3C1D7
:1088C00002F597C1ACF198C1ADF10A6B0AC14EF245
:1088D0000AC14FF202EE50F0200E0A6FEE6A0A2F24
:1088E000FDD702EE70F0200E0A6F010EEE6E0A2F19
:1088F000FCD702EE90F0EE6AEE6A200E75EC10F0F6
:10890000A8CF15F5210E75EC10F0A8CF14F52C8327
:10891000290E75EC10F0326F010E32632C93140E99
:1089200075EC10F0A96F150E75EC10F0B16F160E06
:1089300075EC10F0B26F170E75EC10F0B36F180EE7
:1089400075EC10F0B46F190E75EC10F0B56F1A0ECF
:1089500075EC10F0B66F2AAB02D0010EA96F240E91
:108960009FEC0DF029B1A8CF18F5A8CF59F1819649
:108970002397229B209D2097268325ADE9EC0DF0BF
:10898000210E9FEC0DF0A8CFD1F1D105040DF350CD
:10899000070FA96EC8EC0DF0A8CF11F5D105040D95
:1089A000F350060FA96EC8EC0DF0A8CFD0F111C599
:1089B0000AF1D880640E0A55D880A856A8CF10F5C1
:1089C000326B32C11BF532C11CF532C11DF52B953E
:1089D000120024B718D024A91200249724992A99A8
:1089E000208D209FB96B2ABB0AD0010EE8CF7FF003
:1089F000040E58EC0BF0000EE8CF7FF012008D0E45
:108A000058EC0BF012002497249920AD14D02AAB17
:108A100003D02093209D1200208F209D53EC28F03E
:108A2000CBEC26F02C992B9F010EBA6F65EC28F049
:108A30002499249712002CB7AAD08188060EB06F13
:108A4000288B2CA31200116B126B136B146B020E8C
:108A5000176F186B09EC44F0120024B715D024A945
:108A600012002DB9FFD026B91CD126BDF3D0249910
:108A7000B96BBA2B060E2BBD040EBA6302D0010EE1
:108A8000BA6F65EC28F0120024972499208F209D5E
:108A9000B96B2DB9E7D026BBB0D126B902D126BD1E
:108AA000D9D026B500D12CB9D6EF45F02BBF0BD0CD
:108AB000BA4FDAD0BA4F8AD1BA4F53D0BA4F45D055
:108AC000BA4FE9D11200BA4FBCD0BA4F17D0BA4F43
:108AD000C3D0BA4F03D0BA4FDED112002C732CA3EF
:108AE0000AD0116B126B136B146B020E176F186B9D
:108AF00009EC44F0D0D116EC26F0CDD15A0E9FEC03
:108B00000DF0A86608D0E6EC0FF0010EA86E5A0E24
:108B10009DEC0DF007D0AFEC0FF0000EA86E5A0ED2
:108B20009DEC0DF070EC1FF003EC1FF08BEC22F0CD
:108B30002BEC25F02ABBAFD128BFADD125B108EC75
:108B40001CF025A1D1EC1BF0A6D153EC28F0E9ECE8
:108B500026F0010EBA6F2B8F65EC28F0249924972C
:108B6000120029B126D1268553EC28F0D0C1A8FFE8
:108B7000180E9DEC0DF011C5A8FF190E9DEC0DF01F
:108B8000FCEC26F0010EBA6F65EC28F01200208F85
:108B9000209D249924972C8953EC28F035EC27F05C
:108BA0002B9F010EBA6F65EC28F01200BA4F73D1FB
:108BB000BA4F39D0BA4F3ED0BA4F2ED0BA4F25D087
:108BC0006AD135EC27F0980E526F3A0E536FC6C13A
:108BD00054F1C7C155F1D4EC0BF01FA705D0980E86
:108BE000C66F3A0EC76F1200E80E526F030E536F36
:108BF000C6C154F1C7C155F1D4EC0BF01FB7120038
:108C0000E80EC66F030EC76F1200E80EC65F030EB4
:108C1000C75B050EBA6FD5D7E80EC627030EC7236C
:108C2000040EBA6FCED7640EC627000EC723020EFD
:108C3000BA6FC7D7640EC65F000EC75B030EBA6F6C
:108C4000C0D7268D53EC28F030EC80F0010136ECD3
:108C500029F01200269D1FD12D8953EC28F02BEC12
:108C60002BF012002D9917D12689220E9FEC0DF0C2
:108C7000030EA8640DD00CD02B8528EC0FF047EC28
:108C80002CF023C5CEF1CE67120059EC2CF0120067
:108C900053EC28F023C5CEF1CE67120080EC27F00C
:108CA00012002699F8D0BA4F6FD0BA4F4ED0BA4FB3
:108CB00038D0BA4F17D0BA4F01D01200190E9FEC1E
:108CC0000DF0A8CF32F13207FF0E326301D0322B04
:108CD00032C1A8FF190E9DEC0DF0FCEC26F0050E3C
:108CE000BA6F1200190E9FEC0DF0A8CF32F1322BA3
:108CF000650E326302D0040E326F180E9FEC0DF039
:108D0000A8503225336F650E336301D0320732C16C
:108D1000A8FF190E9DEC0DF0FCEC26F0040EBA6FC6
:108D20001200180E9FEC0DF0A8CF32F13207030E9F
:108D3000326301D0322B32C1A8FF180E9DEC0DF02A
:108D4000FCEC26F0030EBA6F1200180E9FEC0DF02B
:108D5000A8CF32F1322B650E326302D0050E326F8E
:108D6000190E9FEC0DF0A8503225336F650E33635A
:108D700001D0320732C1A8FF180E9DEC0DF0FCECBB
:108D800026F0020EBA6F1200190E9FEC0DF0A8CF5C
:108D900011F5180E9FEC0DF0A8CFD0F111C50AF116
:108DA000D880640E0A55A856A8CF10F52887288BBE
:108DB00072D0268B53EC28F029912A89CDEC27F02C
:108DC0002981010EBA6F65EC28F0120029B10AD092
:108DD000268B53EC28F0CDEC27F0010EBA6F65EC32
:108DE00028F012002B8D268B53EC28F01EEC28F077
:108DF000010EBA6F65EC28F012002AB912D029A131
:108E000010D02C955CEC1FF0230EBA25A96EC8EC8F
:108E10000DF0A8CF18F5A8CF59F12B9D2889288BE4
:108E20003AD02C85326B32C118F5269BBAC1D1F1EC
:108E3000BA05040DF350070FA96EC8EC0DF0A8CFCA
:108E400011F5BA05040DF350060FA96EC8EC0DF02C
:108E5000A8CFD0F111C50AF1D880640E0A55A856E2
:108E6000A8CF10F52889288B16D020AF12002DB975
:108E700043D02CB93CD026A908D02BB531D023C57E
:108E8000CEF1CE6702D080EC27F0B92B0A0E75EC3C
:108E900010F0B96512002BA50DD02B9528EC0FF022
:108EA00003EC1FF02BEC25F025B108EC1CF025A1FC
:108EB000D1EC1BF02B95209F209D70EC1FF053EC04
:108EC00028F0ADEC1BF053EC25F0B96B26992D99E9
:108ED000269B269D26952B9D2C992497249912003C
:108EE00023C5CEF1CE67D1D759EC2CF0CED735ECD7
:108EF00027F065EC28F0C9D72BEC2BF0C6D729EE6C
:108F00004AF0100E396FDE660DD0392FFCD728ECF1
:108F10000FF0010E58EC0BF0020E58EC0BF070EC59
:108F200080F0010178EC0EF0E9EC0DF0A56BA66B7A
:108F3000939C939E819C819E20B509D820B14FD8E7
:108F400020A9B4EF4AF0000003000000F5D776EC4A
:108F500048F02CB13AEC48F0F1EC3CF0E4EC3CF099
:108F6000A62B0E0EA66526D070D89BEC49F01AEC05
:108F700080F00101A1C1A3F1A2C1A4F18DC1A1F1B1
:108F80008EC1A2F1A66B070E89EC10F032C152F12E
:108F900033C153F1A1C154F1A2C155F1D4EC0BF08E
:108FA0001FB701D007D0070E89EC10F032C1A1F134
:108FB00033C1A2F18DC100F58EC101F50B0E75EC28
:108FC00010F00A6F0AC112F50C0E75EC10F00A6F62
:108FD0000AC113F540EC80F00101209512002BEC42
:108FE0003DF027A104D08186000003000000819697
:108FF000A52B050EA56512D028D8060E89EC10F019
:1090000032C152F133C153F18DC154F18EC155F1CA
:10901000D4EC0BF020891FB72099A56B209124B7C1
:109020000AD024B908D0F292F0902A932A91249978
:109030002497D59E1200F292F0902A932A912499B7
:109040002497D59E209927871200EEEC18F0030094
:109050000000030000000300F1EC18F0E1EC18F050
:1090600003000000030000000300E8EC18F0C9EC66
:1090700017F01200FA0ED5EC0CF0FA0ED5EC0CF04D
:10908000FA0ED5EC0CF0FA0ED5EC0CF076EC48F0BC
:109090002CA11200F26AF16AF06AC290E9EC0DF0BC
:1090A000100E926E806A936A816A1D0E946E826AB7
:1090B000956A836A966A846AD56ACD6ACA6A9B6A27
:1090C000020ED36ED180EAC137F10F0E396F030063
:1090D0000000392FFCD781880400050EA9EC0CF0A4
:1090E000819803000000372FF6D7EDD7C28000002B
:1090F000C282C2B2FED7C4CF4DF1C3CF4CF1C60E6F
:109100004E6F030E4F6FEBEC0BF0640E4E6F4F6B18
:109110002FEC0CF048C1C2F149C1C3F1C290C2C1E9
:1091200054F1C3C155F1280E526F0A0E536FD4EC9F
:109130000BF02C911FB703D0020EEA6F2C818DC16A
:1091400054F18EC155F1990E526F3A0E536FD4EC13
:109150000BF02C911FA703D0030EEA6F2C81299BE3
:10916000299D280E9FEC0DF0A8CF54F1290E9FECFD
:109170000DF0A8CF55F1D00E526F070E536FD4ECFF
:109180000BF01FA7298B940E526F110E536FD4EC66
:109190000BF01FA7298D29AB73D029AD71D0680EB4
:1091A000A86E280E9DEC0DF0100EA86E290E9DECF9
:1091B0000DF007C1A8FF2A0E9DEC0DF006C1A8FF17
:1091C0002B0E9DEC0DF008C1A8FF2C0E9DEC0DF0B0
:1091D00097C1A8FF2D0E9DEC0DF098C1A8FF2E0E93
:1091E0009DEC0DF0A86A2F0E9DEC0DF0A86A300ED4
:1091F0009DEC0DF0A86A310E9DEC0DF0A86A320EC0
:109200009DEC0DF0A86A330E9DEC0DF0A86A340EAB
:109210009DEC0DF0A86A350E9DEC0DF097C1A8FFEE
:10922000360E9DEC0DF098C1A8FF370E9DEC0DF0A9
:1092300007C1A8FF380E9DEC0DF006C1A8FF390E3E
:109240009DEC0DF008C1A8FF3A0E9DEC0DF097C102
:10925000A8FF3B0E9DEC0DF098C1A8FF3C0E9DECC5
:109260000DF007C1A8FF3D0E9DEC0DF006C1A8FF53
:109270003E0E9DEC0DF008C1A8FF3F0E9DEC0DF0D9
:10928000280E9FEC0DF0A8CF54F1290E9FEC0DF0A5
:10929000A8CF55F1C2C152F1C3C153F1D4EC0BF0C8
:1092A0001FA71200C2C1A8FF280E9DEC0DF0C3C17C
:1092B000A8FF290E9DEC0DF007C1A8FF2A0E9DEC1A
:1092C0000DF006C1A8FF2B0E9DEC0DF008C1A8FF04
:1092D0002C0E9DEC0DF097C1A8FF2D0E9DEC0DF00E
:1092E00098C1A8FF2E0E9DEC0DF01200800ECF6EDF
:1092F000CE6A3C0E036111D03C0E04610ED0180EF4
:1093000005610BD0200E066108D00C0E076105D058
:10931000640E086102D09D801200000E036F000EE3
:10932000046F0C0E056F170E066F040E076F0A0E02
:10933000086F9D801200360E9FEC0DF0A8CF54F1FF
:10934000370E9FEC0DF0A8CF55F197C152F198C19F
:1093500053F1D4EC0BF01FA719D097C1A8FF360E1C
:109360009DEC0DF098C1A8FF370E9DEC0DF007C1E4
:10937000A8FF380E9DEC0DF006C1A8FF390E9DEC3C
:109380000DF008C1A8FF3A0E9DEC0DF03B0E9FECCE
:109390000DF0A8CF54F13C0E9FEC0DF0A8CF55F185
:1093A00097C152F198C153F1D4EC0BF01FB71200E2
:1093B00097C1A8FF3B0E9DEC0DF098C1A8FF3C0E95
:1093C0009DEC0DF007C1A8FF3D0E9DEC0DF006C110
:1093D000A8FF3E0E9DEC0DF008C1A8FF3F0E9DECCE
:1093E0000DF01200249B9D9A81869E9A620EAD6EAE
:1093F000F1EC0DF0F7EC0DF0AECF05F1180E0561B4
:10940000056BF7EC0DF0AECF04F13C0E0461046B7C
:10941000F7EC0DF0AECF03F13C0E0361036BF7ECFC
:109420000DF0AECF07F10C0E076501D0076FF7EC1A
:109430000DF0AECF06F107C132F1324F1F0E324FA1
:109440001C0E324F1F0E324F1E0E324F1F0E324F68
:109450001E0E324F1F0E324F1F0E324F1E0E324F56
:109460001F0E324F1E0E324F1F0E066502D0010E28
:10947000066FF7EC0DF0AECF08F1640E0861086BD3
:1094800081969E9A20859D8A74EF3CF02891010177
:1094900063EC4BF020B3E9EC1AF0FC6A01EE09F042
:1094A000EE6A0A0EEA62FCD7E9EC0DF076EC49F0C0
:1094B000F7EC18F0239D23ADFED78F6B906B196BE3
:1094C0001A6B208925EC48F020998DC19FF18EC13F
:1094D000A0F18DC1A1F18EC1A2F18DC1A3F18EC108
:1094E000A4F1CC2B0A6B0AC111F54F0E0A6F0AC109
:1094F00010F58DC100F58EC101F5000EE8CF4CF2DC
:1095000020EC80F0010130EC80F0010118EC80F0DB
:10951000010104EC3DF0010140EC80F00101010E7D
:10952000A96E010EAA6EC8EC0DF0A8CF39F1A92AD8
:10953000C8EC0DF0A8CF3AF1AA6A010E396304D045
:109540003E0E3A6301D010D0010EA96E010EAA6E34
:10955000010EA86ECCEC0DF0A92A3E0EA86ECCEC44
:109560000DF0AA6A11EF16F0819881961F6B206B9F
:10957000216B226B236B246B256B266B276B286B6F
:10958000296B2A6B2B6B2C6B2D6B66EC0FF0000E8E
:10959000E8CF7CF0000EE8CF7DF0000EE8CF7EF043
:1095A000000EE8CF7FF0FF0E2E6F2EC17AF0FF0E77
:1095B0002E6F2EC17BF071EC2EF0A3C19FF1A4C1E0
:1095C000A0F1AA6A5C0E9FEC0DF02F0EA86201D0EC
:1095D00006D00ED82F0EA86E5C0E9DEC0DF0270E57
:1095E0009FEC0DF02A85010EA8622A9501EF3CF050
:1095F000A3EC2AF0140E53D0289F29912A9BAA6A23
:10960000220E9FEC0DF0010EA86206D0288F000EEE
:109610000A6F0AC11FF51200020EA86206D0298146
:10962000000E0A6F0AC11FF51200030EA86206D0D1
:109630002A8B000E0A6F0AC11FF51200040EA862E1
:1096400005D0010E0A6F0AC11FF51200050EA862AF
:1096500012002981010E0A6F0AC11FF5120028ECC1
:109660000FF061EC2AF00A0E396FC80ED5EC0CF041
:109670002497249920B1E3EC43F020B139072091DD
:10968000396701D0120020B3120024B7120024B9A8
:109690001200F0D728EC0FF082EC2AF0E4D7396FF3
:1096A000C80ED5EC0CF02497249920B1E3EC43F0DC
:1096B00020B139072091396701D0120024B7120078
:1096C00024B91200F2D76C0ED36E110E926E806A1E
:1096D000030E936E816ADD0E946E826A000E966EA2
:1096E000846A000E956E836A400E9B6E1F0ED56EC7
:1096F000070ECD6ED00EF26E050EF16E080EF06EF6
:10970000210E9D6E000EA06ED06A000EC26E0E0E6F
:10971000C16E8A0EC06EC66A000EC76E280EC66E77
:10972000000EC56E080EC86EBD6ABA6A070EB46E2A
:10973000200E6F6E240EAC6E900EAB6E080EB86EDF
:10974000B06A220EAF6EAE6A9E6A1200010EEB6F17
:109750000F0EEC6F010EBA6FB86B208F218728ECCB
:109760000FF0B7EC1EF0249724992191219399ECE6
:109770001CF09AEC1DF023EC13F020A109D0F5ECBD
:109780003DF0E3EC43F02BEC3DF076EC48F020911B
:1097900021B1D5EF4BF020AFDFEF4BF020B9DFEF79
:1097A0004BF020B3B4EF4AF0E6D7BA4F1CD0BA4F13
:1097B0000AD0BA4F10D0BA4F84D0BA4F58D0040E46
:1097C000BA6F4AEF13F0020EEB27C70EEB61EB6F97
:1097D000020EBA6FC8D7030EEC27630EEC61EC6F74
:1097E000030EBA6FC0D7258D2C87ECC14CF14D6BA1
:1097F000640E4E6F4F6BEBEC0BF0E80E4827030E38
:10980000492348C1C6F149C1C7F1C6C18DF1C7C1DD
:109810008EF121912193209F2497249916EC4CF0EE
:109820002083500EB9EC1AF001EF3EF02D81530E5B
:10983000B9EC1AF062EC80F00101540EB9EC1AF0A8
:1098400012002D91530EB9EC1AF064EC80F0010176
:10985000540EB9EC1AF0470EB9EC1AF030EC80F067
:109860000101D4EC41F0480EB9EC1AF0120028ECDA
:109870000FF09CEC2CF034EC46F0010EE8CF7FF0BA
:10988000BC0E58EC0BF0000EE8CF7FF02497249923
:1098900020A109D0F5EC3DF0E3EC43F02BEC3DF0DA
:1098A00076EC48F0209124B709D024B907D020B92C
:1098B00048EF13F020B3B4EF4AF0EAD7050EBA6FC1
:1098C0004BD72EEC44F0258D2C87ECC14CF14D6B21
:1098D000640E4E6F4F6BEBEC0BF0E80E4827030E57
:1098E000492348C1C6F149C1C7F1C6C18DF1C7C1FD
:1098F0008EF116EC4CF0010EE8CF7FF00C0E58EC18
:109900000BF0000EE8CF7FF012EC3FF0BAEC3FF026
:1099100000EC80F0010123C5CEF1CE67F5D7010E32
:10992000E8CF4CF2FF0EE8CF23F599EC1CF08178DC
:1099300012EC3FF0BAEC3FF000EC80F00101430E76
:10994000B9EC1AF0EB2FF1D7000EE8CF4CF2FF0E76
:10995000E8CF23F514D0818821EC4CF0259D2C977D
:10996000FA0ED5EC0CF0FA0ED5EC0CF0FA0ED5ECA4
:109970000CF08198010EEB6F050EBA6FEDD612EC6C
:109980003FF0BAEC3FF000EC80F0010123C5CEF1CE
:10999000CE67F5D7E0D7FFFFFFFFFFFFFFFFFFFF19
:1099A000FFFFFFFFFFFFFFFFFFFFFFFFFFFFFFFFC7
:1099B000FFFFFFFFFFFFFFFFFFFFFFFFFFFFFFFFB7
:1099C000FFFFFFFFFFFFFFFFFFFFFFFFFFFFFFFFA7
:1099D000FFFFFFFFFFFFFFFFFFFFFFFFFFFFFFFF97
:1099E000FFFFFFFFFFFFFFFFFFFFFFFFFFFFFFFF87
:1099F000FFFFFFFFFFFFFFFFFFFFFFFFFFFFFFFF77
:109A0000AF9BAFAFAFAFD1AFB205B007B008AF09F2
:109A1000AF09AF09AF09B108B2079B049F9F9F9F91
:109A2000AE9FFFFFFFFFFFFFFFFFFFFFFFFFFFFFF7
:109A3000FFFFFFFFFF8F82FFAC04A1149B1A96204B
:109A400092248F288A0E8C10940B8A0C9609870F0B
:109A5000960885129707830785079706850783076A
:109A600096068708820796058A07810696058C0761
:109A7000810594058E088005940490078005930461
:109A80009107800591049208800590049407800551
:109A90008E05950780058C05960880058A06960830
:109AA000820588069707820685079708840683073C
:109AB00097088507800898078707970F8908950DED
:109AC0008B0A8C108E0E912894269922A01CAA1520
:109AD0009707FFFFD7FFB701B403B404B403B4047E
:109AE000B304B304B305B205B206B205B2068136BB
:109AF0008137813781378137FF37FFFFFFFFACFFA9
:109B0000FFFF90FF8903A8008705A5038607A3052B
:109B10008508A007840A9F08840B9F06830D9F0673
:109B2000820E9F06810882049E05830882049E049B
:109B3000840881049D05850881049C0587078104AC
:109B40009C04880781049B04890781049A048A077E
:109B5000810499048B07810498048C07810496057D
:109B60008D07810495058E07810494058F07810474
:109B70009206900782049006910782048E0792074E
:109B800083048B07930883048609940A8404951937
:109B900085049617860498148704991289049B0EED
:109BA0008C049D08B305BA05FFFF8EFFB7008A023B
:109BB000A8018804A5038607A3058608A5058407D0
:109BC000A7058406A8058206AA058205AA058105BF
:109BD00091059504800591059504800591059504EE
:109BE00080059204950480059204950480059204F2
:109BF00095048005920494058005900594068005DF
:109C00009005940680058F05920882058E059208BE
:109C100082058C06900A82068A078E0C84068707C6
:109C200081068C06850781158907870883138918A3
:109C300085118B16870F8D148A0C91128E07AC0E2E
:109C4000FF0AFFB88BFFB205B006AF08AD09AC0B39
:109C5000AA0CA90E8107A7058208A6058407A405FA
:109C60008607A3058707A10589079F058A089E0522
:109C70008C079C058D089B058F0799059008980512
:109C80009207960594079505950793059707920502
:109C9000813581378137813781378137A437B305E3
:109CA000B305B305B305B305B3058F05FFFF8CFFFF
:109CB000A20192009203901085058F1C84078E1DCF
:109CC00083088E1D8308911C8207931B82068E05D4
:109CD000950581068E05970481058E0597048105FB
:109CE0008D05980580058D05990480058D059904DD
:109CF00080058D05990480058D05990480058D05E5
:109D0000990480058D05990480058D0599048005C9
:109D10008D05990480058D05970581058D059705AD
:109D200081058E05950581068E05930682068E05B2
:109D3000910782078F058D0883089005870A830B9A
:109D40009105841C9205851A930586189405A5151E
:109D5000AA11C50CFFFF11F11BA2219A269429908C
:109D60002B8E0D8C05850E850B880588098B088840
:109D70000689088E0786058B07910784058B069355
:109D80000683058C06950582058D05960681048D52
:109D900006970580058D05980580058D059804803A
:109DA000048E0B99048E0B99058E0B98058E0B98DB
:109DB000058E05980480068E05960481058F05960C
:109DC0000581068E05940582078F07900583098E0D
:109DD000088C07840B8D0A8607851B8E05871990D2
:109DE00003891792008B13960FA707ADFFC8FFFFDB
:109DF000059605B305B305B305B305B301AF0581FA
:109E000004AC058107A905810AA605810CA405817A
:109E10000FA10581129E0581139B0583139805866A
:109E2000129605891293058C1290058F118E05925A
:109E3000118B0595108905981086059B0F84059E4A
:109E4000108115A012A310A60DA80BAB09AD06AF8B
:109E500004B2A7FFFFFF03CA0BB10FAB0790118F2E
:109E60000C8D148A0F8A1688118818861486078428
:109E7000088715850683078B068408860681068D6C
:109E8000068307890480069005820C8B0591058165
:109E90000A8D05920481088F05940480069005952B
:109EA000048006900B9505910B9505910B950592F5
:109EB0000B94069105940480079105930580088F03
:109EC000049305810A8E059106810C8C068F06820B
:109ED00006890681058E088308850781068C15840E
:109EE0000883078813860A850A82118716870F89D7
:109EF00014890C8B128C068F10900CAA06AFFFC52C
:109F0000E9FFAC09980F8D0095138A029217880417
:109F1000901986068E1B850788098F0A83068D088F
:109F20009007820590078F078205930690058005AC
:109F300094068F06800596058F05800597058F048A
:109F4000800598048F04800598048E05980B8E0573
:109F5000980B8F04800598048E04810597058E0464
:109F6000810596058D05810695068E048305940569
:109F70008D05830693068D04850690078B0586075D
:109F80008D098A058808880B8706890C8C2D8F2BF4
:109F9000932796249D1FA917D30700FFFFFFFFFFFC
:109FA000000022003500D2000001A8014302AC02EB
:109FB0005403ED035404FF049A0500EE00F00D0E67
:109FC000EE6AEA62FDD71200FFFFFFFFFFFFFFFF0F
:109FD000FFFFFFFFFFFFFFFFFFFFFFFFFFFFFFFF91
:109FE000FFFFFFFFFFFFFFFFFFFFFFFFFFFFFFFF81
:109FF000FFFFFFFFFFFFFFFFFFFFFFFFFFFFFFFF71
:10A0000000000F0016006B008300DC002D016601CC
:10A01000C10116024C02AB0202031B032A034403D4
:10A020006F0375039F9F03BA049A059A0499039BD3
:10A030009F9F9FC0BF9F9F7FBF9F03CD0E96128E95
:10A04000168A0487078B0385038C04800383048BA3
:10A0500004820282048B03840281038B02870281C3
:10A06000038A028802810488038902800387028BA5
:10A0700003810385028C03820482038C03830480A2
:10A08000038C0685048C168713890E8E0395FFCDED
:10A090000084019E029C029B029C039B029B1D9BD1
:10A0A0001D811D81FFFFFCC0850194008403910286
:10A0B0008305900382069003820790028103810248
:10A0C0008F02820481028E02830481028D02840445
:10A0D00081028D02850381028C02860381028A033C
:10A0E000870382028802880482028603890483022D
:10A0F0008A0D84028C0A85028D0887029003E00293
:10A100009AFF8501920283049303820495028203DD
:10A110009602810289028A02810289028A028102F0
:10A1200089028A02810289028A02810288028A03E4
:10A130008202870289048202850387068303810ADB
:10A1400084038404810A870C84068A0A8802FF0734
:10A15000D3849A0299049705960781039402820496
:10A160009302840391028504900287038E0288047F
:10A170008D028A038B028B048A02811C811D811D42
:10A18000941D9C029C029C02C80200FA068D028863
:10A190000F8304870F82038809820281038A028168
:10A1A0000287028C02810287028C02810187028D64
:10A1B00002810187028E02800187038D028002875F
:10A1C000028C02810287028C02810387038A02814A
:10A1D0000388048802810588058402820E8902832F
:10A1E0000C8A0894ECE591088B1188158517840575
:10A1F0008602840585038902830386038A0281031C
:10A2000086038C02810287028C02810287028D0202
:10A21000800287028C02810287028C0281028702FF
:10A220008B038102880289038302870284058305E8
:10A230008703850E8A00950CE60680FF9C029C022F
:10A240009C029702810294028105910281088F028B
:10A2500082098C0285098902880987028B08840299
:10A260008D0982029008930B950998069A04FC01C7
:10A2700005F4038A088807870A8509850483058110
:10A280000B8303810485028206850388028105878A
:10A29000028902810388028A02810388028A02817C
:10A2A0000289028A02810388028A02810488028963
:10A2B00003810686028803820383038102860B835F
:10A2C0000581048208840B84058709860597E7E5E4
:10A2D00098048B098600890C8402880E8203880307
:10A2E000880382028A02870381028C02870281022C
:10A2F0008C02870280038C02870281028C02870213
:10A3000081028C02870281028A0387028203890309
:10A3100086028303870485028504810781038708F9
:10A320008A168F12E90C9F9F03AB038A048B048962
:10A33000048B0589048A0489028C038B9F9F9FC02C
:10A34000C89F9401940A940A96089F05B99FA9FF93
:10A350009B009403940A95099806FF0302830A94CC
:10A360000A9407940497BAFF15C815891589028BBA
:10A37000019B019C019D029D049C159A148A138BDC
:10A38000028A029B019C019D029D159C1589148ADD
:10A39000118DFFA0FFFFFFFF00FF00000E001B005C
:10A3A00048007D00B400E700F0000D012A014B01D8
:10A3B0006401700185018E01A301D601E20115023D
:10A3C000460267029C02CB02EA02210352036003A9
:10A3D00071039C03CD03F8031B045C047D04B804E3
:10A3E000E5040E05410564059705AC05CD05EA05B4
:10A3F0000F0624063D0656067F06A406D50600076E
:10A40000390752076B0784079D07C607DF0718083F
:10A4100037084C086B087C089508A108D408F9088F
:10A42000200945097A099B09E409F909140A330A44
:10A43000540A710A8A0A9F0AC80AED0A120B270BEE
:10A440005A0B770B8C0BA50BBE0BE30B040C390CD2
:10A450005C0C630C860C9F0CAD0CD60C050D2A0D04
:10A46000610D6C0DAB0DB80D050E3C0E5D0E700E42
:10A47000730EBA0ECB0EE40E150F3C0F610F6B0F6F
:10A48000860F8A0FDB0FE20F03F8018A0C85028228
:10A490000A85028394FF00CD0591039101C70591C0
:10A4A00003919DDA83018F0183018F018301880667
:10A4B000870D81078F0183018F0183018F01820145
:10A4C0008607890D83058F0183018F018301A20017
:10A4D00002B40186048A0186018802810185008810
:10A4E000018300860287028201851285018502842C
:10A4F000018400870185018301880284018201892A
:10A50000058403929A9F9203880585018301850142
:10A51000860283018400890282058B0382039202F2
:10A5200082028C02830289048402820186018503EF
:10A53000830186008701820191019D0403A4069195
:10A5400004880281028208860185008602840185D2
:10A5500000860384018401860582018306860282C7
:10A560000180038803850294069201900082FF9D7A
:10A570000194069002918BFF07E70C8C03890387F7
:10A580000286028B0184028E018201910181029177
:10A5900000800093B0B093008100910181018F028F
:10A5A00082028D0284028B028602870389038D0B4F
:10A5B000E707009F019601950282009002810491B5
:10A5C000078D078F04940092028101900183018F0F
:10A5D0000095A0A6950195019501950191018B0A21
:10A5E000900B9501950195019501A40188FF8201C9
:10A5F0008F0190069404FC0001B801950195019526
:10A60000019501950195019501950195FFBC018783
:10A610000295029494FF01C1039304900490049066
:10A6200003900391039103910193A0C490028B0ABC
:10A6300085028903860187058601830186018600DC
:10A6400084018601840085028601820186028601DA
:10A6500080028701880184048B03900AA30201CA47
:10A66000019501941095108694FF00B3018B01872A
:10A670000389018604890186028801800086018899
:10A68000018200860187018301860185018402869B
:10A69000018301850687018604880187BFB488018C
:10A6A0008B0087018C01860185008501860185006C
:10A6B0008501860185008501860183018502860169
:10A6C000810280018301880182049205B70300A4FE
:10A6D0000294049202910180028F0182028E018312
:10A6E000028C0185108B1086029001940096B7A110
:10A6F0008501880083088702820285018701840022
:10A700008700860184008700860184008700860117
:10A710008400860186018400850187018500870801
:10A720008600B60608B50C8C028901820283018777
:10A7300001830186018601830186008600840187EA
:10A7400000860184018601860283018401870884D2
:10A75000058FB1B7960096008D0086018A008604A9
:10A760008700880585008B0482008D059006930381
:10A77000C30104BB04890682028702800180018331
:10A780000187028301850086018501850086018598
:10A790000185018602830185028601810180018392
:10A7A0000588068102890484B3B68605880084077B
:10A7B0008701840284018601860184008601870066
:10A7C000830186018700840086018501830187015A
:10A7D0008402820188028B0DB80901FE0186028C79
:10A7E0000285028B028594FF01FF018601820286A9
:10A7F0000685028704850094A0FC950193029303CB
:10A80000810091018101900183018F0184018D01FB
:10A8100085018D0186018B0187018B0188018901EA
:10A8200089019E01009E00840090008400900084B5
:10A8300000900084009000840090008400900084C8
:10A8400000900084009000840090008400900084B8
:10A85000009000849AA189018A0188018A018701F8
:10A860008C0186018C0185018E0184018E0183019A
:10A870009001810192018100920194039402A4014C
:10A8800001B101950194019501940188028201842E
:10A890000486028101850284018402860282068F79
:10A8A00004919DBF8D0781048A04870288028B0171
:10A8B0008701840183038700840082058601830069
:10A8C0008201820186018300840082008601820168
:10A8D0008400820086018102830082018701820A4E
:10A8E0008A00A10802A70491048F068F048D0182BB
:10A8F000038B0185048C0183048F018005910494EE
:10A9000004950294999C8610861085008501860125
:10A910008500860086018500860086018500860008
:10A9200086018500850186018301850286018301F8
:10A9300084028702800581028902820393059F02B7
:10A94000069E0A8E038A0385018902890187028B8C
:10A950000086018D0086018D0086018D0186018CA7
:10A960000186018B028802880089008A999E8610E0
:10A9700086108D0086018D0086018D0086018D0078
:10A9800086018C0186018C0186018A02880186037A
:10A990008B028E0AA20510B1108600860185018502
:10A9A0000086018501850086018501850086018577
:10A9B0000185008601850185008601850185008667
:10A9C000018501850086018DB1B486108610850051
:10A9D0008E0185008F0085008F0085008F00850027
:10A9E0008F0085008F0085008F00C400069E0B8DB0
:10A9F000028A02870288018A0187018C0086018D04
:10AA00000086018D0086008701840186008601840E
:10AA10000186008600840288068400890585B19E2F
:10AA200086108D10950195019501950195018E0176
:10AA30008610B41000B1008E0086018D0086018D55
:10AA40000086018D108610860086018D0086018D9E
:10AA50000086018DBFCC9601950186018D0086018F
:10AA60008D0086018C008701870F890D9600960066
:10AA7000AC0010991086028D02930493029102801B
:10AA8000028F0282018D0385018A02880188038A70
:10AA90000086018D0096B19C861095109501950158
:10AAA00095019501950195019501B40110991086C4
:10AAB00003870395039503950293029203920391F2
:10AAC00010921086999C8610861095039502950326
:10AAD0009503950395039502870386109C10089DA6
:10AAE0000C8C028903870187018B0187018C00860A
:10AAF000018D0086018D0186018C0186018B028803
:10AB000002880C89088CB1A08610861086008E0001
:10AB100086008E0086008E0086008E0084018E01E5
:10AB200084018E0182028F029206A702089D0C8C7E
:10AB3000028902880187028B0186018C0086028EC1
:10AB40000084048E0182018C01810182018C0181CB
:10AB50000283028801820C8401830886B1A08610DA
:10AB6000861086008E0086008E0086008E0086008D
:10AB70008D0184018B04840180018903830788038C
:10AB800086058A028A009C0003B302860588018636
:10AB90000187028201860186018301860086018584
:10ABA0000185008601850185008601850185018674
:10ABB0000185028302860284028101880585019352
:10ABC00099A0960096009600960096008610861032
:10ABD0009600960096009600AC000C990E8A02959D
:10ABE00001950196019501950195019402940E87B6
:10ABF0000C8899A0950194049405940594059205F8
:10AC00008F048F048F048F049204AB0105990A927C
:10AC100009920490058E048E05900694069406927F
:10AC20000989068AA9A686008B0186028803880303
:10AC300084038B0381038F0391058F0581038C03AC
:10AC400085028803870387038B0196029C00009985
:10AC500002960395039503950A94098D048B04903D
:10AC6000039002920094A9AC86008C0086028A00B0
:10AC700086048900800286018700810386018500A1
:10AC80008303860184008502860182008603860193
:10AC90008000880386018A0386018B0295019C014E
:10ACA00015DF0181019101810191018101910181F2
:10ACB0000191018101910181019100820091B0B265
:10ACC00095019503950395039503940495049503C5
:10ACD0009503B30100B000910182019101810191BE
:10ACE0000181019101810191018101910181019114
:10ACF0001581CEE19401920292029402960295028D
:10AD00009503D60100AB009600960096009600963B
:10AD1000009600960096009600960096E09A95019F
:10AD2000950395029502FF00A68993018C04830187
:10AD300080018B02830082018A01830184008A00E2
:10AD4000830184008A00830184008A0083018300D8
:10AD50008C00820182008C018C0BB40A12AF11842A
:10AD6000018C0186008C0188018A0188018A018892
:10AD7000018A0188018B0286038B0283088D04906F
:10AD8000B8A08F068D0884028C0286018A02880191
:10AD90008A0188018A0188018A0188018B01860164
:10ADA0008C0185028D01A60004A10890028D028409
:10ADB000018C0286018A0188018A0188018A018842
:10ADC000008B0088018C018611861284A2B4920245
:10ADD0008E0780048C03810182018B018201830133
:10ADE0008A01820183018A01820183018A01820131
:10ADF00083018B01810183018B0182058D01830415
:10AE0000B50001B601950195109003850181018F70
:10AE10000183008F0184018E0184018E00840190E2
:10AE20000295AAAB8902810480018704810B860107
:10AE300083018101830186008500820083008501F2
:10AE400085008200830085018500820083008501E2
:10AE500083018201830086018305830086008405C7
:10AE600081018601890087048B009A0112AF128448
:10AE7000018C019400950195019502950B950A8C22
:10AE8000CDB488018A0188018A0188018501820187
:10AE9000850C8201950C95019501CC0101C40196A8
:10AEA0000185018D0185018D0185018D0185018C53
:10AEB0000181108202810F810182AFDC84128F1226
:10AEC0009402940192038001900282018E02840117
:10AED0008C0286018A03890096019C0000B0018ED5
:10AEE0000184018E0184018E0184018E12841284FA
:10AEF00001950195019500969DB48A0C8B0C9500E7
:10AF0000950195018B0C8B0B9401950195018B0C90
:10AF10009C0B0CB50C8A018C019400950195019550
:10AF200002950B950A8CA1B491048E0782028C03C2
:10AF300086018B0188018A0188018A0188018A01C2
:10AF400088018B0186018C0183038D029008A00487
:10AF500011B5108501870186008C0088018B01885E
:10AF6000018A0188018A0188018B0286028B028492
:10AF7000088D0490A1A090048D0883028C038700A3
:10AF80008A0288018A0188018A0188018B01880070
:10AF90008C0086018C01860FAF110CCD0C8A018CC0
:10AFA0000194009501950195019501960095B8A72A
:10AFB00085008C0183048C0184048A018201830151
:10AFC0008A01820183018A01820183018A0183014E
:10AFD00082018B01830082018B0182018D05830038
:10AFE000B60301B5019501950E920F88018A01887B
:10AFF000018A0188018A0188018A01880194B5B516
:10B000008C0A950B950296019600950095008B0190
:10B010008A0CB40C009D0396049404950494049443
:10B020000393039103910490039000939DA89305CB
:10B03000930893058F038F04920495039405930559
:10B040008C038B09A20601B50188028A0286028C54
:10B050000382028E02800491049202910280028E89
:10B060000383028B0286008A0189ACB486018C02BC
:10B0700085018905880187048A0184048E0191076E
:10B080008F0490048F0490049303A70100A9018A00
:10B090000287018A0386018A0485018A028401806D
:10B0A000018A02820182018A02810183018A02806F
:10B0B0000184048A0185028A0187018A0188019539
:10B0C000A29C960095019301810586028107830861
:10B0D0008A06810291018101920181009201810021
:10B0E0009201C80090FF8115FF15C8909201810060
:10B0F0009201810092018100910182018506810106
:10B10000830381078A0881058F019501BA01009F99
:10B11000019501950194019501960295019501957E
:10B12000019501940195F8A6890185048103850C98
:10B130008302FF0AA19491028E0782038C03860189
:10B140008B0188018A0186008607860E84088701A4
:10B15000810088018A0187018B028601B60100A95E
:10B16000018C0186048902850E8702870682018090
:10B170000187018300860087018401860086018D96
:10B180000186008D0186008D01950195B49C860095
:10B190008E008F0882018F0184018F0084018E014F
:10B1A00084018E018401900082018F018E08860047
:10B1B000B90001B100870081038901840081038BFC
:10B1C00001820081028D018100810A8F0A8C038A2D
:10B1D00001800081038B0182008103890184008149
:10B1E0000189018600810089FFAC099008820981EC
:10B1F000088290FF02B800850486048002830784D9
:10B20000018101840184018201830184018201831F
:10B21000018301840182018401820184008301840D
:10B2200001830182018402840780018504830480F4
:10B23000018EC8BB94019502C50194019502DC0101
:10B2400002890791018E0285018B02820082008BA8
:10B2500005810082018900810183008100890181CB
:10B2600001840080008901810184008001890180BE
:10B2700000840081008A018101820081018A0081AD
:10B280000185018B0186028D02820490BC898F01A9
:10B2900081038A01810181048A0182008101800188
:10B2A0008A018200820080018A018200820080017E
:10B2B0008A018101810081018A0181088B01810756
:10B2C0009501B80101BA03940292018002900182B3
:10B2D000018F018401910394029201800290018206
:10B2E000018F0184D0B6950190018B0C8D0A8F08D7
:10B2F000910693049502BC00FFFF89CF91028E074F
:10B3000085018B0288018B00800081078900800104
:10B310008107890081008200840089008100820009
:10B32000840089008001800182038A0081008102FB
:10B3300081018A0088018B0186018D0182029002C1
:10B34000890400C900960096009600960096009623
:10B350000096CBDC930191058101900183018F015F
:10B3600083018F01830191009205D803009F00871C
:10B37000008D0187008C0187008C0187008C01877C
:10B380000B8701810B870181008C0187008C01876D
:10B39000008C0187008C0187008C0087CA9D860085
:10B3A0008D0084018C0284018C03840180008C0157
:10B3B000830180018C01820181018D0182048E0153
:10B3C0008302D30100D1018E0184018D0186018C9D
:10B3D00000820182018C00820182018C0181018244
:10B3E000058D0180018F0381FFD4019103930193A7
:10B3F00000959DF68511950B960195019501950196
:10B4000094008B02950B9502950195018500FFFF35
:10B4100080CE0195029403920491008604890386EC
:10B4200005870286068504860782048709800F86C1
:10B4300007870780068706800788058008870381BD
:10B4400007880180018106880580058907800488B6
:10B450000A8003860C8002850C8001860B800C8894
:10B46000088B8F8BFFFFFFFF90EC5BF0120000005A
:10B47000849083C083FF80948084120085C000F094
:10B48000016A00C086F084C087F0848086C083FF94
:10B490008094808487C083FF8094808412008EC053
:10B4A00083FF809480848094808412007AC083FF1C
:10B4B000809480847BC083FF80948084120000018C
:10B4C000350E836FD5DF00017D510001846F856BE0
:10B4D0000001D89084378537D1DF0001360E836FA5
:10B4E000C7DF00013F0E846F010E856FC7DF0001CB
:10B4F000370E836FBDDF00017C510001846F856BC7
:10B50000020E00017E5D07E13A0E00018427000E65
:10B510000001852310D000017E0507E1200E000107
:10B520008427000E0001852306D0180E0001842711
:10B53000000E0001852300018407000E855B0001D9
:10B54000EF0ED8808455000E855504E2EF0E000101
:10B55000846F856B7CC000F000C001F0006A005071
:10B560000001841301500001851388DF0001200EC3
:10B57000836F7EDF00017C510001846F856B7EDF6D
:10B580000001210E836F74DF00017D510001846F83
:10B59000856B0001D8908437853770DF1200200E4C
:10B5A0000001825D03E10001B60E826F000182514D
:10B5B0007E0803E2220E0001825F210E0001825DFF
:10B5C00004E300018251A30803E20001820E826FAE
:10B5D000210E0001825DF66EF76AD890F636F736D6
:10B5E0009A0EF626A30EF7220900F5CF88F00A007E
:10B5F000F5CF89F000018229DF0FF66EF76AD89047
:10B60000F636F7369A0EF626A30EF7220900F5CF86
:10B610008AF00A00F5CF8BF01200270E0001825D40
:10B6200003E100013B0E826F220E0001825D03E107
:10B6300000013C0E826F6D0E0001825D03E100018E
:10B640003D0E826F200E0001825D03E100013E0E7F
:10B65000826F2E0E0001825D04E3000182513E08DC
:10B6600003E200013E0E826F2E0E0001825DF66E37
:10B67000F76AD890F636F736000EF626A00EF722B7
:10B680000900F5CF88F00A00F5CF89F00001822982
:10B69000D20FF66EF76AD890F636F736000EF62619
:10B6A000A00EF7220900F5CF8AF00A00F5CF8BF043
:10B6B0001200200E0001825D03E100012F0E826F57
:10B6C0002E0E0001825D04E300018251390803E27D
:10B6D00000012F0E826F2E0E0001825DF66EF76A5A
:10B6E000D890F636F736A00EF6269F0EF722090000
:10B6F000F5CF88F00A00F5CF89F000018229D20F3A
:10B70000F66EF76AD890F636F736A00EF6269F0E3C
:10B71000F7220900F5CF8AF00A00F5CF8BF012006E
:10B7200000017C51006E016A013404E20050E60819
:10B73000000E015403E20001E60E7C6F00017D5112
:10B74000006E016A013404E200509B08000E0154AF
:10B7500003E200019B0E7D6FB2DE0001220E836FBB
:10B7600087DE84800001816B00018151EA6A600FED
:10B77000E96E000EEA22EFCF82F00001825106E16D
:10B7800000013A0E826F0001190E816FF86A000104
:10B79000825101E1DCD01A0E0001815D01E3D7D0B6
:10B7A000020E00017E5D02E184DF06D000017E050D
:10B7B00002E133DF01D0F3DE00018E6B88C08CF034
:10B7C00089C08DF000018A5100018C5D00018B5110
:10B7D00000018D5901E3AFD0020E00017E5D1DE135
:10B7E0008CC0F6FF8DC0F7FF010E0F0B05E0D8905F
:10B7F000F732F632E806FBE1010ED890F636F7365E
:10B80000E806FBE1000EF6269A0EF7220900F5CFB6
:10B8100084F00A00F5CF85F03CD000017E051DE1E3
:10B820008CC0F6FF8DC0F7FF010E0F0B05E0D8901E
:10B83000F732F632E806FBE1010ED890F636F7361D
:10B84000E806FBE1240EF626A00EF7220900F5CF4C
:10B8500084F00A00F5CF85F01CD08CC0F6FF8DC0B7
:10B86000F7FF010E0F0B05E0D890F732F632E8062D
:10B87000FBE1010ED890F636F736E806FBE1880EBC
:10B88000F626A40EF7220900F5CF84F00A00F5CFC2
:10B8900085F000018C51010B05E00001845100018D
:10B8A000806F05D085C000F0016A00C080F0000103
:10B8B0008051006E016A0050800B1DE07F0E000178
:10B8C000805F00017F5109E000018051000804E21F
:10B8D00000018007EBDDF8D70DD08EC083FF00019B
:10B8E0008051000807E200018007809480848094E2
:10B8F0008084F5D71BD00001802B00017F510EE022
:10B900008EC083FF00018051000807E2000180071C
:10B910008094808480948084F5D708D00001805181
:10B92000000804E200018007C1DDF8D700018C2B7C
:10B93000000E8D2347D70001812B00018151EA6A57
:10B94000600FE96E000EEA22EFCF82F020D70001EF
:10B95000836B8EDD1200FFFFFFFFFFFFFFFFFFFF86
:10B96000FFFFFFFFFFFFFFFFFFFFFFFFFFFFFFFFE7
:10B97000FFFFFFFFFFFFFFFFFFFFFFFFFFFFFFFFD7
:10B98000FFFFFFFFFFFFFFFFFFFFFFFFFFFFFFFFC7
:10B99000FFFFFFFFFFFFFFFFFFFFFFFFFFFFFFFFB7
:10C000000901306B316B326B336B3451040B04E03C
:10C01000080E346F356B03D0040E346F356B366BFE
:10C02000376B386934C4B5F935C4B6F936C4B7F9D5
:10C0300037C4B8F938C4B9F939C4BAF93AC4BBF944
:10C040003BC4BCF91FC583F91EC584F90CC485F92E
:10C050000DC486F90EC487F90FC488F997C289F90F
:10C0600098C28AF999C28BF99AC28CF99BC28DF950
:10C070009CC28EF99DC28FF99EC290F9F3C591F9C9
:10C08000F4C592F9F5C593F9F6C594F9F7C595F994
:10C09000F8C596F9F9C597F9FAC598F9FBC599F964
:10C0A000FCC59AF9FDC59BF9FEC59CF95FC99DF9D0
:10C0B00060C99EF961C99FF962C9A0F963C9A1F974
:10C0C00064C9A2F965C9A3F966C9A4F96FC9A5F93C
:10C0D00070C9A6F971C9A7F972C9A8F977C9A9F9F0
:10C0E00078C9AAF979C9ABF97AC9ACF97BC9ADF9B4
:10C0F0007CC9AEF97DC9AFF97EC9B0F97FC9B1F984
:10C1000080C9B2F981C9B3F982C9B4F905011F51D7
:10C1100002E0090130812C6A2D6A2E6A2F6AF3C56C
:10C1200027F0F4C528F0F5C529F0F6C52AF0C2ECD1
:10C130006EF0010A02E009013083100E0901BE6FA2
:10C14000BF6B200EBFAF02D0D89003D0BE5D000EF3
:10C15000BF592DE2BEC9E9FFBFC9EAFFD890E93651
:10C16000EA36D890E936EA36800EE926040EEA224D
:10C17000EECF00F0EECF01F0EECF02F0EFCF03F004
:10C180002C6A2D6A2E6A2F6A00C027F001C028F0A1
:10C1900002C029F003C02AF0C2EC6EF0010A02E0EE
:10C1A000090130850901BE2B000EBF23CAD72C6AB6
:10C1B0002D6A2E6A2F6AF7C527F0F8C528F0F9C551
:10C1C00029F0FAC52AF0C2EC6EF0010A02E009017A
:10C1D0003087A40E2C6E700E2D6E7D0E2E6E3F0ECF
:10C1E0002F6E77C927F078C928F079C929F07AC964
:10C1F0002AF0D2EC6EF0010A02E109013089660EE4
:10C200002C6E2D6EA60E2E6E3F0E2F6E77C927F068
:10C2100078C928F079C929F07AC92AF0C9EC6EF0FA
:10C22000010A02E10901308B5C0E2C6E8F0E2D6E1F
:10C23000420E2E6E3E0E2F6E97C227F098C228F047
:10C2400099C229F09AC22AF0D2EC6EF0010A02E1FA
:10C250000901308DAE0E2C6E470E2D6E810E2E6EA6
:10C260003F0E2F6E97C227F098C228F099C229F08E
:10C270009AC22AF0C9EC6EF0010A02E10901308F7E
:10C280009A0E2C6E990E2D6E190E2E6E3F0E2F6E7D
:10C290009BC227F09CC228F09DC229F09EC22AF0C2
:10C2A000D2EC6EF0010A02E109013181AE0E2C6E72
:10C2B000470E2D6E810E2E6E3F0E2F6E9BC227F005
:10C2C0009CC228F09DC229F09EC22AF0C9EC6EF0F3
:10C2D000010A02E10901318338C42CF039C42DF080
:10C2E0003AC42EF03BC42FF034C427F035C428F0F4
:10C2F00036C429F037C42AF0F8EC6CF027C000F0FF
:10C3000028C001F029C002F02AC003F0330E2C6EC1
:10C310002D6E730E2E6E3F0E2F6E00C027F001C0E3
:10C3200028F002C029F003C02AF0C9EC6EF0010A1F
:10C3300002E10901318538C42CF039C42DF03AC42A
:10C340002EF03BC42FF034C427F035C428F036C497
:10C3500029F037C42AF0F8EC6CF027C000F028C0B0
:10C3600001F029C002F02AC003F0CD0E2C6ECC0ED5
:10C370002D6E4C0E2E6E3D0E2F6E00C027F001C0AC
:10C3800028F002C029F003C02AF0D2EC6EF0010AB6
:10C3900002E1090131872C6A2D6A800E2E6E3E0E55
:10C3A0002F6E7FC927F080C928F081C929F082C982
:10C3B0002AF0C9EC6EF0010A02E109013189050198
:10C3C0001E51080802E20901318B2C6A2D6A2E6A7F
:10C3D0002F6AA5C927F0A6C928F0A7C929F0A8C9BE
:10C3E0002AF0C2EC6EF0010A2FE063C92CF064C998
:10C3F0002DF065C92EF066C92FF05FC927F060C91E
:10C4000028F061C929F062C92AF0F8EC6CF027C065
:10C4100000F028C001F029C002F02AC003F0330E5A
:10C420002C6E2D6E730E2E6E3F0E2F6E00C027F0F9
:10C4300001C028F002C029F003C02AF0C9EC6EF058
:10C44000010A02E10901318D2C6A2D6A2E6A2F6AD8
:10C45000A5C927F0A6C928F0A7C929F0A8C92AF0BC
:10C46000C2EC6EF0010A30E063C92CF064C92DF013
:10C4700065C92EF066C92FF05FC927F060C928F0A2
:10C4800061C929F062C92AF0F8EC6CF027C000F00D
:10C4900028C001F029C002F02AC003F0CD0E2C6E96
:10C4A000CC0E2D6E4C0E2E6E3D0E2F6E00C027F062
:10C4B00001C028F002C029F003C02AF0D2EC6EF0CF
:10C4C000010A02E10901318F2C6A2D6A400E2E6E9D
:10C4D0002F6E08C427F009C428F00AC429F00BC441
:10C4E0002AF0C9EC6EF0010A02E10901328108C4A8
:10C4F0002CF009C42DF00AC42EF00BC42FF00CC48C
:10C5000027F00DC428F00EC429F00FC42AF0F7EC70
:10C510006CF027C000F028C001F029C002F02AC04A
:10C5200003F0CD0E2C6ECC0E2D6E4C0E2E6E3E0EEC
:10C530002F6E00C027F001C028F002C029F003C010
:10C540002AF0C9EC6EF0010A02E1090132832C6A7B
:10C550002D6A400E2E6E3F0E2F6E0CC427F00DC4B8
:10C5600028F00EC429F00FC42AF0D2EC6EF0010AB4
:10C5700002E1090132857B0E2C6E140E2D6E8E0E9B
:10C580002E6E3F0E2F6E0CC427F00DC428F00EC483
:10C5900029F00FC42AF0C9EC6EF0010A02E109018A
:10C5A0003287330E2C6E2D6E2E6E3F0E2F6E7BC992
:10C5B00027F07CC928F07DC929F07EC92AF0D2EC89
:10C5C0006EF0010A02E109013289AE0E2C6E470EAF
:10C5D0002D6E810E2E6E3F0E2F6E7BC927F07CC90B
:10C5E00028F07DC929F07EC92AF0C9EC6EF0010A55
:10C5F00002E10901328B9BC22CF09CC22DF09DC23E
:10C600002EF09EC22FF097C227F098C228F099C250
:10C6100029F09AC22AF0C9EC6EF0010A02E1090180
:10C62000328D12000901349536951200FF0E090172
:10C63000385D20E10501B80ED88000550B0E01557C
:10C6400019E222C538F938C900F0016A00BE016854
:10C65000FF0E001801E101500DE138C900F0016A38
:10C6600000BE0168FE0E001801E1015002E0000E5C
:10C6700001D0010E1200D9CFE6FFE1CFD9FF0901A9
:10C68000C06BC16B34C42CF035C42DF036C42EF011
:10C6900037C42FF0B5C927F0B6C928F0B7C929F0BB
:10C6A000B8C92AF0C2EC6EF0010A14E138C42CF0CB
:10C6B00039C42DF03AC42EF03BC42FF0B9C927F08D
:10C6C000BAC928F0BBC929F0BCC92AF0C2EC6EF087
:10C6D000010A02E00901C081F3C52CF0F4C52DF078
:10C6E000F5C52EF0F6C52FF091C927F092C928F0B4
:10C6F00093C929F094C92AF0C2EC6EF0010A02E055
:10C700000901C08377C92CF078C92DF079C92EF0C2
:10C710007AC92FF0A9C927F0AAC928F0ABC929F016
:10C72000ACC92AF0C2EC6EF0010A14E17BC92CF00E
:10C730007CC92DF07DC92EF07EC92FF0ADC927F040
:10C74000AEC928F0AFC929F0B0C92AF0C2EC6EF02A
:10C75000010A02E00901C08905011F510901835D39
:10C7600001E0C08B0CC42CF00DC42DF00EC42EF0D3
:10C770000FC42FF085C927F086C928F087C929F092
:10C7800088C92AF0C2EC6EF0010A02E00901C08DEE
:10C790003AD0100E0901BE6FBF6B200EBFAF02D0A2
:10C7A000D89003D0BE5D000EBF592DE2BEC9E9FF8F
:10C7B000BFC9EAFFD890E936EA36D890E936EA36BA
:10C7C000800EE926040EEA22EECF00F0EECF01F053
:10C7D000EECF02F0EFCF03F02C6A2D6A2E6A2F6A9B
:10C7E00000C027F001C028F002C029F003C02AF0E1
:10C7F000C2EC6EF0010A02E00901C08F0901BE2BF4
:10C80000000EBF23CAD7FBC52CF0FCC52DF0FDC51B
:10C810002EF0FEC52FF099C927F09AC928F09BC9C0
:10C8200029F09CC92AF0C2EC6EF0010A02E009016D
:10C83000C1816FC92CF070C92DF071C92EF072C979
:10C840002FF0A5C927F0A6C928F0A7C929F0A8C9C3
:10C850002AF0C2EC6EF0010A28E15FC92CF060C931
:10C860002DF061C92EF062C92FF09DC927F09EC935
:10C8700028F09FC929F0A0C92AF0C2EC6EF0010A85
:10C8800014E163C92CF064C92DF065C92EF066C9A6
:10C890002FF0A1C927F0A2C928F0A3C929F0A4C983
:10C8A0002AF0C2EC6EF0010A02E00901C1837FC9DF
:10C8B0002CF080C92DF081C92EF082C92FF0B1C9AA
:10C8C00027F0B2C928F0B3C929F0B4C92AF0C2ECE4
:10C8D0006EF0010A02E00901C18505011E5109013E
:10C8E000845D01E0C18797C22CF098C22DF099C2F7
:10C8F0002EF09AC22FF089C927F08AC928F08BC977
:10C9000029F08CC92AF0C2EC6EF0010A14E19BC236
:10C910002CF09CC22DF09DC22EF09EC22FF08DC92E
:10C9200027F08EC928F08FC929F090C92AF0C2ECEF
:10C930006EF0010A02E00901C1892C6A2D6A500ECD
:10C940002E6E410E2F6E08C427F009C428F00AC4C9
:10C9500029F00BC42AF0C9EC6EF0010A02E10901CA
:10C96000C18D08C42CF009C42DF00AC42EF00BC4EC
:10C970002FF00CC427F00DC428F00EC429F00FC40A
:10C980002AF0F7EC6CF027C000F028C001F029C0B5
:10C9900002F02AC003F0CD0E2C6ECC0E2D6E4C0E84
:10C9A0002E6E3E0E2F6E00C027F001C028F002C090
:10C9B00029F003C02AF0C9EC6EF0010A02E1090176
:10C9C000C18FFE0EDB5006E00901C0513613C15184
:10C9D000371305D00901C0513413C1513513E55245
:10C9E000E7CFD9FF1200E66A46DEE5521200010EDB
:10C9F000E66E41DEE55212000201706B05011F0573
:10CA000001E0D7D30201925101E04CD1F00E2C6E1F
:10CA1000850E2D6E990E2E6E3E0E2F6EBBC227F028
:10CA2000BCC228F0BDC229F0BEC22AF08EEC6DF067
:10CA300027C014F428C015F429C016F42AC017F42E
:10CA4000A40E2C6E700E2D6E7D0E2E6E3F0E2F6E70
:10CA500014C427F015C428F016C429F017C42AF00E
:10CA6000F8EC6CF093EC6EF028C004F429C005F4E7
:10CA700004011F0ED8800455000E055503E21F0E59
:10CA8000046F056B000E045D000E055902E2046B95
:10CA9000056B04C4C6F2030E0201C603F3CFC5F250
:10CAA000C5C229F0D1EC6CF027C000F028C001F01D
:10CAB00029C002F02AC003F0960E2C6EB20E2D6E25
:10CAC000CC0E2E6E3D0E2F6E00C027F001C028F058
:10CAD00002C029F003C02AF0E1EC6DF027C014F485
:10CAE00028C015F429C016F42AC017F47FC92CF009
:10CAF00080C92DF081C92EF082C92FF014C427F00F
:10CB000015C428F016C429F017C42AF0F8EC6CF00C
:10CB100027C000F028C001F029C002F02AC003F0AD
:10CB20000CC42CF00DC42DF00EC42EF00FC42FF049
:10CB300000C027F001C028F002C029F003C02AF08D
:10CB4000F8EC6CF027C0E8F228C0E9F229C0EAF25C
:10CB50002AC0EBF20201C65105E1A76BA86BA96BD5
:10CB6000AA6B26D0C6C229F0D1EC6CF027C000F029
:10CB700028C001F029C002F02AC003F000C02CF048
:10CB800001C02DF002C02EF003C02FF09FC227F08D
:10CB9000A0C228F0A1C229F0A2C22AF08EEC6DF04A
:10CBA00027C0A7F228C0A8F229C0A9F22AC0AAF279
:10CBB0002C6A2D6A2E6A2F6AA7C227F0A8C228F015
:10CBC000A9C229F0AAC22AF0D2EC6EF0010A05E14E
:10CBD0000201A76BA86BA96BAA6B9FC22CF0A0C225
:10CBE0002DF0A1C22EF0A2C22FF0A7C227F0A8C23A
:10CBF00028F0A9C229F0AAC22AF0C9EC6EF0010AF5
:10CC000008E19FC2A7F2A0C2A8F2A1C2A9F2A2C2E3
:10CC1000AAF22C6A400E2D6E1C0E2E6E460E2F6E42
:10CC2000A7C227F0A8C228F0A9C229F0AAC22AF0F8
:10CC3000E1EC6DF093EC6EF028C042F229C043F2B3
:10CC40002C6A2D6A7A0E2E6E440E2F6EE8C227F0E3
:10CC5000E9C228F0EAC229F0EBC22AF0E1EC6DF05B
:10CC600093EC6EF028C048F229C049F22C6A2D6A74
:10CC70007A0E2E6E440E2F6EAFC227F0B0C228F08F
:10CC8000B1C229F0B2C22AF0E1EC6DF093EC6EF083
:10CC900028C04AF229C04BF2C6C24EF20201010E70
:10CCA000926FC76BC75153E1C6C2C7F2C7C229F022
:10CCB000D1EC6CF027C004F028C005F029C006F0C4
:10CCC0002AC007F0A7C22CF0A8C22DF0A9C22EF0EE
:10CCD000AAC22FF004C027F005C028F006C029F032
:10CCE00007C02AF0E1EC6DF027C000F028C001F089
:10CCF00029C002F02AC003F000C02CF001C02DF0C2
:10CD000002C02EF003C02FF09BC227F09CC228F077
:10CD10009DC229F09EC22AF0F7EC6CF027C0A3F266
:10CD200028C0A4F229C0A5F22AC0A6F20201C75168
:10CD3000EA6A700FE96E020EEA22EF500401046FF6
:10CD4000056B04C408F30301210E096F04D0010E22
:10CD50000401046F056B0401010E041901E1055182
:10CD600001E091D10201C7050401046F056B010EBA
:10CD7000041901E1055101E07FD0C3C228F0C4C20B
:10CD800029F004C42DF005C42EF04EEC6EF026C040
:10CD900004F027C005F004C028F005C029F0E2EC3B
:10CDA0006CF027C000F028C001F029C002F02AC0B2
:10CDB00003F0960E2C6EB20E2D6ECC0E2E6E3D0E26
:10CDC0002F6E00C027F001C028F002C029F003C078
:10CDD0002AF0E1EC6DF027C014F428C015F429C046
:10CDE00016F42AC017F42C6A2D6A400E2E6E2F6E90
:10CDF000A7C227F0A8C228F0A9C229F0AAC22AF027
:10CE00008EEC6DF027C000F028C001F029C002F0C0
:10CE10002AC003F0C3C208F0C4C209F0060ED880CD
:10CE20000856000E095608C028F009C029F0E2ECA7
:10CE30006CF027C004F028C005F029C006F02AC015
:10CE400007F004C02CF005C02DF006C02EF007C07E
:10CE50002FF000C027F001C028F002C029F003C065
:10CE60002AF0E1EC6DF027C0ABF228C0ACF229C08B
:10CE7000ADF22AC0AEF25FD0045105111FE1146B70
:10CE8000156B166B176BA3C22CF0A4C22DF0A5C2B4
:10CE90002EF0A6C22FF09BC227F09CC228F09DC2A4
:10CEA00029F09EC22AF0F7EC6CF027C0ABF228C044
:10CEB000ACF229C0ADF22AC0AEF23DD0030E286E0E
:10CEC000296A04C42DF005C42EF04EEC6EF026C085
:10CED00004F027C005F004C028F005C029F0E2ECFA
:10CEE0006CF027C000F028C001F029C002F02AC071
:10CEF00003F0960E2C6EB20E2D6ECC0E2E6E3D0EE5
:10CF00002F6E00C027F001C028F002C029F003C036
:10CF10002AF0E1EC6DF027C014F428C015F429C004
:10CF200016F42AC017F4A7C2ABF2A8C2ACF2A9C289
:10CF3000ADF2AAC2AEF20CC42CF00DC42DF00EC49A
:10CF40002EF00FC42FF014C427F015C428F016C417
:10CF500029F017C42AF0F8EC6CF027C014F428C0AC
:10CF600015F429C016F42AC017F4ABC22CF0ACC2D9
:10CF70002DF0ADC22EF0AEC22FF0A3C227F0A4C296
:10CF800028F0A5C229F0A6C22AF0F8EC6CF027C060
:10CF900004F028C005F029C006F02AC007F0B3C28B
:10CFA0002CF0B4C22DF0B5C22EF0B6C22FF004C0E2
:10CFB00027F005C028F006C029F007C02AF0E1ECF0
:10CFC0006DF027C000F028C001F029C002F02AC08F
:10CFD00003F0AFC22CF0B0C22DF0B1C22EF0B2C23D
:10CFE0002FF000C027F001C028F002C029F003C0D4
:10CFF0002AF0F8EC6CF027C010F428C011F429C016
:10D0000012F42AC013F414C42CF015C42DF016C465
:10D010002EF017C42FF010C427F011C428F012C44A
:10D0200029F013C42AF0C9EC6EF0010A04E10401EE
:10D03000046B056B27D004C4C7F2ABC22CF0ACC2A2
:10D040002DF0ADC22EF0AEC22FF0A3C227F0A4C2C5
:10D0500028F0A5C229F0A6C22AF0F8EC6CF027C08F
:10D06000A3F228C0A4F229C0A5F22AC0A6F20201A8
:10D07000C751EA6A700FE96E020EEA22EF5004010E
:10D08000046F056B68D60201C751000801E386D022
:10D09000F00E006E850E016E990E026E3E0E036E4E
:10D0A000C7C229F0D1EC6CF027C004F028C005F00D
:10D0B00029C006F02AC007F004C02CF005C02DF0EE
:10D0C00006C02EF007C02FF000C027F001C028F0E6
:10D0D00002C029F003C02AF0E1EC6DF027C014F47F
:10D0E00028C015F429C016F42AC017F47FC92CF003
:10D0F00080C92DF081C92EF082C92FF014C427F009
:10D1000015C428F016C429F017C42AF0F8EC6CF006
:10D1100027C000F028C001F029C002F02AC003F0A7
:10D120000CC42CF00DC42DF00EC42EF00FC42FF043
:10D1300000C027F001C028F002C029F003C02AF087
:10D14000F8EC6CF027C020F428C021F429C022F4A8
:10D150002AC023F40201C70505E1C3C2BFF2C4C25D
:10D16000C0F205D0030EC703F350BF6FC06B210E92
:10D170000301095D12E1C7C209F30201C751EA6A5E
:10D18000700FE96E020EEA22EFCF0AF303010C29B9
:10D190000C6F640E0C5D01E10C6B0AD00CC420F422
:10D1A0000DC421F40EC422F40FC423F4BF6BC06B72
:10D1B000E8D00CC42CF00DC42DF00EC42EF00FC41A
:10D1C0002FF074C427F075C428F076C429F077C412
:10D1D0002AF0F7EC6CF027C010F428C011F429C035
:10D1E00012F42AC013F42C6A2D6A2E6A2F6A10C416
:10D1F00027F011C428F012C429F013C42AF0D2EC8D
:10D200006EF0010A01E1B2D0F00E2C6E850E2D6E8B
:10D21000990E2E6E3E0E2F6E10C427F011C428F00A
:10D2200012C429F013C42AF08EEC6DF027C010F45C
:10D2300028C011F429C012F42AC013F4A40E2C6ED5
:10D24000700E2D6E7D0E2E6E3F0E2F6E10C427F0C9
:10D2500011C428F012C429F013C42AF0F8EC6CF0C1
:10D2600093EC6EF028C0BFF229C0C0F2030E286E06
:10D27000296ABFC22DF0C0C22EF04EEC6EF026C05F
:10D28000BFF227C0C0F20201BF51C01109E10CC4B6
:10D2900020F40DC421F40EC422F40FC423F465D08D
:10D2A000C351BF5DC451C05904E2C3C2BFF2C4C27E
:10D2B000C0F2BFC228F0C0C229F0E2EC6CF027C077
:10D2C00000F028C001F029C002F02AC003F0960E39
:10D2D0002C6EB20E2D6ECC0E2E6E3D0E2F6E00C03B
:10D2E00027F001C028F002C029F003C02AF0E1ECC9
:10D2F0006DF027C010F428C011F429C012F42AC020
:10D3000013F47FC92CF080C92DF081C92EF082C999
:10D310002FF010C427F011C428F012C429F013C450
:10D320002AF0F8EC6CF027C000F028C001F029C00A
:10D3300002F02AC003F00CC42CF00DC42DF00EC472
:10D340002EF00FC42FF000C027F001C028F002C05B
:10D3500029F003C02AF0F8EC6CF027C020F428C0B4
:10D3600021F429C022F42AC023F40BD00CC420F4E9
:10D370000DC421F40EC422F40FC423F40201BF6BC8
:10D38000C06B120005011F051DE1200E0401046F92
:10D39000056B006B0451005D000E055513E2005152
:10D3A000EA6AC80FE96E020EEA22EF50E66E0051FB
:10D3B000EA6A500FE96E020EEA22E552E750EF6E7C
:10D3C000002BE8D7120005011F050EE10401006BD8
:10D3D000200E005D09E20051EA6AC80FE96E020EF4
:10D3E000EA22EF6A002BF4D7120005011F0523E1A2
:10D3F0000201C751EA6AC80FE96E020EEA22EF5035
:10D40000006E016AD890015004E6FF0E005C000E29
:10D41000015811E2C751EA6AC80FE96E020EEA220A
:10D42000EF28E66EC751EA6AC80FE96E020EEA22DB
:10D43000E552E750EF6E120005011F0501E145D0EE
:10D440002C6A2D6A2E6A2F6A2CC427F02DC428F06E
:10D450002EC429F02FC42AF0D2EC6EF0010A1BE191
:10D460007BC92CF07CC92DF07DC92EF07EC92FF030
:10D470002CC427F02DC428F02EC429F02FC42AF084
:10D48000E1EC6DF027C02CF428C02DF429C02EF457
:10D490002AC02FF41AD077C92CF078C92DF079C999
:10D4A0002EF07AC92FF02CC427F02DC428F02EC4FA
:10D4B00029F02FC42AF0E1EC6DF027C02CF428C02D
:10D4C0002DF429C02EF42AC02FF412000001130EEF
:10D4D0008A6F1C0E8B6F976BF50E986F996B9A6B1A
:10D4E000300E9B6F390E9C6F86EF6AF000010C0EB8
:10D4F0008A6F100E8B6F976BE10E986F996B9A6B1A
:10D500002E0E9B6F3E0E9C6F86EF6AF00001906BB3
:10D5100090C0DEFF84820001706B0001875103E13F
:10D520000001010E876F0001865103E10001010E29
:10D53000866F00018B510001D880885502E28BC0B4
:10D5400088F00001875100018825410806E2410E5C
:10D550000001D88087550001886F86C092F00001D5
:10D56000916B00019151912BEA6A600FE96E000EF8
:10D57000EA22EFCF93F05BD80001906B0001010E1F
:10D58000946F0001935152E00001940501E1F1D83C
:10D59000FFD8010E000194190001946F0001940559
:10D5A00008E1CED8400E0001925D02E20001922B0C
:10D5B000A5D90001902B040E0001905D02E2000E3F
:10D5C00001D0010E036E3C0E0001935D02E0000EDF
:10D5D00001D0010E026E3A0E0001935D02E0000ED2
:10D5E00001D0010E016E2E0E0001935D02E0000ECF
:10D5F00001D0010E011002100314006E00018A51C7
:10D600000001905D02E2000E01D0010E00100DE05D
:10D6100000019151912BEA6A600FE96E000EEA2237
:10D62000EFCF93F004D80001906BABD7120000014C
:10D630009C51D880935502E3000E01D0010E006E7C
:10D640009B51935D02E3000E01D0010E001006E035
:10D650008C6B8D6B8E6B8F6B956B71D09B51935DCB
:10D660008C6F8D6B8E6B8F6B8B29FE0BE842006E7F
:10D67000016A026A036A8CC026F08DC027F08EC052
:10D6800028F08FC029F000C02BF001C02CF002C0A0
:10D690002DF003C02EF048EC70F022C08CF023C0B7
:10D6A0008DF024C08EF025C08FF08AC000F0016A92
:10D6B000026A036A8CC026F08DC027F08EC028F065
:10D6C0008FC029F000C02BF001C02CF002C02DF05B
:10D6D00003C02EF048EC70F022C08CF023C08DF017
:10D6E00024C08EF025C08FF0000197518C279851EF
:10D6F0008D2399518E239A518F233C0E935D02E026
:10D70000000E01D0010E016E3A0E935D02E0000E94
:10D7100001D0010E006E2E0E935D02E0000E01D0CE
:10D72000010E001001100BE08B51E824006E000187
:10D73000005000018C27000E8D238E238F231200B2
:10D740000001750E966FF0D800018705966FECD832
:10D7500000013F0E966FE8D80001150E966FE4D8D1
:10D7600000019205966FE0D800019205966F94EF44
:10D770006CF00001956B8851955D09E29551EA6A5C
:10D78000000FE96E080EEA22EF6A952BF4D712001B
:10D7900000018C518D118E118F1101E1AED000016D
:10D7A0008C510001956F95C0F6FF8DC000F08EC0C2
:10D7B00001F08FC002F00001036A00500001956F74
:10D7C00095C0F7FF8EC000F08FC001F00001026A23
:10D7D000036A00500001956F95C0F8FF0001956B3A
:10D7E000000188510001955D01E37AD00900F5CF71
:10D7F00096F0000189511CE000018939F00B006EA0
:10D80000F00E00019615005C07E200018939F00B6B
:10D810000001965D0001966F0F0E00019615000144
:10D82000895D06E2000189510001965D0001966F55
:10D83000000194051EE1F00E00019615E66E000150
:10D840009551EA6A000FE96E080EEA22E552E750A8
:10D85000EF6E00019639F00BF00BE66E0001952992
:10D86000EA6A000FE96E080EEA22E552E750EF6E11
:10D8700033D0000196390F0B0F0B006E000195514C
:10D88000EA6A000FE96E080EEA22EF50F00B001072
:10D89000E66E00019551EA6A000FE96E080EEA2271
:10D8A000E552E750EF6E0F0E00019615006E000175
:10D8B0009529EA6A000FE96E080EEA22EF50F00B94
:10D8C0000010E66E00019529EA6A000FE96E080E65
:10D8D000EA22E552E750EF6E020E0001952780D74D
:10D8E00000018B29FE0BE842006E00010050000190
:10D8F0008C27000E8D238E238F231200848200013B
:10D90000956B000188510001955D0DE20001955174
:10D91000EA6A000FE96E080EEA22EFCF96F007D808
:10D920000001952BEED71200849201D8120001015C
:10D9300084900001839096BF8382839096AF8392F8
:10D94000838096BD8382839096AD8392838096BBBD
:10D950008382839096AB8392838096B983828390EF
:10D9600096A98392838096B78382839096A78392A9
:10D97000838096B58382839096A58392838096B3A5
:10D980008382839096A38392838096B183828390CF
:10D9900096A1839283808480010100010001966B2F
:10D9A0001200219E05D0219E29AE02D0296C218E25
:10D9B00029C023F0226A336A326A860E246E256AF1
:10D9C0004CEF6FF0219E08D0219E29AE05D0286C27
:10D9D000291EE86A2922218E29C023F028C022F0BE
:10D9E000336A326A8E0E246E256A4CEF6FF02F7EFA
:10D9F000216A88EC6FF0A0EC6FF021B630EF6FF089
:10DA000021A20AD021AA03D021BE30EF6FF021A4B9
:10DA10003CEF6FF039EF6FF021AA05D021AC3CEF5D
:10DA20006FF039EF6FF021A00AD021A808D021BEF5
:10DA300004D021A402D045EF6FF049EF6FF0326AB5
:10DA4000256A2F502A5C316E10E327C033F028C0BE
:10DA500022F029C023F02AC030F02CC027F02DC0BE
:10DA600028F02EC029F0213A09D02CC033F02DC067
:10DA700022F02EC023F02FC030F0316C219E21BC4B
:10DA8000218E30C024F021B078EF6FF01A0E316093
:10DA900078EF6FF0246A2A6A21A408D0276C281E28
:10DAA000291E2A1EE86A282229222A2221AC08D00F
:10DAB000336C221E231E241EE86A222223222422E3
:10DAC000266A315207E02A34293228322732263298
:10DAD000312EF9D7275033262850222229502322CD
:10DAE0002A50242226C032F0219E24AE0BD0326C64
:10DAF000331E221E231E241EE86A332222222322E2
:10DB00002422218E24A006D0D88023322232333220
:10DB10003232302A30C024F04CEF6FF0216A88ECAA
:10DB20006FF0A0EC6FF021B630EF6FF021A205D0BE
:10DB300021BA30EF6FF037EF6FF021BA43EF6FF09B
:10DB400021A005D021B830EF6FF043EF6FF021B87E
:10DB500037EF6FF0256A7F0E2A24246EE86A2522AB
:10DB60002F50245EE86A255A1A0E306E2A6A326AED
:10DB7000336A226A236A2C50275E2D50285A2E5071
:10DB8000295A000E2A5A09E72C5027262D50282200
:10DB90002E502922000E2A2201D0328AD890273610
:10DBA000283629362A36D89032363336223623366E
:10DBB000302EE1D7295028102710D8A4328A4CEFF4
:10DBC0006FF0216A88EC6FF0A0EC6FF021B630EFB7
:10DBD0006FF021A205D021B830EF6FF037EF6FF072
:10DBE00021AA05D021B030EF6FF037EF6FF021B0F0
:10DBF00002D021A802D043EF6FF0256A2F502A24CB
:10DC0000246EE86A25227E0E245EE86A255A326A6E
:10DC1000336A226A236A2E502902F4CF23F0F3CF0D
:10DC200022F02D502902F3503326F4502222000E08
:10DC300023222E502802F3503326F4502222000EC5
:10DC400023222C502902F3503226F4503322000EA6
:10DC5000222223222D502802F3503226F450332260
:10DC6000000E222223222E502702F3503226F45097
:10DC70003322000E222223222C502802F450322676
:10DC8000000E3322222223222D502702F450322666
:10DC9000000E3322222223224CEF6FF028C032F0F4
:10DCA00028502D02F4CF27F0F3CF26F029502E0272
:10DCB000F4CF29F0F3CF28F02D02F3502726F450AB
:10DCC0002822E86A292232502E02F3502726F450E7
:10DCD0002822E86A2922000C216A88EC6FF021B61C
:10DCE00076EF6EF021A20AD021B403D07F0E296E08
:10DCF00019D0800E296E16D0296A14D021B0FCD715
:10DD0000870E2A60F1D77E0E2A64F6D7860E2A5C2B
:10DD100004E0D89029322A2AF9D721A403D0296C0B
:10DD200029AEEAD71200216A88EC6FF021B69DEF88
:10DD30006EF021A20ED021B405D07F0E296EFF0E09
:10DD4000286E1FD0800E296E286A1BD0296A286A87
:10DD500018D021B0FBD78F0E2A60EDD77E0E2A6433
:10DD6000F5D78E0E2A5C05E0D890293228322A2A6F
:10DD7000F8D721A406D0286C291EE86A292229AEEA
:10DD8000E5D71200DBEC6EF021B6000C21B0010CDF
:10DD9000000CDBEC6EF021B6000C21B0000C21B4BD
:10DDA000000C010CDBEC6EF021B6000C21B0000C75
:10DDB00021A4000C010C216A88EC6FF0A0EC6FF03C
:10DDC00021B6120021AE08D021A004D021A802D093
:10DDD00021801200219012002F502A5C0BE12E505E
:10DDE000295C08E12D50285C05E12C50275C02E1FC
:10DDF00021801200D8A002D0218E10D02A502FC02E
:10DE00002AF02F6E29502EC029F02E6E28502DC0DA
:10DE100028F02D6E27502CC027F02C6E2F502A5C36
:10DE200010E0FF0F09E0219021B403D021AE21843E
:10DE3000120021AE219412002F2AD8902E322D32BA
:10DE40002C322C50275E2D50285A2E50295A29BE8C
:10DE5000EAD7D8902736283629362A2EF8D7C8D7B9
:10DE60007F0E2A6EFF0E296E286E276E12007F0E1F
:10DE700021BEFF0E2A6E02D07F0E2A6E800E296E02
:10DE8000286A276AF3D721AE04D0800E2A6E296A49
:10DE9000F7D72A6A296AF4D7235022103310321098
:10DEA000F8E025BEF0D723BE0CD024502510EBE0BF
:10DEB000D89032363336223623362406D8A02506AB
:10DEC000F2D72550D4E12428D2E032AE11D07F0E13
:10DED000321402E133A00CD0332AE86A2222232232
:10DEE00007E3D880233222323332242A2428BFE0A9
:10DEF0002450C9E033C027F022C028F02334296E13
:10DF000024302A6E29322A9E21BE2A8E36EF6FF0E7
:10DF100029362A3602E32184217E06E121802A6AFD
:10DF2000296A286A276A12002A2803E0D880293241
:10DF30001200D890293202E12182120021861200BB
:10DF40002E362F3602E3218C217E06E121882F6AAE
:10DF50002E6A2D6A2C6A12002F2803E0D8802E32F8
:10DF60001200D8902E32EAE1218A1200D9CFE6FFC2
:10DF7000DACFE6FFE1CFD9FFE2CFDAFF0C0EE124E2
:10DF800002E3E168E652E16ED950FA0FE96EFF0E46
:10DF9000DA20EA6E010EEECFDBFF020EEECFDBFFE2
:10DFA000030EEECFDBFF040EEECFDBFF63D8D950BC
:10DFB000010FE96E000EDA20EA6EEECFE6FFEECF3B
:10DFC000E6FFEECFE6FFEFCFE6FF72EC80F0006EEB
:10DFD000060EE15C02E2E16AE552E16E0050DF6E9E
:10DFE000850EDF1404E04DD8EE6AED6A23D0090EE9
:10DFF000DBCF00F00A0EDBCF01F0820E0026FF0E11
:10E0000001223FD800C0EEFF01C0EDFF7E0EF36E8F
:10E01000090EF3CFDBFF0A0EDB6AD950010FE66E63
:10E02000000EDA20E66E26D8F2ECBCF0E552E5529E
:10E03000E552E552010EDBCF00F0020EDBCF01F01E
:10E04000030EDBCF02F0040EDBCF03F000C026F09E
:10E0500001C027F002C028F003C029F00C0EE15CDB
:10E0600002E2E16AE552E16EE552E5CFDAFFE7CF81
:10E07000D9FF1200D950050FE66E000EDA20E66EC9
:10E080001200F80EDBCFE9FFF90EDBCFEAFF12003A
:10E0900026502B02F3CF22F0F4CF23F02C02F350C2
:10E0A0002326000EF420246E26502D02F350242641
:10E0B000000EF420256E26502E02F3502526275000
:10E0C0002B02F3502326F4502422000E2522275041
:10E0D0002C02F3502426F450252227502D02F35011
:10E0E000252628502B02F3502426F45025222850B0
:10E0F0002C02F350252629502B02F350252612001E
:10E10000000000000000000000000000000000000F
:10E1100000000000000000000000000000000000FF
:10E1200000000000000009800000000000006FF007
:10E130000000000000003FE00000000000000000C0
:10E1400000000000000000000000000000000000CF
:10E1500000000000000000000000000000000000BF
:10E16000000000000000000000000000000000208F
:10E170000000000000003AF000000000004BFFA08B
:10E18000000000005CFF91000000006DFE710000C7
:10E1900000017EFD60000000018FFD5000000000C6
:10E1A0009FFB400000000000FA300000000000006B
:10E1B000200000000000000000000000000000003F
:10E1C0000000000000000000000169BCCA720000ED
:10E1D000009FFEDCDFFFB2001DF8200005FDFF30D0
:10E1E000AF3000009F902ED0F800002CF50006F014
:10E1F000F80004ED300005F0AF308FB100000CE006
:10E200001DFDF8000016DF40009FFFDCDEFFC300AD
:10E21000000169BCCA73000000000000000000009B
:10E2200000000000000000000000000000000000EE
:10E2300002900000000001300AB00000000004F06D
:10E240002F600000000004F0AF977777777779F0C0
:10E25000FFFFFFFFFFFFFFF012222222222226F003
:10E2600000000000000004F000000000000003D0E7
:10E27000000000000000000000000000000000009E
:10E28000000000000000000000000000000001404D
:10E2900007D0000000007FF04F800000001CFEF05F
:10E2A000CC00000002EF57F0F70000002EE207F06C
:10E2B000F8000001DE2007F0CE10002DE20007F08C
:10E2C0004FD658FE300007F006FFFFB1000007F000
:10E2D0000014520000000580000000000000000053
:10E2E000000000000000000000000000000002002C
:10E2F0000920000000007F506F40000000002ED079
:10E30000DB000059000007F0F800008E000004F068
:10E31000EA0000CF100006F09F3007FF90001EE0DB
:10E320001EFCDF87FB79EF50019DC6007EFFD50004
:10E3300000000000002100000000000000000000BC
:10E340000000000000000000000000002BB00000F2
:10E3500000000006FFE00000000002CF69E00000BE
:10E3600000007FB109E00000002CE60009E0000099
:10E3700007FB100009E00000CFFCCCCCCEFDDDD0C7
:10E38000DEEEEEEEEFFEEEE00000000009E0000041
:10E390000000000008C000000000000000000000B5
:10E3A000000000000000000000000000000012005B
:10E3B00078ABCDED0000CE20FFEDCCFA00005FB0D1
:10E3C000F90006F0000008F0F9000AB0000004F0BF
:10E3D000F9000AC0000004F0F90008F300000BF097
:10E3E000F90001FE6213BF90F900004EFFFFFB0031
:10E3F000110000016AA940000000000000000000B8
:10E40000000000000000000000000356653000001E
:10E41000004BFFFFFFFFA20008FE968F956AFF30BA
:10E420006F9001F800003ED0EC0008F0000006F00C
:10E43000F6000AE0000004F0F70007F3000009F01E
:10E44000CD1001EF7213AF904D20002DFFFFF900AA
:10E4500000000000478610000000000000000000DF
:10E46000000000000000000011000000000000009B
:10E47000FA00000000000000FA0000000000049014
:10E48000FA0000000039EFF0FA0000017DFFE940DA
:10E49000FA0005BFFF940000FA18EFFB50000000DF
:10E4A000FEFFD71000000000FFB4000000000000D5
:10E4B000520000000000000000000000000000000A
:10E4C0000000000000000000000000000278500082
:10E4D00003ADB4007FFFFC003FFCFF66FA43AFA032
:10E4E000CD101CFE70000BF0F50001FE000005F0E1
:10E4F000F50000BF100004F0EC0007FFB0000AF0C8
:10E500006FD9CF78FB329F9007EFE6009FFFFB00AB
:10E51000000100000388500000000000000000001F
:10E520000000000000000000000355200000000073
:10E5300004DFFFFB10000B604FD7459FD0001CE0AD
:10E54000DD000005F50005F0F7000000F80004F01C
:10E55000F8000000F70008F0BE200006F2005FA0FF
:10E560002EF9547F947CFC0002AFFFFFFFFE700089
:10E570000001467775300000000000000000000038
:10E58000000000000000000000000000000000008B
:10E59000000000000000000000000000000000007B
:10E5A000000006A10000098000001FF900006FF0C4
:10E5B00000000DF500003FE000000010000000002A
:10E5C000000000000000000000000000000000004B
:10E5D000000000000000000000000000000000003B
:10E5E000000000000000000000000000000000002B
:10E5F0000000300000000000BAAEF0000000000093
:10E60000FFE930000000000053000000000000009F
:10E610000000100000000000978CF00000000000D7
:10E62000FFFB50000000000075100000000000001B
:10E6300000000000000000000000000000000000DA
:10E6400000000000000000000000000000000000CA
:10E6500000000000000000000000000000000000BA
:10E660000000000000000000756AE00000000000EB
:10E67000FFFD700000000000A83000000000000056
:10E68000000000000000000000000000000000008A
:10E69000000000000000000000000000000000007A
:10E6A000000000000000000000000000000000006A
:10E6B00000100000000000002CFFA000000000007F
:10E6C000DD78FA0000000000F2005F0000000000AA
:10E6D000F0004F1000000000EA23DC000000000002
:10E6E0004FFFE200000000000154000000000000A5
:10E6F000000000000000000000000000000000001A
:10E7000000001111111111100000FFFFFFFFFFF0B9
:10E7100000009FA7777777700000D6000000000008
:10E720000002F300000000000001FFCBBBBBBBB048
:10E7300000004FFEEEEEEEE00000AB200000000017
:10E740000001F100000000000002FA555555555037
:10E750000000AFFFFFFFFFF00000024444444440CC
:10E76000FFFFFFFFFFFFFFFFFFFFFFFFFFFFFFFFB9
:10E77000FFFFFFFFFFFFFFFFFFFFFFFFFFFFFFFFA9
:10E78000FFFFFFFFFFFFFFFFFFFFFFFFFFFFFFFF99
:10E79000FFFFFFFFFFFFFFFFFFFFFFFFFFFFFFFF89
:10F5100000037ACDEEDCA84000000000000018DFF8
:10F52000FFFFFFFFFFFE920000000007EFFFFFDC80
:10F53000BBCEFFFFFF91000000BFFFC76543223332
:10F5400057BFFFFD20000BFFC40000000000002497
:10F550006EFFD1007FFA000000000000000001BF34
:10F56000FA00EFC00000000000000000000DFF20C6
:10F57000FF6000000000000000000005FF60FF4089
:10F5800000000000000000000003FF70FF8000008A
:10F590000000000000000006FF50CFF30000000054
:10F5A00000000000001DFF104FFE300000000000B2
:10F5B000000001CFF80007FFD71000000000000195
:10F5C0007EFFB000005EFFFB9854333458BFFFFA53
:10F5D000000000019FFFFFFFFFFFFFFFFD50000045
:10F5E0000000017BFFFFFFFFFFE94000000000007B
:10F5F00000000246776541000000000000000000A6
:10F6000000000000000000000000000000000000FA
:10F6100000000000000000000000000000000000EA
:10F6200000000000000000010000000000000000D9
:10F6300000000000001FA00000000000000000010A
:10F640004400009F90000000000000000004FF0044
:10F6500002FF50000000000000000004FF000AFF4D
:10F6600010000000000000000004FF003FFC00004C
:10F670000000000000000004FF00BFFC77777777F0
:10F68000777777777779FF00FFFFFFFFFFFFFFFFB7
:10F69000FFFFFFFFFF00FFFFFFFFFFFFFFFFFFFF79
:10F6A000FFFFFF00333333333333333333333336F6
:10F6B000FF00000000000000000000000004FF0048
:10F6C000000000000000000000000004FF00000037
:10F6D00000000000000000000004FF000000000027
:10F6E0000000000000000003CC000000000000004B
:10F6F000000000000000000000000000000000000A
:10F7000000000000000000000000000000000000F9
:10F7100000000000000000000000000000000000E9
:10F7200000000000000000000000000000000000D9
:10F7300000083000000000000000002AFF0000BFA9
:10F74000D10000000000000008FFFF000AFFB30026
:10F75000000000000003DFFFFF004FFA0000000080
:10F760000000006FFFDBFF00CFE0000000000000A2
:10F7700008FFF808FF00FF800000000000009FFE67
:10F780004008FF00FF40000000000009FFD2000811
:10F79000FF00FF4000000000009FFD100008FF0078
:10F7A000FF800000000008FFD1000008FF00FFE01C
:10F7B000000000008FFE20000008FF009FFA0000FC
:10F7C000001AFFE200000008FF002EFFD62138EFEC
:10F7D000FD2000000008FF0004FFFFFFFFFFC10045
:10F7E00000000008FF00003DFFFFFFE700000000F1
:10F7F0000008FF00000059BB950000000000000B4E
:10F80000FF000000000000000000000000000000F9
:10F8100000000000000000000000000000000000E8
:10F8200000000000000000000000000000000000D8
:10F8300000000000000000000000002000000000A8
:10F8400000000000005E300004F80000000000002E
:10F85000000008FFD0001EFE200000000000000095
:10F8600004DFF8007FF50000000000000000002F1A
:10F87000FE00DFC000000007950000000009FF3017
:10F88000FF700000000CF70000000004FF60FF5054
:10F890000000000EF80000000003FF70FF60000091
:10F8A000002FFA0000000004FF60FFB00000007F9E
:10F8B000FE0000000009FF30BFF4000002EFFF70FF
:10F8C0000000002FFE004FFE60005EFDBFF500004F
:10F8D00003EFF70009FFFFDFFFF32FFFB656BFFF6F
:10F8E000C000008FFFFFFE4004FFFFFFFFFC100081
:10F8F00000028CDB7100002BFFFFFE800000000087
:10F90000000000000000156630000000000000004C
:10F9100000000000000000000000000000000000E7
:10F9200000000000000000000000000000000000D7
:10F930000000000000000000000000000004EFC014
:10F940000000000000000000000001AFFFC0000048
:10F9500000000000000000005EFFFFC0000000008B
:10F9600000000000001BFFD4CFC00000000000001A
:10F97000000006EFF800CFC0000000000000000209
:10F98000BFFC3000CFC0000000000000007FFF700F
:10F990000000CFC00000000000002CFFB2000000FB
:10F9A000CFC0000000000007FFE600000000CFC04D
:10F9B0000000000003CFFA1000000000CFC00000DC
:10F9C00000008FFFEAAAAAAAAAAAEFEAAAAAAA0096
:10F9D000FFFFFFFFFFFFFFFFFFFFFFFFFF00FFFF36
:10F9E000FFFFFFFFFFFFFFFFFFFFFF004444444412
:10F9F00044444444DFD44444440000000000000078
:10FA00000000CFC000000000000000000000000067
:10FA1000CFC000000000000000000000000079706E
:10FA200000000000000000000000000000000000D6
:10FA300000000000000000000000000000000000C6
:10FA40000000000000000000000000200000000096
:10FA5000001234567200000003F80000ABCDEFFF37
:10FA6000FFFFF80000001EFF8000FFFFFFFFFFFF09
:10FA7000F900000028FFF300FFDAA98767FFB00054
:10FA80000000007FFB00FF70000006FF1000000078
:10FA9000000CFF10FF7000000BFA000000000005D2
:10FAA000FF50FF7000000DF7000000000002FF7023
:10FAB000FF7000000EF7000000000002FF70FF70F2
:10FAC00000000EFA000000000004FF60FF7000005C
:10FAD0000BFE10000000000AFF30FF70000006FF60
:10FAE000B0000000006FFD00FF70000000DFFD406F
:10FAF000000029FFF500FF700000003FFFFEBABDC7
:10FB0000FFFF9000FF7000000003DFFFFFFFFFF822
:10FB1000000055200000000007DFFFFFEA30000072
:10FB2000000000000000000134420000000000005E
:10FB300000000000000000000000000000000000C5
:10FB400000000000000000000000000000000012A3
:10FB5000333321000000000000000049CEFFFFFF0A
:10FB6000FFEB7100000000007EFFFFFFFFFFFFFFC3
:10FB7000FF900000003DFFFFFCBAFFFBABEFFFFD75
:10FB8000200004FFFE83001CFD2000028EFFD10038
:10FB90001EFF900000BFE100000001CFF900AFF7A9
:10FBA000000005FF50000000001DFF10FFB0000026
:10FBB0000AFE000000000006FF50FF5000000DFB91
:10FBC000000000000002FF70FF2000000DFC00009C
:10FBD00000000003FF60FF3000000AFF200000006B
:10FBE0000008FF30FF70000005FFC1000000004F5B
:10FBF000FD00EFE1000000CFFD50000028FFF40001
:10FC00007FFD0000002DFFFFDBCDFFFF70000CD259
:10FC100000000001BFFFFFFFFFE500000110000032
:10FC20000000039DFFFEB600000000000000000081
:10FC300000000000000000000000000000000000C4
:10FC400000000000000000000000000000000000B4
:10FC500000000000000000000000000000000000A4
:10FC60000000CC7000000000000000000000000058
:10FC7000FF90000000000000000000000000FF9066
:10FC8000000000000000000000000400FF900000E1
:10FC90000000000000000049EF00FF90000000009D
:10FCA000000000049EFFFF00FF9000000000000025
:10FCB00038DFFFFFFE00FF9000000000017DFFFF26
:10FCC000FFD94000FF9000000005BFFFFFFD83004B
:10FCD0000000FF90000039EFFFFFE8300000000057
:10FCE000FF90006CFFFFFE94000000000000FF92F8
:10FCF0008EFFFFFB5000000000000000FFEFFFFF41
:10FD0000D7100000000000000000FFFFFFA400006B
:10FD10000000000000000000FFFD71000000000076
:10FD2000000000000000BA400000000000000000D9
:10FD300000000000000000000000000000000000C3
:10FD400000000000000000000000000000000000B3
:10FD500000000000000000000000000000000000A3
:10FD60000000000000000367620000000000244261
:10FD700000000004DFFFFFB20000003CFFFFC400F2
:10FD8000008FFFFFFFFE300005FFFFFFFF7008FF41
:10FD9000FB77AFFFE1003FFFA78DFFF64FFC200090
:10FDA00002DFF900BFE300008FFEDFB00000002E8D
:10FDB000FF00FF60000008FFFE1000000008FF4089
:10FDC000FF10000000CFF70000000004FF60FF00FC
:10FDD0000000003FF90000000003FF60FF2000006A
:10FDE000005FFF1000000005FF50FF80000003EFE0
:10FDF000FFA00000000AFF20DFF600005EFCCFF845
:10FE00000000004FFD004FFFC89DFFF33FFFA20021
:10FE100006FFF50007FFFFFFFE4006FFFFDCEFFFD8
:10FE2000A000004CFFFF9100005EFFFFFFFA000002
:10FE300000002430000000018EFFFB4000000000A5
:10FE400000000000000000110000000000000000A1
:10FE500000000000000000000000000000000000A2
:10FE6000000000000000000000000002210000006F
:10FE700000000000000000017DFFFFEA30000000EC
:10FE800000044000006EFFFFFFFFFA000000006F5B
:10FE9000E20008FFFFB99BEFFFC0000000BFFA00BF
:10FEA0004FFF70000005EFF80000000CFF10DFF3BB
:10FEB000000000001EFF10000006FF50FF80000041
:10FEC000000006FF50000004FF60FF40000000003B
:10FED00001FF70000004FF60FF300000000001FF20
:10FEE00070000007FF40FF700000000004FF4000AA
:10FEF000000DFE00EFE2000000000BFD0000009F7F
:10FF0000F8007FFD300000007FF400001AFFD100F0
:10FF10000BFFFB520008FF60136AFFFE200000AFDA
:10FF2000FFFFFFFFFFEFFFFFFFC200000004BFFF66
:10FF3000FFFFFFFFFFFFC500000000000269CDEFDB
:10FF4000FFEDB962000000000000000000000000AA
:10FF500000000000000000000000000000000000A1
:10FF600000000000FFFFFFFFFFFFFFFFFFFFFFFF9D
:10FF7000FFFFFFFFFFFFFFFFFFFFFFFFFFFFFFFF91
:10FF8000FFFFFFFFFFFFFFFFFFFFFFFFFFFFFFFF81
:10FF9000FFFFFFFFFFFFFFFFFFFFFFFFFFFFFFFF71
:10FFA000FFFFFFFFFFFFFFFFFFFFFFFFFFFFFFFF61
:10FFB000FFFFFFFFFFFFFFFFFFFFFFFFFFFFFFFF51
:10FFC000FFFFFFFFFFFFFFFFFFFFFFFFFFFFFFFF41
:10FFD000FFFFFFFFFFFFFFFFFFFFFFFFFFFFFFFF31
:10FFE000FFFFFFFFFFFFFFFFFFFFFFFFFFFFFFFF21
:10FFF000FFFFFFFFFFFFFFFFFFFFFFFFFFFFFFFF11
:020000040001F9
:10000000D7EC85F00501206921691200FFFFFFFF91
:10001000FFFFFFFFFFFFFFFFFFFFFFFFFFFFFFFFF0
:10002000EAEC84F056EFA8F0FFFFFFFFFFFFFFFFB1
:10003000C9EFB3F071EFB9F0C2EFB9F00000FFFF04
:1000400080EC83F005011E6B1200FFFFFFFFFFFF36
:10005000D1EFB3F0FFFFFFFFFFFFFFFFFFFFFFFF49
:1000600056EFA8F0FFFFFFFFFFFFFFFFFFFFFFFFBF
:10007000FFFFFFFFFFFFFFFFFFFFFFFFFFFFFFFF90
:10008000C7ECACF00501030E236F56EFA8F0FFFF9D
:10009000FFFFFFFFFFFFFFFFFFFFFFFFFFFFFFFF70
:1000A0001200FFFFFFFFFFFFFFFFFFFFFFFFFFFF4C
:1000B00066EF6AF076EF6AF0FFFFFFFFFFFFFFFFDA
:1000C00012EFA7F01DEFBAF049EFBAF0FFFFFFFF04
:1000D000FFFFFFFFFFFFFFFFFFFFFFFFFFFFFFFF30
:1000E00032EFB2F0D9CFE6FFDACFE6FFE1CFD9FFAA
:1000F000E2CFDAFFE652006801687F0E026E036A03
:10010000D950FA0FE96EFF0EDA20EA6EEE500016B3
:10011000EE500116EE500216EE5003166AD800C0DB
:10012000EEFF01C0EEFF02C0EEFF03C0EEFFFD0ECA
:10013000DB50800B02E0010E01D0000EE66E59D8B4
:10014000060EE926000EEA22E552E750EF6EFC0E9D
:10015000DBCF00F0FD0EDBCF01F0D890003601368A
:10016000FC0E00C0DBFFFD0E01C0DBFFDB50E66EC6
:1001700040D8040EE926000EEA22E552E750EE6E62
:10018000ED6AFD0EDB50006E016AFF0E001818E1EB
:10019000015016E12ED8EECF00F0EECF01F0EECFF9
:1001A00002F0EFCF03F0005001100210031006E040
:1001B000210E04017C6F7D6B800E0BD0040E09D0E4
:1001C000FD0EDB5008E115D8EE6AEE6AEE6AEE6AC3
:1001D000010EDF6E06D0020EDF6E0BD8EE52EE522D
:1001E000EE8EDF50E552E552E5CFDAFFE7CFD9FFDB
:1001F0001200F80EDBCFE9FFF90EDBCFEAFF1200A9
:10020000BB073BBCFFD03B3C0CF83AF297493AA302
:100210003AE93A6018043A1E099039DF4C01399DD9
:100220003EE5395EED3A39258D333901BAC638CA13
:10023000DC82389E4D8438789D9F3842AC34381823
:10024000C9A33C78BD453BF902CC3BA0443E3B589A
:1002500023623B14FA313AD06DA43A93FBDD3A4F56
:10026000F8033A12718D39DB55AB39AB1277398609
:100270001EEA3952542C3924B2373900DBDA38C936
:1002800044673FA100003F809EED3F5C96533F4195
:10029000B8523F1E19CE3F01CAC13EE1CCCD3ECC83
:1002A00000003EC033333EB3B4393EA8ED913E9CCE
:1002B00026E93E91A1CB3E85F3B63E7D48E93E6EF0
:1002C00006F73FDF06253FB1902E3F98DCC73F85FC
:1002D00008313F6C0C4A3F52020C3F3B73823F2671
:1002E00051EC3F18F3B63F0D86593F08D6A13F04A5
:1002F000A2343F04816F3F0467383F040BE13F03A2
:1003000047AE3F01C2273F26E2193F3851EC3F4834
:10031000068E3F50E9103F578A723F5E18933F6444
:10032000C1553F68154D3F6C91003F6EB7803F70DF
:100330009C783F72538F3F74CFAB3F751DE73F777B
:1003400058103ED91F8A3F1317593F27E8A73F3857
:1003500019653F42B2FF3F4BF1413F53F4F13F5A21
:100360002DE03F60EAB33F6352BD3F6644D03F6833
:1003700085F03F69C7113F6AF4883F6B3C363F6D9B
:10038000AA3BC0B8AA3BC13844FEC19084D4C1D5B1
:10039000CFA2C21B0558C25DAD3BC29C2CCFC2DEB2
:1003A00040F6C31DA22BC352E459C38666EDC3AC0D
:1003B00002D0C3DCA9ABC40C9D93C4330720C46531
:1003C0006C0BC00B6C0BC08BE798C0D959DCC121FA
:1003D000ADBDC16B1F2EC1A7F2BFC1ECFCC7C227C8
:1003E000C193C26D3EA3C29FF7DEC2CB5544C30288
:1003F000540CC326AE9EC354C955C3872522C3AD32
:10040000EC0E3E22F9C93DA9F2A83D5CA08A3D163A
:10041000A1233CCFEC893C92D09A3C4FD3523C1262
:10042000B7263BCF333A3B9B787B3B72CAC03B3D00
:10043000C4D73B14BF583AE84EA53AB6FF0A3A8EE5
:1004400078BE3EBC01903E52DB713E0B57373DC13A
:100450006C183D8674223D3FFBBA3D07C21A3CC072
:10046000AB443C887C103C4CDE0E3C1F74913BFA44
:100470006ABB3BC4B56C3B99E0573B70FA8F3B3C81
:10048000000040800000410000004148000041940D
:10049000000041D833334219333342590000429AA5
:1004A000000042DA000043120000433B0000436FAB
:1004B00080004398000043C3000043F9C000441E7D
:1004C00047AE3FC147AE40410A3D4097AE1440DFC2
:1004D0005C294123AE1441673D7141A4E14841E8E4
:1004E000CCCD4224C28F425C6148428DAE1442B4EE
:1004F000947B42E66B8543133D71433C07AE4370EA
:10050000BEBE3F525D853F14EEEE3ED9FE4C3E9F8F
:10051000D9993E6785273E296EAD3DF54E043DB025
:100520005C8D3D7CEACD3D3D0BB03D152C233CEA76
:1005300012963CB84F6E3C9076823C62DE9F3C3116
:1005400066E03F7D35C63F660D7C3F4507EA3F21AB
:1005500053093EFCC4B53EC2B51C3E92F8A53E58B8
:1005600090BC3E1EB79E3DF148C33DBF42493D97FA
:1005700000D43D6F21693D3C14F53D142E983CE9B3
:10058000000EF36E00EE00F00D0E01D81200EA60CE
:1005900002D0EE6AFCD7F350E9601200EE6AFCD795
:1005A000FFFFFFFFFFFFFFFFFFFFFFFFFFFFFFFF5B
:1005B000FFFFFFFFFFFFFFFFFFFFFFFFFFFFFFFF4B
:1005C000FFFFFFFFFFFFFFFFFFFFFFFFFFFFFFFF3B
:1005D000FFFFFFFFFFFFFFFFFFFFFFFFFFFFFFFF2B
:1005E000FFFFFFFFFFFFFFFFFFFFFFFFFFFFFFFF1B
:1005F000FFFFFFFFFFFFFFFFFFFFFFFFFFFFFFFF0B
:100600002E29C943D8A2017C363DA154F0EC130633
:10061000A762F305C7C08C739398D92B4CBCCA82D0
:100620009B1E3C57D4FD16E04267186F178A12E5EF
:100630004EBED6C49EDA49DEFBA08EF52FBB7AEE05
:1006400068A99179B2153F07C2948910220B215FE6
:100650007F809A5D905A27323E35E7CCF7BF0397EB
:1006600019FFB330A548D1B55ED72A9256ACC6AAB9
:10067000B84FD238A496B67DFC76E26B749CF10438
:100680009D455970716420875B8665CF2DE602A871
:10069000601BAD25B0AEF6B9461C696140340F7ED3
:1006A000475523A351DD3AAF5CC3CEF9C5BA26EA5C
:1006B000532C6E0D28850984DFD3F4CD8141524D32
:1006C000DC6AC837C16CFAABE124087BBD0C4AB1C7
:1006D00088788B9563E36DE8CBE9FED5003B391D47
:1006E000EFF20EB75866E4D077A6F87275EB0A4BB6
:1006F0004431B450ED8F1A1F99DB338D119F148351
:100700000901BD6B0901306B316B0901326B336B31
:100710000901346B356B0901366B376B0901386998
:1007200013EE00F0010EF86E04018C0E346F4A0EC9
:10073000356F4A0E366F3F0E376F00C528F001C582
:1007400029F0E2EC6CF027C000F028C001F029C0CD
:1007500002F02AC003F02C6A2D6A7A0E2E6E440E27
:100760002F6E00C027F001C028F002C029F003C09E
:100770002AF08EEC6DF027C008F428C009F429C0D7
:100780000AF42AC00BF40401006B100E0401005D92
:1007900001E3FAD0DC0E2C6E680E2D6E800E2E6EEC
:1007A0003D0E2F6E08C427F009C428F00AC429F0B2
:1007B0000BC42AF0F7EC6CF027C004F028C005F059
:1007C00029C006F02AC007F004C02CF005C02DF0A7
:1007D00006C02EF007C02FF034C427F035C428F02F
:1007E00036C429F037C42AF0E1EC6DF027C000F0E0
:1007F00028C001F029C002F02AC003F00401005112
:10080000040DF3CFE9FFF4CFEAFF800EE926040ED2
:10081000EA2200C0EEFF01C0EEFF02C0EEFF03C0FF
:10082000EEFF020EF76E04010051002500250025A1
:10083000800FF66E0900F5CF41F40900F5CF40F4C2
:100840000900F5CF43F40800F5CF42F4800FF66EAF
:10085000F72A0900F5CF49F40900F5CF48F409005B
:10086000F5CF4BF40800F5CF4AF404010051040D14
:10087000F3CFE9FFF4CFEAFF800EE926040EEA2267
:10088000EECF08F0EECF09F0EECF0AF0EFCF0BF08D
:1008900040C42CF041C42DF042C42EF043C42FF0CC
:1008A00008C027F009C028F00AC029F00BC02AF0C0
:1008B000F7EC6CF027C004F028C005F029C006F062
:1008C0002AC007F048C42CF049C42DF04AC42EF0C9
:1008D0004BC42FF004C027F005C028F006C029F053
:1008E00007C02AF0E1EC6DF027C000F028C001F04D
:1008F00029C002F02AC003F004010051040DF3CF17
:10090000E9FFF4CFEAFF6B0EE926050EEA2200C0EC
:10091000EEFF01C0EEFF02C0EEFF03C0EEFF0401D8
:100920000051040DF3CFE9FFF4CFEAFF6B0EE92687
:10093000050EEA22EECF00F0EECF01F0EECF02F08E
:10094000EFCF03F02C6A2D6A2E6A2F6A00C027F0C1
:1009500001C028F002C029F003C02AF0D2EC6EF0EA
:10096000010A0FE104010051040DF3CFE9FFF4CFB8
:10097000EAFF6B0EE926050EEA22EE6AEE6AEE6ADF
:10098000EE6A0401002B01D70401100E006F200E47
:100990000401005D12E204010051040DF3CFE9FFF0
:1009A000F4CFEAFF800EE926040EEA22EE6AEE6A30
:1009B000EE6AEE6A0401002BEAD712ECA4F00501FE
:1009C000236B0501226B0501316B0501326B0501BB
:1009D000666B120013EE00F004018C0E346F4A0EA9
:1009E000356F4A0E366F3F0E376F00C528F001C5D0
:1009F00029F0E2EC6CF027C000F028C001F029C01B
:100A000002F02AC003F02C6A2D6A7A0E2E6E440E74
:100A10002F6E00C027F001C028F002C029F003C0EB
:100A20002AF08EEC6DF027C008F428C009F429C024
:100A30000AF42AC00BF402C528F003C529F0E2EC41
:100A40006CF027C000F028C001F029C002F02AC0D5
:100A500003F02C6A2D6A7A0E2E6E440E2F6E00C0A3
:100A600027F001C028F002C029F003C02AF08EEC64
:100A70006DF027C00CF428C00DF429C00EF42AC074
:100A80000FF4DC0E2C6E680E2D6E800E2E6E3D0E59
:100A90002F6E08C427F009C428F00AC429F00BC43B
:100AA0002AF0F7EC6CF027C000F028C001F029C054
:100AB00002F02AC003F000C02CF001C02DF002C0EB
:100AC0002EF003C02FF034C427F035C428F036C40C
:100AD00029F037C42AF0E1EC6DF027C024F428C0D7
:100AE00025F429C026F42AC027F40401286B296BB9
:100AF0002A6B2B6B0CC430F40DC431F40EC432F4E9
:100B00000FC433F413C529F0D1EC6CF027C000F00A
:100B100028C001F029C002F02AC003F02C6A2D6A17
:100B2000C80E2E6E420E2F6E00C027F001C028F0B6
:100B300002C029F003C02AF08EEC6DF027C07BF9CB
:100B400028C07CF929C07DF92AC07EF912C529F098
:100B5000D1EC6CF027C000F028C001F029C002F0F1
:100B60002AC003F02C6A2D6AC80E2E6E420E2F6E1C
:100B700000C027F001C028F002C029F003C02AF00D
:100B80008EEC6DF027C077F928C078F929C079F983
:100B90002AC07AF9BBEC93F012ECA4F00501236BA8
:100BA0000501226B0501316BBFECA4F0120050D897
:100BB0000901BD5105E1010EBD6F00EC60F002D0EE
:100BC000F3EC64F04BEC8CF0BFECA4F00501235186
:100BD000030A27E0020A1DE0010A12E092EC9AF0F3
:100BE00012ECA4F0E3EC69F00301010E066FBDEC1A
:100BF00090F0050123510F0824E2020E236F23D049
:100C000092EC9AF04CEC98F016EC63F00501236935
:100C10001BD0030E235D01E117D0236B4EEC8EF049
:100C200013D012ECA4F0E3EC69F0C2EC69F002011D
:100C3000C76B926B92EC9AF0FCEC64F00501236BAD
:100C400003D04EEC8EF000D0E4EC99F0F7EF64F0B6
:100C500000C528F001C529F0E2EC6CF027C000F0D7
:100C600028C001F029C002F02AC003F02C6A2D6AC6
:100C70007A0E2E6E440E2F6E00C027F001C028F0B1
:100C800002C029F003C02AF08EEC6DF027C008F4F2
:100C900028C009F429C00AF42AC00BF402C528F0C0
:100CA00003C529F0E2EC6CF027C000F028C001F089
:100CB00029C002F02AC003F02C6A2D6A7A0E2E6E2B
:100CC000440E2F6E00C027F001C028F002C029F0AA
:100CD00003C02AF08EEC6DF027C00CF428C00DF490
:100CE00029C00EF42AC00FF410C529F0D1EC6CF025
:100CF00027C000F028C001F029C002F02AC003F08C
:100D00002C6A2D6AC80E2E6E420E2F6E00C027F080
:100D100001C028F002C029F003C02AF08EEC6DF06B
:100D200027C034F428C035F429C036F42AC037F47B
:100D300011C529F0D1EC6CF027C000F028C001F0FB
:100D400029C002F02AC003F02C6A2D6AC80E2E6E4C
:100D5000420E2F6E00C027F001C028F002C029F01B
:100D600003C02AF08EEC6DF027C038F428C039F4A7
:100D700029C03AF42AC03BF41CC529F0D1EC6CF030
:100D800027C000F028C001F029C002F02AC003F0FB
:100D90002C6A2D6AC80E2E6E420E2F6E00C027F0F0
:100DA00001C028F002C029F003C02AF08EEC6DF0DB
:100DB00027C05FF928C060F929C061F92AC062F92B
:100DC0001DC529F0D1EC6CF027C000F028C001F05F
:100DD00029C002F02AC003F02C6A2D6AC80E2E6EBC
:100DE000420E2F6E00C027F001C028F002C029F08B
:100DF00003C02AF08EEC6DF027C063F928C064F9B7
:100E000029C065F92AC066F908C529F0D1EC6CF053
:100E100027C000F028C001F029C002F02AC003F06A
:100E20002C6A2D6AC80E2E6E420E2F6E00C027F05F
:100E300001C028F002C029F003C02AF08EEC6DF04A
:100E400027C0D2F928C0D3F929C0D4F92AC0D5F9CE
:100E500009C529F0D1EC6CF027C000F028C001F0E2
:100E600029C002F02AC003F02C6A2D6AC80E2E6E2B
:100E7000420E2F6E00C027F001C028F002C029F0FA
:100E800003C02AF08EEC6DF027C0E2F928C0E3F928
:100E900029C0E4F92AC0E5F90AC529F0D1EC6CF0C3
:100EA00027C000F028C001F029C002F02AC003F0DA
:100EB0002C6A2D6AC80E2E6E420E2F6E00C027F0CF
:100EC00001C028F002C029F003C02AF08EEC6DF0BA
:100ED00027C0D6F928C0D7F929C0D8F92AC0D9F92E
:100EE0000BC529F0D1EC6CF027C000F028C001F050
:100EF00029C002F02AC003F02C6A2D6AC80E2E6E9B
:100F0000420E2F6E00C027F001C028F002C029F069
:100F100003C02AF08EEC6DF027C0E6F928C0E7F98F
:100F200029C0E8F92AC0E9F90CC529F0D1EC6CF028
:100F300027C000F028C001F029C002F02AC003F049
:100F40002C6A2D6AC80E2E6E420E2F6E00C027F03E
:100F500001C028F002C029F003C02AF08EEC6DF029
:100F600027C0DAF928C0DBF929C0DCF92AC0DDF98D
:100F70000DC529F0D1EC6CF027C000F028C001F0BD
:100F800029C002F02AC003F02C6A2D6AC80E2E6E0A
:100F9000420E2F6E00C027F001C028F002C029F0D9
:100FA00003C02AF08EEC6DF027C0EAF928C0EBF9F7
:100FB00029C0ECF92AC0EDF90EC529F0D1EC6CF08E
:100FC00027C000F028C001F029C002F02AC003F0B9
:100FD0002C6A2D6AC80E2E6E420E2F6E00C027F0AE
:100FE00001C028F002C029F003C02AF08EEC6DF099
:100FF00027C0DEF928C0DFF929C0E0F92AC0E1F9ED
:101000000FC529F0D1EC6CF027C000F028C001F02A
:1010100029C002F02AC003F02C6A2D6AC80E2E6E79
:10102000420E2F6E00C027F001C028F002C029F048
:1010300003C02AF08EEC6DF027C0EEF928C0EFF95E
:1010400029C0F0F92AC0F1F917C529F0D1EC6CF0EC
:1010500027C000F028C001F029C002F02AC003F028
:101060002C6A2D6AC80E2E6E420E2F6E00C027F01D
:1010700001C028F002C029F003C02AF08EEC6DF008
:1010800027C07FF928C080F929C081F92AC082F9D8
:101090002C6A2D6A160E2E6E430E2F6E08C427F092
:1010A00009C428F00AC429F00BC42AF0F8EC6CF04B
:1010B00027C000F028C001F029C002F02AC003F0C8
:1010C00002C528F003C529F0E2EC6CF027C004F05B
:1010D00028C005F029C006F02AC007F004C02CF093
:1010E00005C02DF006C02EF007C02FF000C027F07D
:1010F00001C028F002C029F003C02AF0F7EC6CF020
:1011000093EC6EF028C004F429C005F405011B51CE
:1011100064E01B51006E016A04010451005C05513A
:1011200001585BE21BC529F0D1EC6CF027C004F03C
:1011300028C005F029C006F02AC007F0850E2C6EE5
:10114000EB0E2D6E1F0E2E6E410E2F6E04C027F07B
:1011500005C028F006C029F007C02AF08EEC6DF01B
:1011600027C000F028C001F029C002F02AC003F017
:101170000CC42CF00DC42DF00EC42EF00FC42FF0B3
:1011800000C027F001C028F002C029F003C02AF0F7
:10119000F8EC6CF027C06FF928C070F929C071F91C
:1011A0002AC072F97FC92CF080C92DF081C92EF0B8
:1011B00082C92FF06FC927F070C928F071C929F0D2
:1011C00072C92AF0F8EC6CF027C06FF928C070F9EA
:1011D00029C071F92AC072F905D009016F6B706BD3
:1011E000716B726B05011B5164E01B51006E016A4B
:1011F00004010451005C055101585BE267C529F008
:10120000D1EC6CF027C004F028C005F029C006F02E
:101210002AC007F0850E2C6EEB0E2D6E1F0E2E6E63
:10122000410E2F6E04C027F005C028F006C029F03B
:1012300007C02AF08EEC6DF027C000F028C001F046
:1012400029C002F02AC003F00CC42CF00DC42DF00C
:101250000EC42EF00FC42FF000C027F001C028F0FC
:1012600002C029F003C02AF0F8EC6CF027C0C2F9E4
:1012700028C0C3F929C0C4F92AC0C5F97FC92CF018
:1012800080C92DF081C92EF082C92FF0C2C927F084
:10129000C3C928F0C4C929F0C5C92AF0F8EC6CF01C
:1012A00027C0C2F928C0C3F929C0C4F92AC0C5F9AA
:1012B00005D00901C26BC36BC46BC56B05011B5123
:1012C00064E01B51006E016A04010451005C055189
:1012D00001585BE268C529F0D1EC6CF027C004F03E
:1012E00028C005F029C006F02AC007F0850E2C6E34
:1012F000EB0E2D6E1F0E2E6E410E2F6E04C027F0CA
:1013000005C028F006C029F007C02AF08EEC6DF069
:1013100027C000F028C001F029C002F02AC003F065
:101320000CC42CF00DC42DF00EC42EF00FC42FF001
:1013300000C027F001C028F002C029F003C02AF045
:10134000F8EC6CF027C0C6F928C0C7F929C0C8F965
:101350002AC0C9F97FC92CF080C92DF081C92EF0AF
:1013600082C92FF0C6C927F0C7C928F0C8C929F01B
:10137000C9C92AF0F8EC6CF027C0C6F928C0C7F933
:1013800029C0C8F92AC0C9F906D009016F6B706B72
:10139000400E716F726F05011B5164E01B51006EAE
:1013A000016A04010451005C055101585BE269C502
:1013B00029F0D1EC6CF027C004F028C005F029C05A
:1013C00006F02AC007F0850E2C6EEB0E2D6E1F0E58
:1013D0002E6E410E2F6E04C027F005C028F006C007
:1013E00029F007C02AF08EEC6DF027C000F028C06D
:1013F00001F029C002F02AC003F00CC42CF00DC487
:101400002DF00EC42EF00FC42FF000C027F001C045
:1014100028F002C029F003C02AF0F8EC6CF027C0D5
:10142000CAF928C0CBF929C0CCF92AC0CDF97FC9A7
:101430002CF080C92DF081C92EF082C92FF0CAC9C5
:1014400027F0CBC928F0CCC929F0CDC92AF0F8EC97
:101450006CF027C0CAF928C0CBF929C0CCF92AC042
:10146000CDF907D009016F6B706B800E716F400E64
:10147000726F05011B5164E01B51006E016A04018B
:101480000451005C055101585BE26AC529F0D1ECBA
:101490006CF027C004F028C005F029C006F02AC06F
:1014A00007F0850E2C6EEB0E2D6E1F0E2E6E410E6C
:1014B0002F6E04C027F005C028F006C029F007C031
:1014C0002AF08EEC6DF027C000F028C001F029C092
:1014D00002F02AC003F00CC42CF00DC42DF00EC491
:1014E0002EF00FC42FF000C027F001C028F002C07A
:1014F00029F003C02AF0F8EC6CF027C0CEF928C020
:10150000CFF929C0D0F92AC0D1F97FC92CF080C900
:101510002DF081C92EF082C92FF0CEC927F0CFC996
:1015200028F0D0C929F0D1C92AF0F8EC6CF027C016
:10153000CEF928C0CFF929C0D0F92AC0D1F905D0F9
:101540000901CE6BCF6BD06BD16B18C529F0D1ECF4
:101550006CF027C000F028C001F029C002F02AC0BA
:1015600003F02C6A2D6AC80E2E6E420E2F6E00C03C
:1015700027F001C028F002C029F003C02AF08EEC49
:101580006DF027C0F3F528C0F4F529C0F5F52AC0A1
:10159000F6F519C529F0D1EC6CF027C004F028C08D
:1015A00005F029C006F02AC007F0660E2C6EE60E84
:1015B0002D6EC70E2E6E420E2F6E04C027F005C092
:1015C00028F006C029F007C02AF08EEC6DF027C085
:1015D00000F028C001F029C002F02AC003F00CC4BA
:1015E0002CF00DC42DF00EC42EF00FC42FF000C04F
:1015F00027F001C028F002C029F003C02AF0F8EC5F
:101600006CF027C0F7F528C0F8F529C0F9F52AC015
:10161000FAF57FC92CF080C92DF081C92EF082C95E
:101620002FF0F7C527F0F8C528F0F9C529F0FAC55D
:101630002AF0F8EC6CF027C0F7F528C0F8F529C0BF
:10164000F9F52AC0FAF51AC529F0D1EC6CF027C0DB
:1016500000F028C001F029C002F02AC003F02C6A73
:101660002D6AC80E2E6E420E2F6E00C027F001C0EC
:1016700028F002C029F003C02AF08EEC6DF027C0DC
:10168000FBF528C0FCF529C0FDF52AC0FEF513C501
:1016900029F0D1EC6CF027C000F028C001F029C07F
:1016A00002F02AC003F02C6A2D6AC80E2E6E420E7C
:1016B0002F6E00C027F001C028F002C029F003C03F
:1016C0002AF08EEC6DF027C07BF928C07CF929C088
:1016D0007DF92AC07EF912C529F0D1EC6CF027C043
:1016E00000F028C001F029C002F02AC003F02C6AE3
:1016F0002D6AC80E2E6E420E2F6E00C027F001C05C
:1017000028F002C029F003C02AF08EEC6DF027C04B
:1017100077F928C078F929C079F92AC07AF915C56E
:1017200029F0D1EC6CF027C000F028C001F029C0EE
:1017300002F02AC003F02C6A2D6AC80E2E6E420EEB
:101740002F6E00C027F001C028F002C029F003C0AE
:101750002AF08EEC6DF027C097F228C098F229C0CD
:1017600099F22AC09AF214C529F0D1EC6CF027C086
:1017700000F028C001F029C002F02AC003F02C6A52
:101780002D6AC80E2E6E420E2F6E00C027F001C0CB
:1017900028F002C029F003C02AF08EEC6DF027C0BB
:1017A0009BF228C09CF229C09DF22AC09EF297C2EB
:1017B0002CF098C22DF099C22EF09AC22FF09BC245
:1017C00027F09CC228F09DC229F09EC22AF0F7ECB7
:1017D0006CF027C09FF228C0A0F229C0A1F22AC055
:1017E000A2F20CC42CF00DC42DF00EC42EF00FC4C8
:1017F0002FF008C427F009C428F00AC429F00BC44C
:101800002AF0F7EC6CF027C000F028C001F029C0E6
:1018100002F02AC003F0F00E2C6E850E2D6E990E8C
:101820002E6E3E0E2F6E00C027F001C028F002C0C1
:1018300029F003C02AF08EEC6DF027C014F428C004
:1018400015F429C016F42AC017F414C427F015C4DF
:1018500028F016C429F017C42AF093EC6EF028C0C3
:1018600004F429C005F40401000E045D000E0559BE
:1018700002E2046B056BFF0ED8800455000E05557F
:1018800002E20469056B04C44FF205011E51020116
:10189000C36FC46B1200010E02019025906F000E01
:1018A0009121916F0501185109E108C4EBF509C4B4
:1018B000ECF50AC4EDF50BC4EEF54ED0F3C52CF0F3
:1018C000F4C52DF0F5C52EF0F6C52FF008C427F0AD
:1018D00009C428F00AC429F00BC42AF0F7EC6CF014
:1018E00027C000F028C001F029C002F02AC003F090
:1018F00038C42CF039C42DF03AC42EF03BC42FF07C
:1019000034C427F035C428F036C429F037C42AF08F
:10191000F8EC6CF027C004F028C005F029C006F0F0
:101920002AC007F004C02CF005C02DF006C02EF030
:1019300007C02FF000C027F001C028F002C029F036
:1019400003C02AF08EEC6DF027C0EBF528C0ECF553
:1019500029C0EDF52AC0EEF508C42CF009C42DF01D
:101960000AC42EF00BC42FF0EBC527F0ECC528F00D
:10197000EDC529F0EEC52AF0C9EC6EF0010A08E1C8
:1019800008C4EBF509C4ECF50AC4EDF50BC4EEF59B
:10199000DC0E2C6E680E2D6E800E2E6E3D0E2F6EA0
:1019A000EBC527F0ECC528F0EDC529F0EEC52AF00F
:1019B000C9EC6EF0010A01E097D0DC0E2C6E680EC7
:1019C0002D6E800E2E6E3D0E2F6EEBC527F0ECC5F2
:1019D00028F0EDC529F0EEC52AF0F7EC6CF027C031
:1019E00000F028C001F029C002F02AC003F000C0B6
:1019F0002CF001C02DF002C02EF003C02FF034C433
:101A000027F035C428F036C429F037C42AF0E1ECB9
:101A10006DF027C024F428C025F429C026F42AC07C
:101A200027F4DC0E2C6E680E2D6E800E2E6E3D0E91
:101A30002F6EEBC527F0ECC528F0EDC529F0EEC5FB
:101A40002AF0F7EC6CF027C000F028C001F029C0A4
:101A500002F02AC003F000C02CF001C02DF002C03B
:101A60002EF003C02FF038C427F039C428F03AC450
:101A700029F03BC42AF0E1EC6DF027C028F428C01F
:101A800029F429C02AF42AC02BF408C42CF009C474
:101A90002DF00AC42EF00BC42FF0EBC527F0ECC5D7
:101AA00028F0EDC529F0EEC52AF08EEC6DF027C0C8
:101AB00000F028C001F029C002F02AC003F02C6A0F
:101AC0002D6AC80E2E6E420E2F6E00C027F001C088
:101AD00028F002C029F003C02AF0E1EC6DF06CECB4
:101AE0006EF029C064F50BD00401246B256B266BC6
:101AF000276B286B296B2A6B2B6B0501646B0CC45D
:101B000030F40DC431F40EC432F40FC433F40201C6
:101B10004C5103E1BBEC93F002D0BAECADF00501FF
:101B20006351040DF3CFE9FFF4CFEAFF6B0EE92612
:101B3000050EEA22EECF00F0EECF01F0EECF02F07C
:101B4000EFCF03F02C6A2D6A7A0E2E6E440E2F6EA4
:101B500000C027F001C028F002C029F003C02AF01D
:101B6000E1EC6DF093EC6EF028C044F229C045F230
:101B700005016351040DF3CFE9FFF4CFEAFF800EB6
:101B8000E926040EEA22EECF04F0EECF05F0EECF08
:101B900006F0EFCF07F0100E6325040DF3CFE9FF39
:101BA000F4CFEAFF800EE926040EEA22EECF08F019
:101BB000EECF09F0EECF0AF0EFCF0BF008C02CF01B
:101BC00009C02DF00AC02EF00BC02FF004C027F082
:101BD00005C028F006C029F007C02AF0F8EC6CF028
:101BE00027C000F028C001F029C002F02AC003F08D
:101BF0002C6A2D6A7A0E2E6E440E2F6E00C027F0CE
:101C000001C028F002C029F003C02AF0E1EC6DF019
:101C100093EC6EF028C046F229C047F205011F057B
:101C20001BE19BC22CF09CC22DF09DC22EF09EC2E7
:101C30002FF010C427F011C428F012C429F013C4E7
:101C40002AF0E1EC6DF027C010F428C011F429C08F
:101C500012F42AC013F408D030C410F431C411F4C3
:101C600032C412F433C413F410C42CF011C42DF098
:101C700012C42EF013C42FF070C427F071C428F0E2
:101C800072C429F073C42AF0C9EC6EF0010A05E1B0
:101C90000501235102E1226B236912000401066B46
:101CA000076BFCEC64F00201000ED880BF55000EFB
:101CB000C05501E34DD20501185101E0D2D020C436
:101CC000EFF521C4F0F522C4F1F523C4F2F56FC994
:101CD0002CF070C92DF071C92EF072C92FF020C4FC
:101CE00027F021C428F022C429F023C42AF0C9EC2B
:101CF0006EF0010A11E134C467F935C468F936C4DD
:101D000069F937C46AF938C46BF939C46CF93AC453
:101D10006DF93BC46EF9A4D0C2C92CF0C3C92DF033
:101D2000C4C92EF0C5C92FF020C427F021C428F063
:101D300022C429F023C42AF0C9EC6EF0010A11E193
:101D40005FC967F960C968F961C969F962C96AF967
:101D500063C96BF964C96CF965C96DF966C96EF937
:101D60007FD0C6C92CF0C7C92DF0C8C92EF0C9C98B
:101D70002FF020C427F021C428F022C429F023C466
:101D80002AF0C9EC6EF0010A11E1D2C967F9D3C992
:101D900068F9D4C969F9D5C96AF9E2C96BF9E3C927
:101DA0006CF9E4C96DF9E5C96EF95AD0CAC92CF0CD
:101DB000CBC92DF0CCC92EF0CDC92FF020C427F00F
:101DC00021C428F022C429F023C42AF0C9EC6EF003
:101DD000010A11E1D6C967F9D7C968F9D8C969F903
:101DE000D9C96AF9E6C96BF9E7C96CF9E8C96DF9AF
:101DF000E9C96EF935D0CEC92CF0CFC92DF0D0C9C4
:101E00002EF0D1C92FF020C427F021C428F022C41D
:101E100029F023C42AF0C9EC6EF0010A11E1DAC9F5
:101E200067F9DBC968F9DCC969F9DDC96AF9EAC98A
:101E30006BF9EBC96CF9ECC96DF9EDC96EF910D00D
:101E40005FC967F960C968F961C969F962C96AF966
:101E500063C96BF964C96CF965C96DF966C96EF936
:101E6000C1D034C467F935C468F936C469F937C4D8
:101E70006AF938C46BF939C46CF93AC46DF93BC4DA
:101E80006EF9F7C52CF0F8C52DF0F9C52EF0FAC59E
:101E90002FF020C427F021C428F022C429F023C445
:101EA0002AF0C9EC6EF0010A4FE1F3C52CF0F4C53D
:101EB0002DF0F5C52EF0F6C52FF020C427F021C473
:101EC00028F022C429F023C42AF0F7EC6CF027C0D4
:101ED00000F028C001F029C002F02AC003F038C485
:101EE0002CF039C42DF03AC42EF03BC42FF034C48A
:101EF00027F035C428F036C429F037C42AF0F8ECAE
:101F00006CF027C004F028C005F029C006F02AC0F4
:101F100007F004C02CF005C02DF006C02EF007C05D
:101F20002FF000C027F001C028F002C029F003C044
:101F30002AF08EEC6DF027C0EFF528C0F0F529C02F
:101F4000F1F52AC0F2F54ED0FBC52CF0FCC52DF002
:101F5000FDC52EF0FEC52FF020C427F021C428F0C7
:101F600022C429F023C42AF0F7EC6CF027C000F05B
:101F700028C001F029C002F02AC003F038C42CF0B8
:101F800039C42DF03AC42EF03BC42FF034C427F0EE
:101F900035C428F036C429F037C42AF0F8EC6CF0C8
:101FA00027C004F028C005F029C006F02AC007F0B9
:101FB00004C02CF005C02DF006C02EF007C02FF095
:101FC00000C027F001C028F002C029F003C02AF0A9
:101FD0008EEC6DF027C0EFF528C0F0F529C0F1F5C3
:101FE0002AC0F2F520C42CF021C42DF022C42EF01A
:101FF00023C42FF0EFC527F0F0C528F0F1C529F074
:10200000F2C52AF0C9EC6EF0010A08E120C4EFF530
:1020100021C4F0F522C4F1F523C4F2F5DC0E2C6ED8
:10202000680E2D6E800E2E6E3D0E2F6EEFC527F0C2
:10203000F0C528F0F1C529F0F2C52AF0C9EC6EF020
:10204000010A69E1DC0E2C6E680E2D6E800E2E6E7C
:102050003D0E2F6EEFC527F0F0C528F0F1C529F031
:10206000F2C52AF0F7EC6CF027C000F028C001F0B0
:1020700029C002F02AC003F000C02CF001C02DF0EE
:1020800002C02EF003C02FF067C927F068C928F0FE
:1020900069C929F06AC92AF0E1EC6DF027C024F47F
:1020A00028C025F429C026F42AC027F4DC0E2C6EA3
:1020B000680E2D6E800E2E6E3D0E2F6EEFC527F032
:1020C000F0C528F0F1C529F0F2C52AF0F7EC6CF064
:1020D00027C000F028C001F029C002F02AC003F098
:1020E00000C02CF001C02DF002C02EF003C02FF074
:1020F0006BC927F06CC928F06DC929F06EC92AF0A8
:10210000E1EC6DF027C028F428C029F429C02AF496
:102110002AC02BF409D00401246B256B266B276B96
:10212000286B296B2A6B2B6BCFEC9BF0F5EC69F0DD
:102130000201010EC16F21ECA4F005012329236FD8
:10214000100E235D04E2010E0401066F076B02D03E
:102150000501236B0401010E061901E1075101E19C
:102160009DD5050123510F0803E2010E236F04D012
:10217000C2EC69F00501236B120092EC9AF00501A4
:10218000236B08C420F409C421F40AC422F40BC44C
:1021900023F40201010E926F0401066B076B2C6A97
:1021A0002D6A800E2E6E3F0E2F6E20C427F021C4A4
:1021B00028F022C429F023C42AF0F7EC6CF027C0E1
:1021C00020F428C021F429C022F42AC023F40501F8
:1021D0001F0509E1B7C293F2B8C294F2B9C295F2F1
:1021E000BAC296F208D074C493F275C494F276C45D
:1021F00095F277C496F293C22CF094C22DF095C25A
:102200002EF096C22FF020C427F021C428F022C45B
:1022100029F023C42AF0C9EC6EF0010A01E0A3D230
:102220000CC42CF00DC42DF00EC42EF00FC42FF0F2
:1022300020C427F021C428F022C429F023C42AF0A6
:10224000C9EC6EF0010A01E08ED20201926B03012B
:10225000066B2C6A2D6A2E6A3F0E2F6E20C427F063
:1022600021C428F022C429F023C42AF0F8EC6CF031
:1022700027C020F428C021F429C022F42AC023F466
:102280000501185101E0E9D020C4EFF521C4F0F5B3
:1022900022C4F1F523C4F2F52C6A2D6A2E6A3F0E92
:1022A0002F6E20C427F021C428F022C429F023C4B3
:1022B0002AF0F8EC6CF027C000F028C001F029C02B
:1022C00002F02AC003F06FC92CF070C92DF071C95B
:1022D0002EF072C92FF000C027F001C028F002C014
:1022E00029F003C02AF0C9EC6EF0010A11E134C4F0
:1022F00067F935C468F936C469F937C46AF938C46E
:102300006BF939C46CF93AC46DF93BC46EF9A4D0C9
:10231000C2C92CF0C3C92DF0C4C92EF0C5C92FF015
:1023200020C427F021C428F022C429F023C42AF0B5
:10233000C9EC6EF0010A11E15FC967F960C968F97B
:1023400061C969F962C96AF963C96BF964C96CF951
:1023500065C96DF966C96EF97FD0C6C92CF0C7C9C9
:102360002DF0C8C92EF0C9C92FF020C427F021C410
:1023700028F022C429F023C42AF0C9EC6EF0010A27
:1023800011E1D2C967F9D3C968F9D4C969F9D5C9C6
:102390006AF9E2C96BF9E3C96CF9E4C96DF9E5C9F9
:1023A0006EF95AD0CAC92CF0CBC92DF0CCC92EF089
:1023B000CDC92FF020C427F021C428F022C429F071
:1023C00023C42AF0C9EC6EF0010A11E1D6C967F9FD
:1023D000D7C968F9D8C969F9D9C96AF9E6C96BF9E1
:1023E000E7C96CF9E8C96DF9E9C96EF935D0CEC90C
:1023F0002CF0CFC92DF0D0C92EF0D1C92FF020C4B8
:1024000027F021C428F022C429F023C42AF0C9EC03
:102410006EF0010A11E1DAC967F9DBC968F9DCC9B4
:1024200069F9DDC96AF9EAC96BF9EBC96CF9ECC95C
:102430006DF9EDC96EF910D05FC967F960C968F927
:1024400061C969F962C96AF963C96BF964C96CF950
:1024500065C96DF966C96EF9DDD034C467F935C454
:1024600068F936C469F937C46AF938C46BF939C4F4
:102470006CF93AC46DF93BC46EF9F7C52CF0F8C598
:102480002DF0F9C52EF0FAC52FF020C427F021C495
:1024900028F022C429F023C42AF0C9EC6EF0010A06
:1024A0004FE1F3C52CF0F4C52DF0F5C52EF0F6C5BF
:1024B0002FF020C427F021C428F022C429F023C41F
:1024C0002AF0F7EC6CF027C000F028C001F029C01A
:1024D00002F02AC003F038C42CF039C42DF03AC4FD
:1024E0002EF03BC42FF034C427F035C428F036C496
:1024F00029F037C42AF0F8EC6CF027C004F028C0AB
:1025000005F029C006F02AC007F004C02CF005C071
:102510002DF006C02EF007C02FF000C027F001C03C
:1025200028F002C029F003C02AF08EEC6DF027C01D
:10253000EFF528C0F0F529C0F1F52AC0F2F54ED02C
:10254000FBC52CF0FCC52DF0FDC52EF0FEC52FF00F
:1025500020C427F021C428F022C429F023C42AF083
:10256000F7EC6CF027C000F028C001F029C002F0A1
:102570002AC003F038C42CF039C42DF03AC42EF030
:102580003BC42FF034C427F035C428F036C429F0FA
:1025900037C42AF0F8EC6CF027C004F028C005F02E
:1025A00029C006F02AC007F004C02CF005C02DF0A9
:1025B00006C02EF007C02FF000C027F001C028F0A1
:1025C00002C029F003C02AF08EEC6DF027C0EFF5B1
:1025D00028C0F0F529C0F1F52AC0F2F520C42CF08E
:1025E00021C42DF022C42EF023C42FF0EFC527F014
:1025F000F0C528F0F1C529F0F2C52AF0C9EC6EF05B
:10260000010A08E120C4EFF521C4F0F522C4F1F578
:1026100023C4F2F52C6A2D6A2E6A3F0E2F6E20C459
:1026200027F021C428F022C429F023C42AF0F7ECB3
:102630006CF027C020F428C021F429C022F42AC05D
:1026400023F4DC0E2C6E680E2D6E800E2E6E3D0E69
:102650002F6EEFC527F0F0C528F0F1C529F0F2C5BF
:102660002AF0C9EC6EF0010A69E1DC0E2C6E680EEE
:102670002D6E800E2E6E3D0E2F6EEFC527F0F0C52D
:1026800028F0F1C529F0F2C52AF0F7EC6CF027C06C
:1026900000F028C001F029C002F02AC003F000C0F9
:1026A0002CF001C02DF002C02EF003C02FF067C93E
:1026B00027F068C928F069C929F06AC92AF0E1EC55
:1026C0006DF027C024F428C025F429C026F42AC0C0
:1026D00027F4DC0E2C6E680E2D6E800E2E6E3D0ED5
:1026E0002F6EEFC527F0F0C528F0F1C529F0F2C52F
:1026F0002AF0F7EC6CF027C000F028C001F029C0E8
:1027000002F02AC003F000C02CF001C02DF002C07E
:102710002EF003C02FF06BC927F06CC928F06DC9EB
:1027200029F06EC92AF0E1EC6DF027C028F428C02A
:1027300029F429C02AF42AC02BF409D00401246BFF
:10274000256B266B276B286B296B2A6B2B6BCFECC9
:102750009BF005012329236F100E235D04E2010E77
:102760000401066F076B0401010E061901E1075110
:1027700001E112D5120013EE00F0010EF86E050112
:1027800063690401706B716B726B736B0401006B96
:10279000100E0401005D02E34BEF98F0020EF76E9D
:1027A00004010051002500250025F66E0900F5CF33
:1027B00059F40900F5CF58F40900F5CF5BF408008F
:1027C000F5CF5AF4400FF66E0900F5CF5DF409001D
:1027D000F5CF5CF40900F5CF5FF40800F5CF5EF4A7
:1027E000400FF66E0900F5CF41F40900F5CF40F433
:1027F0000900F5CF43F40800F5CF42F4400FF66E20
:102800000900F5CF45F40900F5CF44F40900F5CFF0
:1028100047F40800F5CF46F4400FF66EF72A09009A
:10282000F5CF49F40900F5CF48F40900F5CF4BF492
:102830000800F5CF4AF4400FF66E0900F5CF4DF4CD
:102840000900F5CF4CF40900F5CF4FF40800F5CF9F
:102850004EF4D40E2C6E400E2D6E180E2E6E380EC9
:102860002F6E58C427F059C428F05AC429F05BC40D
:102870002AF0D2EC6EF0010A01E1DED0450E2C6E9A
:10288000120E2D6EBD0E2E6E3B0E2F6E58C427F00D
:1028900059C428F05AC429F05BC42AF0C9EC6EF080
:1028A000010A01E1C9D04B0E2C6E890E2D6EC90EA6
:1028B0002E6E380E2F6E5CC427F05DC428F05EC407
:1028C00029F05FC42AF0D2EC6EF0010A01E1B4D025
:1028D0009A0E2C6E990E2D6E190E2E6E3E0E2F6EC8
:1028E0005CC427F05DC428F05EC429F05FC42AF000
:1028F000C9EC6EF0010A01E19FD0440E2C6E8B0EE4
:102900002D6E6C0E2E6E3E0E2F6E40C427F041C40D
:1029100028F042C429F043C42AF0D2EC6EF0010A38
:1029200001E18AD05C0E2C6E8F0E2D6EA20E2E6EE3
:102930003F0E2F6E40C427F041C428F042C429F056
:1029400043C42AF0C9EC6EF0010A76E0250E2C6E25
:10295000060E2D6E010E2E6E3F0E2F6E48C427F010
:1029600049C428F04AC429F04BC42AF0D2EC6EF0D6
:10297000010A62E0C70E2C6E4B0E2D6E770E2E6E86
:102980003F0E2F6E48C427F049C428F04AC429F0EE
:102990004BC42AF0C9EC6EF0010A4EE05C0E2C6EBE
:1029A0008F0E2D6E020E2E6E3F0E2F6E44C427F03A
:1029B00045C428F046C429F047C42AF0D2EC6EF092
:1029C000010A3AE02C6A2D6AE00E2E6E3F0E2F6E41
:1029D00044C427F045C428F046C429F047C42AF06F
:1029E000C9EC6EF0010A28E0750E2C6E930E2D6E68
:1029F000D80E2E6E3E0E2F6E4CC427F04DC428F01C
:102A00004EC429F04FC42AF0D2EC6EF0010A14E053
:102A1000DF0E2C6E4F0E2D6E6D0E2E6E3F0E2F6E36
:102A20004CC427F04DC428F04EC429F04FC42AF0FE
:102A3000C9EC6EF0010A02E10901358B0401005175
:102A4000040DF3CFE9FFF4CFEAFF800EE926040E70
:102A5000EA22EECF04F0EECF05F0EECF06F0EFCF96
:102A600007F004C02CF005C02DF006C02EF007C002
:102A70002FF024C427F025C428F026C429F027C449
:102A80002AF0F7EC6CF027C000F028C001F029C054
:102A900002F02AC003F058C42CF059C42DF05AC4D7
:102AA0002EF05BC42FF000C027F001C028F002C058
:102AB00029F003C02AF0E1EC6DF027C02CF428C007
:102AC0002DF429C02EF42AC02FF41CEC6AF0040166
:102AD0000051040DF3CFE9FFF4CFEAFF800EE926A1
:102AE000040EEA22EECF04F0EECF05F0EECF06F0B2
:102AF000EFCF07F02CC42CF02DC42DF02EC42EF0F7
:102B00002FC42FF004C027F005C028F006C029F01C
:102B100007C02AF0F8EC6CF027C000F028C001F0E4
:102B200029C002F02AC003F004010051040DF3CFC4
:102B3000E9FFF4CFEAFF800EE926040EEA2200C086
:102B4000EEFF01C0EEFF02C0EEFF03C0EEFF100E6D
:102B500004010025040DF3CFE9FFF4CFEAFF800E56
:102B6000E926040EEA22EECF04F0EECF05F0EECF18
:102B700006F0EFCF07F004C02CF005C02DF006C022
:102B80002EF007C02FF028C427F029C428F02AC44B
:102B900029F02BC42AF0F7EC6CF027C000F028C015
:102BA00001F029C002F02AC003F05CC42CF05DC41F
:102BB0002DF05EC42EF05FC42FF000C027F001C0DE
:102BC00028F002C029F003C02AF0E1EC6DF027C024
:102BD0002CF428C02DF429C02EF42AC02FF41CECAC
:102BE0006AF0100E04010025040DF3CFE9FFF4CFC5
:102BF000EAFF800EE926040EEA22EECF04F0EECFC3
:102C000005F0EECF06F0EFCF07F02CC42CF02DC46A
:102C10002DF02EC42EF02FC42FF004C027F005C0D5
:102C200028F006C029F007C02AF0F8EC6CF027C0A5
:102C300000F028C001F029C002F02AC003F0100EF5
:102C400004010025040DF3CFE9FFF4CFEAFF800E65
:102C5000E926040EEA2200C0EEFF01C0EEFF02C02A
:102C6000EEFF03C0EEFF04010051040DF3CFE9FFB6
:102C7000F4CFEAFF800EE926040EEA22EECF00F040
:102C8000EECF01F0EECF02F0EFCF03F0100E040113
:102C90000025040DF3CFE9FFF4CFEAFF800EE9260B
:102CA000040EEA22EECF04F0EECF05F0EECF06F0F0
:102CB000EFCF07F004C02CF005C02DF006C02EF0B9
:102CC00007C02FF000C027F001C028F002C029F093
:102CD00003C02AF0F8EC6CF027C02CF428C02DF4C7
:102CE00029C02EF42AC02FF404010051040DF3CFA3
:102CF000E9FFF4CFEAFF800EE926040EEA22EECFC8
:102D000008F0EECF09F0EECF0AF0EFCF0BF008C0DD
:102D10002CF009C02DF00AC02EF00BC02FF040C4DB
:102D200027F041C428F042C429F043C42AF0E1EC62
:102D30006DF027C004F028C005F029C006F02AC0B5
:102D400007F0100E04010025040DF3CFE9FFF4CFC6
:102D5000EAFF800EE926040EEA22EECF10F0EECF55
:102D600011F0EECF12F0EFCF13F010C02CF011C025
:102D70002DF012C02EF013C02FF044C427F045C42C
:102D800028F046C429F047C42AF0E1EC6DF027C0D2
:102D90000CF028C00DF029C00EF02AC00FF00CC0B6
:102DA0002CF00DC02DF00EC02EF00FC02FF004C07F
:102DB00027F005C028F006C029F007C02AF0F8EC7B
:102DC0006CF027C000F028C001F029C002F02AC032
:102DD00003F02CC42CF02DC42DF02EC42EF02FC4E3
:102DE0002FF000C027F001C028F002C029F003C076
:102DF0002AF08EEC6DF027C040F428C041F429C0C1
:102E000042F42AC043F404010051040DF3CFE9FF5A
:102E1000F4CFEAFF800EE926040EEA22EECF08F096
:102E2000EECF09F0EECF0AF0EFCF0BF008C02CF098
:102E300009C02DF00AC02EF00BC02FF048C427F0B7
:102E400049C428F04AC429F04BC42AF0E1EC6DF0E3
:102E500027C004F028C005F029C006F02AC007F0FA
:102E6000100E04010025040DF3CFE9FFF4CFEAFFB3
:102E7000800EE926040EEA22EECF10F0EECF11F01C
:102E8000EECF12F0EFCF13F010C02CF011C02DF0E8
:102E900012C02EF013C02FF04CC427F04DC428F000
:102EA0004EC429F04FC42AF0E1EC6DF027C00CF0BD
:102EB00028C00DF029C00EF02AC00FF00CC02CF075
:102EC0000DC02DF00EC02EF00FC02FF004C027F063
:102ED00005C028F006C029F007C02AF0F8EC6CF015
:102EE00027C000F028C001F029C002F02AC003F07A
:102EF0002CC42CF02DC42DF02EC42EF02FC42FF096
:102F000000C027F001C028F002C029F003C02AF059
:102F10008EEC6DF027C048F428C049F429C04AF46B
:102F20002AC04BF440C42CF041C42DF042C42EF012
:102F300043C42FF02CC427F02DC428F02EC429F050
:102F40002FC42AF0F7EC6CF027C004F028C005F07D
:102F500029C006F02AC007F048C42CF049C42DF05F
:102F60004AC42EF04BC42FF004C027F005C028F04F
:102F700006C029F007C02AF0E1EC6DF027C000F090
:102F800028C001F029C002F02AC003F0040100515A
:102F9000040DF3CFE9FFF4CFEAFF6B0EE926050E2F
:102FA000EA2200C0EEFF01C0EEFF02C0EEFF03C048
:102FB000EEFF04010051040DF3CFE9FFF4CFEAFF67
:102FC0006B0EE926050EEA22EECF00F0EECF01F0FF
